:020000020000FC
:100000000C9400F118951895189518951895189551
:100010001895189518951895189518951895189578
:100020000C9421AF0C948CEA189518951895189596
:100030000C94E7AE0C943EAE189518950C9434AF22
:100040000C9423F0189518950C949EB41895189557
:10005000189518950C945BAF1895189518951895E8
:1000600018951895189518950C94AF5318951895E0
:1000700018951895189518950C941DB618951895FF
:100080000C94C0F018951895189518951F1C1F1EF4
:100090001F1E1F1F1E1F1E1F00000000038007C021
:1000A0000E401C00180038003000FF00FF00300038
:1000B0003000FF00FF003000380018001C000E4028
:1000C00007C003800000000000000000FC00FF00EB
:1000D000FF80FFC0E3C0E1C0E1C0E3C0FFC0FF801C
:1000E000FF00FC00E000E000E000E000E000E000D5
:1000F000E000E0000000000006091C081C090600E2
:10010000001E11111E10001E3F736060F8F860F8A9
:10011000F86060733F1E00000000000000FEFFC397
:10012000C3C3C3FFFEC0C0C00000417567203236A4
:1001300020323030390004050000010101030000C5
:10014000D8D2D0C8D52DCFD0C8CDD2000000000065
:1001500000000000C2E2EEE40A00D1E1F0EEF10A94
:1001600000D1F2F0E5EBEAE020E2EBE5E2EE0A0096
:10017000D1F2F0E5EBEAE020E2EFF0E0E2EE0A0097
:10018000CEF2ECE5EDE00A00D1F2F0E5EBEAE0209A
:10019000E2E2E5F0F50A00D1F2F0E5EBEAE020E278
:1001A000EDE8E70A00CFF0EEECEEF2EAE00A00D06C
:1001B000E5E3E8F1F2F00A00CAF3F0F12FDDEAE23C
:1001C0000A00CFE5F7E0F2FC0A00CAEEE40A00CA32
:1001D000EEEFE8FF0A00D8F22FD6E5EDE00A00D8EE
:1001E000F20A00C8F2EEE30A00D1E4E0F7E00A0008
:1001F0003E303C0A003E543C0A00CF2D0A00CF2B73
:100200000A00C7E0EFE8F1FC0A00C4E0F2E02FC208
:10021000F0E5ECFF0A00C0E2F2EE2FD4E0F1EEE2EE
:10022000EAE00A0030300A00C1EBEEEAE8F0EEE264
:10023000EAE020EAEBE0E2E8E0F2F3F0FB2000C7BE
:10024000E0EFE8F1FC0A00000102030405060708DC
:10025000090A0B0C0D0E0F10111213141516171896
:10026000191A1B1C1D1E1F20212223242526272886
:10027000292A2B2C2D2E2F30313233343536373876
:10028000393A3B3C3D3E3F40414243444546474866
:10029000494A4B4C4D4E4F50515253545556575856
:1002A000595A5B5C5D5E5F60616263C2EAEBFEF7B8
:1002B000E5ED20EDE0203234303020E1EEE4202086
:1002C0002000C2EAEBFEF7E5ED20EDE02034383007
:1002D0003020E1EEE420202000C2EAEBFEF7E5ED5D
:1002E00020EDE0203936303020E1EEE420202000FF
:1002F000C2EAEBFEF7E5ED20EDE020313932303097
:1003000020E1EEE4202000C2EAEBFEF7E5ED20ED6F
:10031000E020333834303020E1EEE4202000C2EA1F
:10032000EBFEF7E5ED20EDE020353736303020E10B
:10033000EEE4202000C2EAEBFEF7E5ED20EDE02040
:1003400031313532303020E1EEE42000C0D6CF3AF2
:10035000257520256C750A002020202020C4EEE1A0
:10036000F0EE20EFEEE6E0EBEEE2E0F2FC21202002
:1003700020202020002020202020D1EFE0F1E8E103
:10038000EE20E7E020EFEEEAF3EFEAF32120202071
:10039000200020202020202020C6E4E5EC20C2E020
:1003A000F120F1EDEEE2E021202020202020002AA3
:1003B0002A2A20CDD2D62027D8D2D0C8D52D4D2755
:1003C000202A2A2A2000202020202020202020202F
:1003D0002020C8D2CEC32020202020202020202072
:1003E000202000303033300000000000000000000A
:1003F0000000000000000000183C3C181800180025
:1004000066662400000000006C6CFE6CFE6C6C00E4
:10041000183E603C067C180000C6CC183066C6004A
:10042000386C3876DCCC76001818300000000000FC
:100430000C18303030180C0030180C0C0C18300030
:1004400000663CFF3C6600000018187E181800008B
:1004500000000000001818300000007E00000000BE
:100460000000000000181800060C183060C0800062
:100470007CC6CED6E6C67C001838181818187E0040
:100480007CC6061C3066FE007CC6063C06C67C00A8
:100490001C3C6CCCFE0C1E00FEC0C0FC06C67C00E2
:1004A0003860C0FCC6C67C00FEC60C183030300078
:1004B0007CC6C67CC6C67C007CC6C67E060C7800A0
:1004C000001818000018180000181800001818303C
:1004D000060C1830180C060000007E00007E00009C
:1004E0006030180C183060007CC60C18180018001A
:1004F0007CC6DEDEDEC07800386CC6FEC6C6C6002E
:10050000FC66667C6666FC003C66C0C0C0663C005B
:10051000F86C6666666CF800FE6268786862FE00D9
:10052000FE6268786860F0003C66C0C0CE663A0043
:10053000C6C6C6FEC6C6C6003C18181818183C0029
:100540001E0C0C0CCCCC7800E6666C786C66E60071
:10055000F06060606266FE00C6EEFEFED6C6C600B3
:10056000C6E6F6DECEC6C6007CC6C6C6C6C67C00DB
:10057000FC66667C6060F0007CC6C6C6C6CE7C0E9B
:10058000FC66667C6C66E6007CC660380CC67C0047
:100590007E7E5A1818183C00C6C6C6C6C6C67C0061
:1005A000C6C6C6C6C66C3800C6C6C6D6D6FE6C0061
:1005B000C6C66C386CC6C6006666663C18183C0039
:1005C000FEC68C183266FE003C30303030303C00C5
:1005D000C06030180C0602003C0C0C0C0C0C3C00EB
:1005E00010386CC60000000000000000000000FF92
:1005F00030180C00000000000000780C7CCC760065
:10060000E0607C666666DC0000007CC6C0C67C00DC
:100610001C0C7CCCCCCC760000007CC6FEC07C00E0
:100620003C6660F86060F000000076CCCC7C0CF892
:10063000E0606C766666E6001800381818183C0012
:10064000060006060666663CE060666C786CE600AE
:100650003818181818183C000000ECFED6D6D60042
:100660000000DC666666660000007CC6C6C67C00CC
:100670000000DC66667C60F0000076CCCC7C0C1E52
:100680000000DC766060F00000007EC07C06FC00AC
:100690003030FC3030361C000000CCCCCCCC7600A6
:1006A0000000C6C6C66C38000000C6D6D6FE6C0078
:1006B0000000C66C386CC6000000C6C6C67E06FCCC
:1006C00000007E4C18327E000E18187018180E00AC
:1006D00018181818181818007018180E1818700024
:1006E00076DC0000000000000000000000000000B8
:1006F00000000000000000000000000000000000FA
:1007000046A9A848080906000000000000000000F3
:1007100000000000000000000000000000000000D9
:1007200000000000000000000000000000000000C9
:100730000C123C103C10120C0000000000000000E5
:1007400000000000000000000000000000000000A9
:100750000000000000000000000000000000000099
:100760000000000000000000000000000000000089
:100770000000000000000000000000000000000079
:100780000000000000000000000000000000000069
:100790000000000000000000000000000000000059
:1007A0000000000000000000000000000000000049
:1007B0000000000000000000F15B55510000000047
:1007C0000000000000000000000000000000000029
:1007D0000000000000000000000000000000000019
:1007E0000000000000000000000000000000000009
:1007F00000000000000000000000000000000000F9
:1008000000000000000000000000000000000000E8
:1008100000000000000000000000000000000000D8
:1008200000000000000000000000000000000000C8
:1008300024FE6268786862FE1C22495551552A1CC4
:1008400000000000000000000000000000000000A8
:100850000000000000000000000000000000000098
:100860001C2259555955221C0000000000000000B0
:10087000000000000000000004041F0404001F002A
:100880000000000000000000000000000000000068
:100890000000000000000000000000000000000058
:1008A0000000000000000000000000000000000048
:1008B000480078CCFCC0780090D0D2F5B2B0970058
:1008C0000000000000000000000000000000000028
:1008D0000000000000000000000000000000000018
:1008E0000000000000000000000000000000000008
:1008F0003E66C6C6FEC6C600FE66607C6666FC0036
:10090000FC66667C6666FC00FE6660606060F00007
:100910001E3666666666FFC3FE6268786862FE0021
:10092000D6D67C387CD6D6007CC6063C06C67C0073
:10093000C6C6CEDEF6E6C60038C6CEDEF6E6C60091
:10094000E6666C786C66E6001E3666666666C6000D
:10095000C6EEFEFED6C6C600C6C6C6FEC6C6C600E3
:100960007CC6C6C6C6C67C00FEC6C6C6C6C6C6000F
:10097000FC6666667C60F0007CC6C0C0C0C67C00B9
:100980007E5A181818183C00C6C6C67E06C67C00DB
:100990007CD6D6D67C103800C6C66C386CC6C6006D
:1009A000CCCCCCCCCCCCFE06C6C6C67E0606060099
:1009B000D6D6D6D6D6D6FE00D6D6D6D6D6D6FF032F
:1009C000F0F0B03C36363C00C6C6C6F6DEDEF600B9
:1009D000F060607C66667C00788C063E068C780051
:1009E000DCD6D6F6D6D6DC007EC6C6C67E66C60087
:1009F0000000780C7CCC7600067CC07CC6C67C00EF
:100A00000000FC667C66FC000000FE666060F00092
:100A100000003C6C6C6CFEC600007CC6FEC07C0016
:100A20000000D67C387CD60000007CC61CC67C004A
:100A30000000C6CEDEF6E6000038C6CEDEF6E600E2
:100A40000000E66C786CE60000003E666666E60034
:100A50000000C6FEFED6C6000000C6C6FEC6C60022
:100A600000007CC6C6C67C000000FEC6C6C6C60026
:100A70000000FC66667C60F000007CC6C0C67C009E
:100A800000007E5A18183C000000C6C6C67E067CD0
:100A900000007CD6D67C10380000C66C386CC600CE
:100AA0000000CCCCCCCCFE060000C6C67E060600FC
:100AB0000000D6D6D6D6FE000000D6D6D6D6FF0386
:100AC0000000F0B03C363C000000C6C6F6DEF60082
:100AD0000000F0607C66FC0000007CC61EC67C0046
:100AE0000000DCD6F6D6DC0000007EC67E66C600BE
:100AF00000000000000000000000000000000000F6
:100B000000000000000000000000000000000000E5
:100B100000001818181818181818000018180000E5
:100B2000D8D8D8000000000000000000000000003D
:100B30000000000066FFE6666666FF6600000000D3
:100B40001010387CC6C0C078040606C67C38101069
:100B5000000043E6460C0C181830306267C20000F3
:100B60000000304848483048C5CECCCC4A3100005F
:100B700030301020000000000000000000000000E5
:100B80000000183860C0C0C0C0C0C0603818000085
:100B9000000030380C0606060606060C3830000049
:100BA0000000000000105438FE385410000000000F
:100BB00000000000000018187E7E181800000000D9
:100BC0000000000000000000000000003030102095
:100BD00000000000000000007E7E00000000000019
:100BE00000000000000000000000000030300000A5
:100BF00000000306060C0C181830306060C00000BE
:100C000000007CFEC6C6C6C6C6C6C6C6FE7C0000C0
:100C10000000183878181818181818187E7E000068
:100C200000007CFEC6060C183060C0C0FEFE00004E
:100C300000007CFEC606063C3C0606C6FE7C0000A4
:100C40000000060E1E3666C6C6FFFF06060600003A
:100C50000000FEFEC0C0FCFE060606C6FE7C0000CC
:100C600000007CFEC6C0C0FCFEC6C6C6FE7C0000FE
:100C70000000FEFE06060C18303030303030000028
:100C800000007CFEC6C6447CFEC6C6C6FE7C0000D4
:100C900000007CFEC6C6C6FE7E0606C6FE7C0000C0
:100CA0000000000000003030000000003030000084
:100CB0000000000000003030000000003030102044
:100CC00000000000040C18306030180C0400000014
:100CD000000000000000FE0000FE00000000000018
:100CE00000000000406030180C1830604000000028
:100CF00000007CFEC6C6060C183030003030000004
:100D000000007C828282BAAAAA9C8080807E000039
:100D10000000387CC6C6C6C6FEFEC6C6C6C60000F3
:100D20000000FCFEC6C6C6FCFEC6C6C6FEFC000031
:100D300000007CFEC6C0C0C0C0C0C0C6FE7C0000B3
:100D40000000F8FCC6C6C6C6C6C6C6C6FCF800008B
:100D50000000FEFEC0C0C0FCFCC0C0C0FEFE000023
:100D60000000FEFEC0C0C0FCFCC0C0C0C0C000008F
:100D700000007CFEC6C0C0DEDEC6C6C6FE7C00002B
:100D80000000C6C6C6C6C6FEFEC6C6C6C6C60000AB
:100D900000007E7E18181818181818187E7E00009B
:100DA00000001E1E0C0C0C0C0C0C0CCCFC78000073
:100DB0000000C2C6CCD8F0E0E0F0D8CCC6C200003B
:100DC0000000C0C0C0C0C0C0C0C0C0C0FEFE0000A7
:100DD000000082C6EEFED6D6C6C6C6C6C6C600008F
:100DE0000000C6C6C6E6F6DECEC6C6C6C6C600004B
:100DF00000007CFEC6C6C6C6C6C6C6C6FE7C0000CF
:100E00000000FCFEC6C6C6FEFCC0C0C0C0C00000DC
:100E100000007CC6C6C6C6C6C6D6D6D6D67C0804D2
:100E20000000FCFEC6C6C6FCFCC6C6C6C6C60000A0
:100E300000007CFEC6C0C0FC7E0606C6FE7C00002C
:100E400000007E7E181818181818181818180000B6
:100E50000000C6C6C6C6C6C6C6C6C6C6FE7C00005C
:100E60000000C6C6C6C6C6C6C6C6C66C38100000D8
:100E70000000C2C6C6C6C6C6D6D6D6FEEE44000020
:100E80000000C6C6C66C3838386CC6C6C6C6000078
:100E90000000C3C3C3C3663C181818181818000014
:100EA0000000FEFE06060C183060C0C0FEFE00000A
:100EB0000000787860606060606060607878000052
:100EC0000000C06060303018180C0C0606030000EB
:100ED00000003C3C0C0C0C0C0C0C0C0C3C3C0000C2
:100EE0000010386CC6000000000000000000000088
:100EF0000000000000000000000000000000FEFEF6
:100F00000030302010000000000000000000000051
:100F10000000000000787C0C7CFCCCCCFE7E000045
:100F20000000C0C0C0C0FCFEC6C6C6C6FEFC0000B5
:100F300000000000007CFEC6C0C0C0C6FE7C0000F1
:100F40000000060606067EFEC6C6C6C6FE7E000079
:100F500000000000007CFEC6C6FEC0C6FE7C00008D
:100F600000001C3C3030FCFC3030303030300000B1
:100F700000000000007EFEC6C6C6FE7E06C6FE7CE1
:100F80000000C0C0C0C0FCFEC6C6C6C6C6C60000C3
:100F90000000181800787818181818187E7E0000BD
:100FA00000000C0C003C3C0C0C0C0C0C0C0C7C7869
:100FB0000000C0C0C0C6CCD8F0E0F0D8CCC600005D
:100FC0000000707030303030303030303C1C000069
:100FD00000000000006CFED6D6D6D6D6D6D60000CD
:100FE0000000000000B8FCC6C6C6C6C6C6C60000E3
:100FF00000000000007CFEC6C6C6C6C6FE7C00001F
:101000000000000000BCFEC6C6C6C6FEFCC0C0C0D4
:1010100000000000007AFEC6C6C6C6FE7E060606B2
:101020000000000000BCFEC6C0C0C0C0C0C00000C0
:1010300000000000007EFEC6C07C06C6FEFC00006C
:10104000000000303030FCFC303030303C1C000000
:101050000000000000C6C6C6C6C6C6C6FE7A0000AE
:101060000000000000C6C6C6C6C6C66C3810000028
:101070000000000000C6C6C6C6C6D6D6FE6C00007C
:101080000000000000C6C66C3810386CC6C60000F0
:101090000000000000C6C6C6C6C6FE7E06067E7CF0
:1010A0000000000000FEFE0C183060C0FEFE0000D4
:1010B00000000C181818187018181818180C0000D0
:1010C00000001818181818181818181818181818D0
:1010D000000060303030301C303030303060000084
:1010E00000000062D68C000000000000000000003C
:1010F000000000000010386CC6C6C6C6C6FE000060
:1011000000000000000000000000000000000000DF
:1011100000000000000000000000000000000000CF
:10112000609090906E1B1B181818181B1B0E000067
:1011300000000000000000000000000000000000AF
:10114000000000000000000000000000000000009F
:10115000000000000000000000000000000000008F
:10116000000000000000000000000000000000007F
:10117000000000000000000000000000000000006F
:1011800000000C163030307C207C303030160C00E3
:10119000000000000000000000000000000000004F
:1011A000000000000000000000000000000000003F
:1011B000000000000000000000000000000000002F
:1011C000000000000000000000000000000000001F
:1011D000000000000000000000000000000000000F
:1011E00000000000000000000000000000000000FF
:1011F00000000000000000000000000000000000EF
:1012000000000000000000000000000000000000DE
:1012100000000000000000000000000000000000CE
:1012200000000000000000000000000000000000BE
:1012300000000000000000000000000000000000AE
:10124000000000000000000000000000000000009E
:10125000000000000000000000000000000000008E
:10126000000000000000000000000000000000007E
:10127000000000000000000000000000000000006E
:10128000000000000000000000000000000000005E
:1012900000F15B555100000000000000000000005C
:1012A000000000000000000000000000000000003E
:1012B000000000000000000000000000000000002E
:1012C000000000000000000000000000000000001E
:1012D000000000000000000000000000000000000E
:1012E00000000000000000000000000000000000FE
:1012F00000000000000000000000000000000000EE
:1013000000000000000000000000000000000000DD
:1013100000000000000000000000000000000000CD
:1013200000000000000000000000000000000000BD
:1013300000000000000000000000000000000000AD
:10134000000000000000000000000000000000009D
:10135000000000000000000000000000000000008D
:10136000000000000000000000000000000000007D
:10137000000000000000000000000000000000006D
:10138000C600FEFEC0C0C0FEFEC0C0C0FEFE000023
:10139000001C224955515549221C00000000000044
:1013A000000000000000000000000000000000003D
:1013B000000000000000000000000000000000002D
:1013C000000000000000000000000000000000001D
:1013D000000000000000000000000000000000000D
:1013E000001C2259555955221C0000000000000025
:1013F00000000000000000000000000000000000ED
:1014000000000000000000000000000000000000DC
:101410000000003030FCFC303000FCFC000000001C
:1014200000000000000000000000000000000000BC
:1014300000000000000000000000000000000000AC
:10144000000000000000000000000000000000009C
:10145000000000000000000000000000000000008C
:10146000000000000000000000000000000000007C
:10147000000000000000000000000000000000006C
:10148000000000006C007CC6C6C6FEC0C0C07C0068
:10149000000090909090D0D0F0B2B59592909700C7
:1014A000000000000000000000000000000000003C
:1014B000000000000000000000000000000000002C
:1014C000000000000000000000000000000000001C
:1014D000000000000000000000000000000000000C
:1014E00000000000000000000000000000000000FC
:1014F00000000000000000000000000000000000EC
:101500000000387CC6C6C6C6FEFEC6C6C6C60000FB
:101510000000FEFEC0C0FCFEC6C6C6C6FEFC000043
:101520000000FCFEC6C6C6FCFEC6C6C6FEFC000029
:101530000000FEFEC6C0C0C0C0C0C0C0C0C0000029
:1015400000003E2626262626266666667EFFC38186
:101550000000FEFEC0C0C0FCFCC0C0C0FEFE00001B
:101560000000D6D654547C387CD6D6D6D6D60000C9
:1015700000007CFEC606041C1E0606C6FE7C00009B
:101580000000C6C6C6CEDEF6E6C6C6C6C6C60000A3
:101590006C3800C6C6C6CEDEF6E6C6C6C6C60000B5
:1015A0000000C2C6CCD8F0E0E0F0D8CCC6C2000043
:1015B00000003E3E2626262626262626E6C60000D3
:1015C000000082C6EED6D6D6C6C6C6C6C6C60000BF
:1015D0000000C6C6C6C6C6FEFEC6C6C6C6C6000053
:1015E00000007CFEC6C6C6C6C6C6C6C6FE7C0000D7
:1015F0000000FEFEC6C6C6C6C6C6C6C6C6C6000033
:101600000000FCFEC6C6C6FEFCC0C0C0C0C00000D4
:1016100000007CFEC6C0C0C0C0C0C0C6FE7C0000CA
:101620000000FF18181818181818181818180000B3
:101630000000C6C6C6C6C6C67E3E06C6FE7C000004
:101640000000107CFED6D6D6D6D6FE7C1010000048
:101650000000C6C6C66C3838386CC6C6C6C60000A0
:101660000000CCCCCCCCCCCCCCCCCCCCFCFE06067C
:101670000000C6C6C6C6C6FE7E06060606060000F2
:101680000000D6D6D6D6D6D6D6D6D6D6FEFE000002
:101690000000D6D6D6D6D6D6D6D6D6D6FEFF0303EB
:1016A0000000F0B0B0303C3E323232323E3C0000FE
:1016B0000000C2C2C2C2F2FACACACACAFAF2000022
:1016C0000000606060607C7E626262627E7C00001E
:1016D0000000387C6606061E1E0606667C38000082
:1016E0000000CCD2D2D2D2F2F2D2D2D2D2CC0000EE
:1016F00000007EFEC6C6C67E3E66C6C6C6C60000E2
:101700000000000000780C0C7CFCCCCCCC7E0000EF
:101710000000047CFCC0F8FCC6C6C6C67C380000CD
:1017200000000000007C7E66667C66667E7C0000B1
:1017300000000000007C7C6C606060606060000005
:1017400000000000003C2C2C2C2C2C2C6CFEFE826B
:1017500000000000007CFEC6C6FEC0C6FE7E000083
:101760000000000000D6D6547C387CD6D6D60000C7
:1017700000000000007C7E46041C06467E7C0000C3
:101780000000000000C6C6CEDEF6E6C6C6C60000F3
:1017900000006C3800C6C6CEDEF6E6C6C6C600003F
:1017A000000000000062666C7870786C6662000071
:1017B00000000000003E262626262626E6C600005B
:1017C0000000000000C6EEFED6C6C6C6C6C60000B3
:1017D00000000000006666667E7E66666666000043
:1017E00000000000007CFEC6C6C6C6C6FE7C000027
:1017F00000000000007E7E66666666666666000023
:101800000000000000FCFEC6C6C6C6C6FEFCC0C086
:1018100000000000007CFEC6C0C0C0C6FE7C000008
:101820000000000000FCFC30303030303030000070
:101830000000000000CCCCCCCCFC7C1838F0E000E0
:1018400000001010107CFED6D6D6D6FE7C101010EC
:101850000000000000C6C66C3810386CC6C6000018
:101860000000000000C6C6C6C6C6C6C6FEFF03030B
:101870000000000000CCCCCCFC7C0C0C0C0C00005C
:101880000000000000D6D6D6D6D6D6D6FEFE000082
:101890000000000000D6D6D6D6D6D6D6FEFF03036B
:1018A0000000000000F0B0303C363636363C000018
:1018B0000000000000C2C2C2F2DADADADAF2000096
:1018C00000000000006060607C666666667C000068
:1018D00000000000003C7E46061E06467E3C0000DE
:1018E0000000000000CCDED2D2F2D2D2DECC00006A
:1018F00000000000007CFCCCCC7C3C6CCCCC00001C
:1019000000000000000000000000000000000000D7
:1019100000000000000000000000000000000000C7
:1019200000000000000000000000000000000000B7
:1019300000000000000000000000000000000000A7
:101940000000000000000000000000000000000097
:101950000000000000000000000000000000000087
:101960000000000000000C001E001E001E001E00F3
:101970001E001E001E001E001E001E000C000000A7
:1019800000001E001E001E001E00000000000000DF
:1019900000000000F3C0F3C0F3C0F3C0F3C071C097
:1019A0006180C30082000000000000000000000011
:1019B0000000000000000000000000000000000027
:1019C0000000000019801980198019803300FFC0C1
:1019D000FFC0FFC0330033006600FFC0FFC0FFC080
:1019E000660066006600CC00CC000000000000002D
:1019F000000000000C003F007F80FFC0EDC0EDC084
:101A0000EC00EC007C007F003F800FC00DC0EDC0FB
:101A1000EDC0EDC07F807F803F000C000000000023
:101A2000000000007000F8C0D9C0F9C073800380C6
:101A3000070007000E000E001C001C0038003800D4
:101A400070007380E7C0E6C0C7C0038000000000DC
:101A5000000000001E003F007F8073807380738051
:101A60007F803F001E003E007C00FEC0F7C0E3C048
:101A7000E380E380F780FFC07FC03CC0000000002F
:101A8000000000001E001E001E001E001E000E00B2
:101A90000E001C0018000000000000000000000004
:101AA0000000000000000000000000000000000036
:101AB0000000000003000F000E001C001C003C0092
:101AC0003800380038003800380038003800380056
:101AD0003C001C001C000E000F0003000000000072
:101AE0000000000030003C001C000E000E000F0043
:101AF00007000700070007000700070007000700AE
:101B00000F000E000E001C003C0030000000000022
:101B1000000000000000000000000C001E001E007D
:101B2000CCC0FFC0FFC0DE401F007F807380330049
:101B300000000000000000000000000000000000A5
:101B400000000000000000001E001E001E001E001D
:101B5000FFC0FFC0FFC0FFC01E001E001E001E0011
:101B60000000000000000000000000000000000075
:101B70000000000000000000000000000000000065
:101B8000000000000000000000001E001E001E00FB
:101B90001E001E000E000E001C00180000000000B9
:101BA0000000000000000000000000000000000035
:101BB000FFC0FFC0FFC0FFC0000000000000000029
:101BC0000000000000000000000000000000000015
:101BD0000000000000000000000000000000000005
:101BE00000000000000000000000000000000000F5
:101BF0001E003F003F003F003F001E0000000000AD
:101C000000000000000000C001C001C0038003808C
:101C1000070007000E000E001C001C0038003800F2
:101C200070007000E000E000C00000000000000054
:101C3000000000001E003F007F807380E1C0E1C013
:101C4000E1C0E1C0E1C0E1C0E1C0E1C0E1C0E1C08C
:101C5000E1C0E1C073807F803F001E0000000000F3
:101C60000000000007000F001F003F007F0077000A
:101C7000670047000700070007000700070007008C
:101C8000070007000700070007000700000000002A
:101C9000000000003F007F80FFC0F3C0E1C0E1C052
:101CA00001C001C001C0038007800F001E003C007E
:101CB0007800F000E000FFC0FFC0FFC0000000009F
:101CC000000000001F003F807FC073C061C001C0E2
:101CD00001C003800F000E000F80038001C001C00F
:101CE00001C0C1C0E3C0FF807F803E000000000053
:101CF000000000000380078007800F801F801F8086
:101D00003F807B807380E380E380FFC0FFC0FFC023
:101D100003800380038003800380038000000000B1
:101D2000000000003F807F807F8070007000E00036
:101D3000E000EF00FF80FFC0F3C0E1C001C001C0C0
:101D400001C0C1C0E380FF807F003E0000000000B2
:101D5000000000001E003F007F807380E180E000F3
:101D6000E000EE00FF00FF80F3C0E1C0E1C0E1C091
:101D7000E1C0E1C0F3C07F803F001E000000000012
:101D800000000000FFC0FFC0FFC001C0038003804F
:101D9000070007000E000E001C001C003800380071
:101DA000700070007000E000E000E0000000000043
:101DB000000000001E003F007F8073806180618012
:101DC000618073803F003F007F80F3C0E1C0E1C0CD
:101DD000E1C0E1C0F3C07F803F001E0000000000B2
:101DE000000000001E007F807F80F3C0E1C0E1C0E2
:101DF000E1C0E1C0E1C0F3C07FC07FC03FC001C00F
:101E000001C0C1C0E380FF807F003E0000000000F1
:101E1000000000000000000000003C003C003C000E
:101E20003C00000000000000000000003C003C00FE
:101E30003C003C000000000000000000000000002A
:101E4000000000000000000000003C003C003C00DE
:101E50003C00000000000000000000003C003C00CE
:101E60003C003C000C001C0038000000000000009A
:101E700000000000000000800180038007800F0048
:101E80001E003C007800F000E000F00078003C000C
:101E90001E000F000780038001800080000000000A
:101EA0000000000000000000000000000000FF80B3
:101EB000FF80FF80000000000000FF80FF80FF80A7
:101EC0000000000000000000000000000000000012
:101ED00000000000000040006000700078003C003E
:101EE0001E000F00078003C001C003C007800F0061
:101EF0001E003C0078007000600040000000000000
:101F0000000000001E003F007F80F380E3C0E1C0BE
:101F1000E1C001C001C003C0038007800F001E00A4
:101F20001C00000000001C001C001C000000000041
:101F3000000000003F007F80FFC0E1C0CCC0DEC0D9
:101F4000DEC0D2C0D2C0D2C0D2C0D2C0DEC0DEC0DD
:101F5000CF80C700E040FFC07FC03F80000000008E
:101F6000000000000FC01FC01FC01DC01DC039C031
:101F700039C039C039C039C071C071C07FC07FC09D
:101F80007FC0FFC0E1C0E1C0E1C0E1C000000000CF
:101F900000000000FE00FF00FF80E780E380E38098
:101FA000E380E780FF80FF00FF80E3C0E1C0E1C085
:101FB000E1C0E1C0E3C0FFC0FF80FF0000000000FF
:101FC000000000001E003F007F807FC0F1C0E0C025
:101FD000E0C0E000E000E000E000E000E000E0C081
:101FE000E0C0F1C07FC07F803F001E000000000005
:101FF00000000000FC00FE00FF00FF80E780E3C05F
:10200000E1C0E1C0E1C0E1C0E1C0E1C0E1C0E3C0C6
:10201000E380E780FF80FF00FE00FC00000000007E
:1020200000000000FFC0FFC0FFC0FFC0E000E000F4
:10203000E000E000FF00FF00FF00FF00E000E00024
:10204000E000E000FFC0FFC0FFC0FFC000000000D4
:1020500000000000FFC0FFC0FFC0FFC0E000E000C4
:10206000E000E000FF80FF80FF80E000E000E00093
:10207000E000E000E000E000E000E0000000000020
:10208000000000001E003F007F807F80F1C0E1C0A3
:10209000E000E000E000E7C0E7C0E7C0E7C0E7C05D
:1020A000E0C0F1C07FC07F803F801E0000000000C4
:1020B00000000000E1C0E1C0E1C0E1C0E1C0E1C05A
:1020C000E1C0E1C0FFC0FFC0FFC0FFC0E1C0E1C090
:1020D000E1C0E1C0E1C0E1C0E1C0E1C0000000003A
:1020E000000000000E000E000E000E000E000E009C
:1020F0000E000E000E000E000E000E000E000E0070
:102100000E000E000E000E000E000E00000000007B
:102110000000000001C001C001C001C001C001C039
:1021200001C001C001C001C001C001C0E1C0E1C0E7
:10213000E1C0F3C07FC07FC03F801F0000000000EF
:1021400000000000E1C0E1C0E380E380E700E700B9
:10215000EE00FE00FC00FE00EE00EF00E700E7806E
:10216000E380E380E3C0E1C0E1C0E1C00000000023
:1021700000000000E000E000E000E000E000E0001F
:10218000E000E000E000E000E000E000E000E0004F
:10219000E000E000FFC0FFC0FFC0FFC00000000083
:1021A00000000000C0C0E1C0E1C0E1C0F3C0F3C066
:1021B000FFC0FFC0FFC0FFC0EDC0EDC0EDC0EDC06F
:1021C000EDC0E1C0E1C0E1C0E1C0E1C0000000003D
:1021D00000000000E1C0E1C0E1C0F1C0F1C0F9C001
:1021E000F9C0F9C0FDC0EDC0EDC0EFC0E7C0E7C069
:1021F000E7C0E3C0E3C0E1C0E1C0E1C0000000000F
:10220000000000001E003F007F807F80F3C0E1C01F
:10221000E1C0E1C0E1C0E1C0E1C0E1C0E1C0E1C0B6
:10222000E1C0F3C07F807F803F001E0000000000FF
:1022300000000000FC00FF00FF80FFC0E3C0E1C021
:10224000E1C0E3C0FFC0FF80FF00FC00E000E00051
:10225000E000E000E000E000E000E000000000003E
:10226000000000003C007E007F00FF00F780E3805C
:10227000E380E380E380E380E380E380EB80EF8032
:10228000EF80EF007F007F803DC019C0000000009C
:1022900000000000FC00FF00FF80FFC0E3C0E1C0C1
:1022A000E1C0E3C0FF80FF00FE00FF00E700E78021
:1022B000E380E380E3C0E1C0E1C0E1C000000000D2
:1022C000000000001E003F003F807FC07BC071C047
:1022D00071C078007C003F001F800FC003C0E1C0C8
:1022E000E1C0F3C07FC07F803F801E00000000007F
:1022F00000000000FFC0FFC0FFC0FFC01E001E00A6
:102300001E001E001E001E001E001E001E001E00DD
:102310001E001E001E001E001E001E000000000009
:1023200000000000E1C0E1C0E1C0E1C0E1C0E1C0E7
:10233000E1C0E1C0E1C0E1C0E1C0E1C0E1C0E1C095
:10234000E1C0F3C07F807F803F001E0000000000DE
:1023500000000000E1C0E1C0E1C0E1C0E1806180B7
:102360006180738073807380738033003300330027
:102370003F001E001E001E000C000C0000000000AC
:1023800000000000E1C0E1C0E1C0E1C0E1C0EDC07B
:10239000EDC0EDC0EDC0EDC0EDC0EDC0EDC0FFC0C3
:1023A000FFC07F80738073806180618000000000C7
:1023B00000000000E1C0E1C0E1C0E1C073807380B3
:1023C00073803F001E001E001E003F007F80738050
:1023D0007380E1C0E1C0E1C0E1C0E1C000000000E5
:1023E00000000000E1C0E1C0E1C0E1C07380738083
:1023F00073003F001E001E000C000C000C000C00BF
:102400000C000C000C000C000C000C000000000084
:10241000000000003FC03FC03FC03FC001C003807C
:102420000380070007000E000E001C001C0038008F
:10243000380070007FC07FC07FC07FC000000000F8
:10244000000000000F000F000C000C000C000C003E
:102450000C000C000C000C000C000C000C000C001C
:102460000C000C000C000C000F000F00000000001E
:10247000000018001800180018000C000C000C00D8
:102480000C0006000600060006000300030003001F
:102490000300018001800180018000000000000035
:1024A00000000F000F0003000300030003000300FF
:1024B0000300030003000300030003000300030004
:1024C0000300030003000F000F00000000000000E5
:1024D000000006000F000F000F00198019801980FE
:1024E00030C00000000000000000000000000000FC
:1024F00000000000000000000000000000000000DC
:1025000000000000000000000000000000000000CB
:1025100000000000000000000000000000000000BB
:1025200000000000FFC0FFC0FFC00000000000006E
:10253000000006000600060006000600000000007D
:10254000000000000000000000000000000000008B
:10255000000000000000000000000000000000007B
:102560000000000000000000000000003E007F00AE
:10257000FF80C78003801F807F80FF80E780C3804B
:10258000C380E780FF807FC039C0000000000000EA
:102590000000E000E000E000E000E000EF00FF806D
:1025A000FF80F3C0E1C0E1C0E1C0E1C0E1C0E1C033
:1025B000E1C0F3C0FF80FF80EF00000000000000DA
:1025C0000000000000000000000000003F007F80CD
:1025D000FF80F3C0E1C0E000E000E000E000E000C8
:1025E000E1C0F3C0FF807F803F00000000000000DA
:1025F000000001C001C001C001C001C03DC07FC0DA
:102600007FC0F3C0E1C0E1C0E1C0E1C0E1C0E1C012
:10261000E1C0F3C07FC07FC03DC0000000000000EB
:102620000000000000000000000000003F007F806C
:102630007F80F3C0E1C0FFC0FFC0FFC0E000E0004A
:10264000E1C0F3C07F807F803F00000000000000F9
:1026500000000F801F801F801C001C007F007F0077
:102660007F007F001C001C001C001C001C001C00C4
:102670001C001C001C001C001C00000000000000CE
:10268000000000000000000000003DC07FC0FFC04F
:10269000F3C0E1C0E1C0E1C0E1C0F3C0FFC07FC052
:1026A0003FC001C0E3C0FFC07F8000000000000009
:1026B00000007000700070007000700077007F8074
:1026C0007FC07BC071C071C071C071C071C071C06A
:1026D00071C071C071C071C071C000000000000005
:1026E00000001C001C001C00000000001C001C005E
:1026F0001C001C001C001C001C001C001C001C00FA
:102700001C001C001C001C001C000000000000003D
:1027100000001C001C001C00000000001C001C002D
:102720001C001C001C001C001C001C001C001C00C9
:102730001C001C007C007C007800000000000000F1
:102740000000E000E000E000E000E000E1C0E3C0E5
:10275000E780E700EE00FC00FC00FE00EE00E70072
:10276000E700E380E3C0E1C0E1C00000000000003A
:1027700000001C001C001C001C001C001C001C0095
:102780001C001C001C001C001C001C001C001C0069
:102790001C001C001C001C001C00000000000000AD
:1027A000000000000000000000000000DB80FFC00F
:1027B000FFC0FFC0DDC0CCC0CCC0CCC0CCC0CCC042
:1027C000CCC0CCC0CCC0CCC0CCC00000000000004D
:1027D000000000000000000000000000EE00FF808C
:1027E000FFC0FFC0F3C0E1C0E1C0E1C0E1C0E1C093
:1027F000E1C0E1C0E1C0E1C0E1C0000000000000B4
:102800000000000000000000000000003F007F808A
:10281000FFC0F3C0E1C0E1C0E1C0E1C0E1C0E1C080
:10282000E1C0F3C0FFC07F803F0000000000000057
:102830000000000000000000EF00FF80FFC0FBC0B0
:10284000F1C0F1C0F1C0F1C0FBC0FFC0FF80EF00DC
:10285000E000E000E000E000E00000000000000018
:102860000000000000000000000000001DC07FC04C
:102870007FC0F3C0E1C0E1C0E1C0E1C0F3C07FC0F0
:102880007FC01FC001C001C001C0000000000000E7
:10289000000000000000000000000000E3C0FFC0D6
:1028A000FFC0F800F000E000E000E000E000E00021
:1028B000E000E000E000E000E000000000000000B8
:1028C0000000000000000000000000003F007F80CA
:1028D000FFC0F1C0E000F0007C003F800FC003C0EB
:1028E00001C0E3C0FFC07F803F0000000000000087
:1028F0000000000004000C001C001C003F003F0012
:102900003F001C001C001C001C001C001C001C00C4
:102910001C001C001F001F000F0000000000000032
:10292000000000000000000000000000E1C0E1C065
:10293000E1C0E1C0E1C0E1C0E1C0E1C0E1C0E1C08F
:10294000E1C0F3C0FFC07FC03DC000000000000038
:10295000000000000000000000000000E1C0E1C035
:10296000E1C0E1C0E1C0F3C07380738073803F00B9
:102970003F001E001E000C000C00000000000000C4
:10298000000000000000000000000000C0C0C0C047
:10299000CCC0CCC0EDC0EDC0EDC06D806D807F803F
:1029A0007F807F803F003300330000000000000084
:1029B000000000000000000000000000E1C0E1C0D5
:1029C000E1C073803F001E001E001E001E003F007D
:1029D0007F80F3C0E1C0E1C0E1C000000000000062
:1029E000000000000000000000000000E1C0E1C0A5
:1029F00071C071C071C03B803B803B001F001F0055
:102A00000E001E007C007C0078000000000000002A
:102A1000000000000000000000000000FFC0FFC038
:102A2000FFC003C0078007800F001E001C003C0091
:102A30007800F000FFC0FFC0FFC0000000000000F1
:102A4000000007000F000C000C000C000C000C0034
:102A50001C003C0030003C001C000C000C000C0072
:102A60000C000C000C000F0007000000000000002C
:102A7000000006000600060006000600060006002C
:102A80000600060006000600060006000600060016
:102A90000600060006000600060000000000000018
:102AA00000000E000F0003000300030003000300FA
:102AB000038001C000C001C00380030003000300C5
:102AC0000300030003000F000E00000000000000E0
:102AD00000000000000000000000000000003800BE
:102AE0007E2047E001C00000000000000000000060
:102AF00000000000000000000000000000000000D6
:102B000000000000000000000000000000000000C5
:102B100000000000000000000000000000000000B5
:102B200000000000000000000000000000000000A5
:102B30000000000000000000000000000000000095
:102B40000000000000000000000000000000000085
:102B50000000000000000000000000000000000075
:102B60000000000000000000000000000000000065
:102B70000000000000000000000000000000000055
:102B80000000000000000000000000000000000045
:102B90006000F1C093E097F0F7706E300E101C00EB
:102BA0001C0018001800180018001C001C000E1053
:102BB0000E10077007F003E001C0000000000000E5
:102BC0000000000000000000000000000000000005
:102BD00000000000000000000000000000000000F5
:102BE00000000000000000000000000000000000E5
:102BF00000000000000000000000000000000000D5
:102C000000000000000000000000000000000000C4
:102C100000000000000000000000000000000000B4
:102C200000000000000000000000000000000000A4
:102C30000000000000000000000000000000000094
:102C40000000000000000000000000000000000084
:102C50000000000000000000000000000000000074
:102C60000000000000000000000000000000000064
:102C70000000000000000000000000000000000054
:102C80000000000000000000000000000000000044
:102C90000000000000000000000000000000000034
:102CA0000000000000000000000000000000000024
:102CB0000000038007C00E401C00180038003000E0
:102CC000FF00FF0030003000FF00FF003000380040
:102CD00018001C000E4007C0038000000000000028
:102CE00000000000000000000000000000000000E4
:102CF00000000000000000000000000000000000D4
:102D000000000000000000000000000000000000C3
:102D100000000000000000000000000000000000B3
:102FE0007E20136012A012A01220122012200000D6
:102FF00000000000000000000000000000000000D1
:1030000000000000000000000000000000000000C0
:1030100000000000000000000000000000000000B0
:1030200000000000000000000000000000000000A0
:1032B0000000738073800000FFC0FFC0FFC0FFC02C
:1032C000E000E000E000FF00FF00FF00E000E000A1
:1032D000E000FFC0FFC0FFC0FFC000000000000012
:1032E0000F00108020404F20482048204F202040D1
:1032F00010800F000000000000000000000000002F
:1033000000000000000000000000000000000000BD
:1033100000000000000000000000000000000000AD
:10332000000000000000000000000000000000009D
:10333000000000000000000000000000000000008D
:10334000000000000000000000000000000000007D
:10335000000000000000000000000000000000006D
:10336000000000000000000000000000000000005D
:10337000000000000000000000000000000000004D
:10338000000000000000000000000000000000003D
:10339000000000000000000000000000000000002D
:1033A000000000000000000000000000000000001D
:1033B000000000000000000000000000000000000D
:1033C00000000000000000000000000000000000FD
:1033D0000F00108020404E2049204E2049202040E0
:1033E00010800F000000000000000000000000003E
:1033F00000000000000000000000000000000000CD
:1034000000000000000000000000000000000000BC
:1034100000000000000000000000000000000000AC
:10342000000000000000000000000000000000009C
:10343000000000000000000000000000000000008C
:10344000000000000000000000000000000000007C
:10345000000000000000000000000000000000006C
:1034600000000000000000000000060006001F80B1
:103470001F8006000600000000001F801F80000063
:10348000000000000000000000000000000000003C
:10349000000000000000000000000000000000002C
:1034A000000000000000000000000000000000001C
:1034B000000000000000000000000000000000000C
:1034C00000000000000000000000000000000000FC
:1034D00000000000000000000000000000000000EC
:1034E00000000000000000000000000000000000DC
:1034F00000000000000000000000000000000000CC
:1035000000000000000000000000000000000000BB
:1035100000000000000000000000000000000000AB
:10352000000000000000000000000000000000009B
:10353000000000000000000000000000000000008B
:10354000000000000000000000000000000000007B
:10355000000000000000000000000000000000006B
:10356000000000000000000000000000000000005B
:10357000000000000000000000000000000000004B
:10358000000000000000000000000000000000003B
:10359000000000000000000000000000000000002B
:1035A000000000000000000000000000000000001B
:1035B00000000000330033003300000000003F0033
:1035C0007F807F80F3C0FFC0FFC0FFC0E000E0004D
:1035D000E1C0F3C07F807F803F000000000000005A
:1035E0000000CC00CC00CC00CDC0CDC0CDC0ED40A3
:1035F000EDC0FC80FC00FDC0DD00DC00CC00CC0098
:10360000CC00CC00CC00CC00CC00000000000000BE
:1036100000000000000000000000000000000000AA
:10362000000000000000000000000000000000009A
:10363000000000000000000000000000000000008A
:10364000000000000000000000000000000000007A
:10365000000000000000000000000000000000006A
:10366000000000000000000000000000000000005A
:10367000000000000000000000000000000000004A
:10368000000000000000000000000000000000003A
:10369000000000000000000000000000000000002A
:1036A000000000000000000000000000000000001A
:1036B000000000000000000000000000000000000A
:1036C00000000000000000000000000000000000FA
:1036D00000000000000000000000000000000000EA
:1036E00000000000000000000000000000000000DA
:1036F00000000000000000000000000000000000CA
:1037000000000000000000000000000000000000B9
:1037100000000000000000000000000000000000A9
:103720000000000000000000000000000000000099
:1037300000000FC01FC01FC01DC01DC039C039C050
:1037400039C039C039C071C071C07FC07FC07FC06F
:10375000FFC0E1C0E1C0E1C0E1C000000000000026
:103760000000FF80FF80FF80E000E000E000E0005C
:10377000FE00FF00FF80FFC0E3C0E1C0E1C0E1C088
:10378000E3C0FFC0FF80FF80FE00000000000000DB
:103790000000FE00FF00FF80E780E380E380E3801D
:1037A000E780FF80FF00FF80E3C0E1C0E1C0E1C02F
:1037B000E1C0E3C0FFC0FF80FF0000000000000088
:1037C0000000FFC0FFC0FFC0FFC0E000E000E0005D
:1037D000E000E000E000E000E000E000E000E000E9
:1037E000E000E000E000E000E00000000000000079
:1037F00000003F803F803F803B803B803B803B80A0
:103800003B807B8073807380738073807380738050
:10381000FFC0FFC0FFC0E1C0E1C000000000000029
:103820000000FFC0FFC0FFC0FFC0E000E000E000FC
:10383000E000FF00FF00FF00FF00E000E000E0000C
:10384000E000FFC0FFC0FFC0FFC00000000000009C
:103850000000CCC0CCC0EDC0EDC0EDC06D806D806F
:103860003F001E003F007F806D806D80EDC0EDC089
:10387000EDC0EDC0CCC0CCC0CCC00000000000004A
:1038800000003E007F00FF00FF80E780C380438090
:1038900007801F001F800F8001C001C0C1C0C1C0D0
:1038A000E3C0FFC0FFC07F801E00000000000000DA
:1038B0000000E1C0E1C0E1C0E1C0E3C0E3C0E7C097
:1038C000E7C0EFC0EFC0FDC0F9C0F9C0F1C0F1C062
:1038D000E1C0E1C0E1C0E1C0E1C0000000000000C3
:1038E0000000DEC0DEC0CCC0C0C0E1C0E1C0E3C0AB
:1038F000E7C0E7C0EFC0FDC0F9C0F9C0F1C0F1C03A
:10390000E1C0E1C0E1C0E1C0E1C000000000000092
:103910000000E1C0E1C0E380E380E700E700EE00E3
:10392000FE00FC00FE00EE00EF00E700E780E38011
:10393000E380E3C0E1C0E1C0E1C00000000000009E
:1039400000003FC03FC03FC03FC039C039C039C090
:1039500039C039C039C039C039C039C039C039C09F
:1039600039C039C0F9C0F1C0E1C00000000000005A
:103970000000C0C0E1C0E1C0E1C0F3C0F3C0FFC0BF
:10398000FFC0FFC0FFC0EDC0EDC0EDC0EDC0EDC099
:10399000E1C0E1C0E1C0E1C0E1C000000000000002
:1039A0000000E1C0E1C0E1C0E1C0E1C0E1C0E1C0B0
:1039B000E1C0FFC0FFC0FFC0FFC0E1C0E1C0E1C087
:1039C000E1C0E1C0E1C0E1C0E1C0000000000000D2
:1039D00000001E003F007F807F80F3C0E1C0E1C097
:1039E000E1C0E1C0E1C0E1C0E1C0E1C0E1C0E1C0CF
:1039F000F3C07F807F803F001E00000000000000B9
:103A00000000FFC0FFC0FFC0FFC0E1C0E1C0E1C0D7
:103A1000E1C0E1C0E1C0E1C0E1C0E1C0E1C0E1C09E
:103A2000E1C0E1C0E1C0E1C0E1C000000000000071
:103A30000000FC00FF00FF80FFC0E3C0E1C0E1C068
:103A4000E3C0FFC0FF80FF00FC00E000E000E000FA
:103A5000E000E000E000E000E00000000000000006
:103A600000001E003F007F807FC0F1C0E0C0E0C0CA
:103A7000E000E000E000E000E000E000E0C0E0C0C6
:103A8000F1C07FC07F803F001E00000000000000EA
:103A90000000FFC0FFC0FFC0FFC01E001E001E00D0
:103AA0001E001E001E001E001E001E001E001E0026
:103AB0001E001E001E001E001E0000000000000070
:103AC0000000E1C0E1C0E1C0E1C0E1C0E1C073803D
:103AD00073803F003F001F001F000E000E000E000D
:103AE0000E000E00FC00FC00F800000000000000CA
:103AF00000001E001E003F007F80FFC0FFC0EDC021
:103B0000CCC0CCC0CCC0CCC0CCC0EDC0FFC0FFC0CE
:103B10007F803F001E001E001E000000000000000D
:103B20000000E1C0E1C0E1C0E1C073807380738038
:103B30003F001E001E001E003F007F8073807380C8
:103B4000E1C0E1C0E1C0E1C0E1C000000000000050
:103B50000000E380E380E380E380E380E380E380B0
:103B6000E380E380E380E380E380E380E380E3C0FD
:103B7000FFC0FFC0FFC001C001C000000000000086
:103B80000000E1C0E1C0E1C0E1C0E1C0E1C0E1C0CE
:103B9000E1C0F1C0FFC0FFC07FC03FC001C001C095
:103BA00001C001C001C001C001C000000000000050
:103BB0000000CCC0CCC0CCC0CCC0CCC0CCC0CCC031
:103BC000CCC0CCC0CCC0CCC0CCC0CCC0CCC0CCC095
:103BD000CCC0FFC0FFC0FFC0FFC00000000000005D
:103BE0000000CCC0CCC0CCC0CCC0CCC0CCC0CCC001
:103BF000CCC0CCC0CCC0CCC0CCC0CCC0CCC0FFC032
:103C0000FFC0FFC0FFC000C000C0000000000000F7
:103C10000000F000F000F000F00030003000300054
:103C200030003E003F803FC03FC031C030C030C098
:103C300031C03FC03FC03F803E0000000000000098
:103C40000000C0C0C0C0C0C0C0C0C0C0C0C0C0C0F4
:103C5000C0C0C0C0F8C0FCC0FEC0CEC0C6C0C6C098
:103C6000C6C0CEC0FEC0FCC0F8C00000000000000E
:103C70000000E000E000E000E000E000E000E00024
:103C8000E000FE00FF00FF80FF80E3C0E1C0E1C074
:103C9000E3C0FF80FF80FF00FE0000000000000086
:103CA00000003E007F007F80FF80F3C0E1C0C1C004
:103CB00001C00FC01FC01FC00FC001C0C1C0E1C004
:103CC000F3C0FF807F807F003E0000000000000006
:103CD0000000C700CF80DFC0DFC0DDC0D8C0D8C0C3
:103CE000F8C0F8C0F8C0F8C0F8C0F8C0D8C0D8C054
:103CF000DDC0DFC0DFC0CF80C700000000000000D3
:103D000000000FC03FC07FC0FFC0F1C0E1C0E1C0F4
:103D1000F1C07FC03FC01FC03FC039C039C079C0AB
:103D200079C0F1C0F1C0E1C0E1C0000000000000B6
:103D30000000000000000000000000003E007F00C6
:103D4000FF80C78003801F807F80FF80E780C38063
:103D5000C380E780FF807FC039C000000000000002
:103D6000000000001FC07FC0FFC0E000C000DF00F7
:103D7000FF80FFC0F3C0E1C0E1C0E1C0E1C0E1C02D
:103D8000E1C0F3C0FFC07F803F00000000000000E2
:103D9000000000000000000000000000FE00FF0026
:103DA000FF80E780E380E700FE00FF00FF80E3C0C4
:103DB000E1C0E3C0FFC0FF80FF0000000000000082
:103DC000000000000000000000000000FFC0FFC075
:103DD000FFC0F000F000F000F000F000F000F00094
:103DE000F000F000F000F000F00000000000000023
:103DF0000000000000000000000000003F803F8045
:103E00003F803B803B803B807380738073807380F6
:103E1000FFC0FFC0FFC0E1C0E1C000000000000023
:103E20000000000000000000000000003F007F8054
:103E30007F80F3C0E1C0FFC0FFC0FFC0E000E00032
:103E4000E1C0F3C07F807F803F00000000000000E1
:103E5000000000000000000000000000CCC0CCC04A
:103E6000EDC06D807F807F803F003F006D806D8062
:103E70006D80EDC0EDC0CCC0CCC0000000000000E3
:103E80000000000000000000000000007F00FF8034
:103E9000FFC063C001C007800700078003C001C0E6
:103EA00001C063C0FFC0FF807F0000000000000071
:103EB000000000000000000000000000E1C0E1C0C0
:103EC000E3C0E3C0E7C0E7C0EFC0EDC0FDC0F9C08C
:103ED000F9C0F1C0F1C0E1C0E1C000000000000085
:103EE000000033003F003F001E000000E1C0E1C0C1
:103EF000E3C0E3C0E7C0E7C0EFC0EDC0FDC0F9C05C
:103F0000F9C0F1C0F1C0E1C0E1C000000000000054
:103F1000000000000000000000000000E1C0E3C05D
:103F2000E780E700EE00FC00FC00FE00EE00E7008A
:103F3000E700E380E3C0E1C0E1C000000000000052
:103F40000000000000000000000000003FC03FC073
:103F50003FC039C039C039C039C039C039C039C093
:103F600039C039C0F1C0F1C0E1C00000000000005C
:103F7000000000000000000000000000E1C0E1C0FF
:103F8000E1C0E1C0F3C0F3C0F3C0FFC0FFC0EDC0AB
:103F9000EDC0EDC0E1C0E1C0E1C0000000000000E4
:103FA000000000000000000000000000E1C0E1C0CF
:103FB000E1C0E1C0E1C0FFC0FFC0FFC0E1C0E1C09F
:103FC000E1C0E1C0E1C0E1C0E1C0000000000000CC
:103FD0000000000000000000000000003F007F80A3
:103FE000FFC0F3C0E1C0E1C0E1C0E1C0E1C0E1C099
:103FF000E1C0F3C0FFC07F803F0000000000000070
:10400000000000000000000000000000FFC0FFC032
:10401000FFC0E1C0E1C0E1C0E1C0E1C0E1C0E1C07A
:10402000E1C0E1C0E1C0E1C0E1C00000000000006B
:10403000000000000000000000000000EF00FF8012
:10404000FBC0F1C0F1C0F1C0F1C0F1C0FBC0FF8006
:10405000EF00E000E000E000E000000000000000F1
:104060000000000000000000000000003F007F8012
:10407000FF80F3C0E1C0E000E000E000E000E0000D
:10408000E1C0F3C0FF807F803F000000000000001F
:10409000000000000000000000000000FFC0FFC0A2
:1040A000FFC01E001E001E001E001E001E001E007F
:1040B0001E001E001E001E001E000000000000006A
:1040C000000000000000000000000000E1C0E1C0AE
:1040D00071C071C071803B803B801B001F001F00BE
:1040E0000E001E007C007C00780000000000000034
:1040F000000000000C000C000C000C006D80FFC0E4
:10410000FFC0DEC0CCC0CCC0CCC0DEC0FFC0FFC092
:104110006D800C000C000C000C0000000000000082
:1041200000000000000000000000000071C071C02D
:1041300071C03B801F001F000E000E000E001F000C
:104140003F807BC071C071C071C0000000000000E2
:10415000000000000000000000000000E380E38099
:10416000E380E380E380E380E380E380E380E38037
:10417000FFC0FFC0FFC003C003C00000000000007C
:10418000000000000000000000000000E1C0E1C0ED
:10419000E1C0E1C0E1C0E1C0F1C0FFC07FC03FC0ED
:1041A00001C001C001C001C001C00000000000004A
:1041B000000000000000000000000000CCC0CCC0E7
:1041C000CCC0CCC0CCC0CCC0CCC0CCC0CCC0CCC08F
:1041D000CCC0CCC0FFC0FFC0FFC00000000000008A
:1041E000000000000000000000000000CCC0CCC0B7
:1041F000CCC0CCC0CCC0CCC0CCC0CCC0CCC0CCC05F
:10420000FFC0FFC0FFC000C000C0000000000000F1
:10421000000000000000000000000000F800F800AE
:10422000F8003800380038003F003F803FC039C0F8
:1042300038C039C03FC03FC03F80000000000000D0
:10424000000000000000000000000000C0C0C0C06E
:10425000C0C0C0C0C0C0FCC0FEC0FEC0CEC0C6C092
:10426000C6C0CEC0FEC0FCC0F8C000000000000008
:10427000000000000000000000000000E000E0007E
:10428000E000E000E000FF00FF80FFC0E3C0E1C00D
:10429000E1C0E3C0FFC0FF80FF000000000000009D
:1042A0000000000000000000000000007F00FF8010
:1042B000FFC063C001C001C00FC00FC00FC001C06C
:1042C00001C063C0FFC0FF807F000000000000004D
:1042D000000000000000000000000000C700CF80C8
:1042E000DFC0DDC0D8C0F8C0F8C0F8C0D8C0D8C0A2
:1042F000D8C0DDC0DF80CF80C70000000000000014
:104300000000000000000000000000001FC03FC0CF
:104310007FC079C071C071C079C03FC01FC03FC0AD
:1043200039C079C071C0F1C0E1C0000000000000D8
:10433000000000000000000000000000000000007D
:10434000000000000000000000000000000000006D
:1043500000000000000000000000000000001E0639
:104360000206171B0A1B0C240A2D0A2D0E1C130211
:104370000809080E0800002910000B131A09250966
:1043800030091F162B1630012F012810351500009B
:104390000000000028060306211B0E1B10240E2D12
:1043A0000E2D121C18020C090C0E0C000029150011
:1043B000101A1A0D250D300D1F1B2B1B30032F0259
:1043C0002815351A00000000000028060306211BEE
:1043D000141B1624142D142D181C1D021309130E62
:1043E00013030A291A00161D1A13251330131F2050
:1043F0002B2030032F02281A351F00000000000078
:1044000028060306211B0E1B10240E2D0E2D121C38
:1044100018020C090C0E0C0000291500101A1A0DB8
:10442000250D300D1F1B2B1B30032F022815351AAD
:10443000000000000000320603062B1B1E1B202478
:104440001E2D1E2D221C27021C091C0E1C030A29CE
:10445000240020271A1D251D301D1F2A2B2A30035A
:104460002F02282435290000000000003C06040625
:10447000351B221B2424222D212D251C2C021F0933
:104480001F0E1F030C292900242E1A20252030205E
:104490001F312B3130032F032829352E0000000057
:1044A000000028060306211B0F1B11240F2D0E2DC3
:1044B000121C18020C090C0E0C0000291500101A11
:1044C0000000000000000000000030032F02000088
:1044D00000000000000000003C060406351B231B02
:1044E0002524232D222D261C2C022009200E2003FA
:1044F0000C292900242E000000000000000000000C
:1045000030032F03000000000000000000001E0622
:10451000030617000F0011090F120D12111C0F00D6
:104520000B070B0C0B0000290C0000000000000022
:1045300000000000000030022F0200000000000018
:104540000000000028060306210019001B091912AB
:1045500017121B1C19001507150C15000029160051
:1045600000000000000000000000000030032F02E7
:1045700000000000000000000000280603062100E3
:1045800019001B09191217121B1C19001507150C0D
:1045900015030A29160000000000000000000000BA
:1045A000000030032F0200000000000000000000A7
:1045B000320603062B002300250923122112251C95
:1045C00023001F071F0C1F030B2920000000000001
:1045D000000000000000000030032F020000000077
:1045E0000000000000003C06040635002D002F09E5
:1045F0002D122B122F1C2D002907290C29030B2902
:104600002A0000000000000000000000000030034D
:104610002F03000000000000000000005E439443F0
:1046200036446C44A244D8440E454445B045E64562
:104630005E43CA4336446C44A244D8440E457A458E
:10464000B045E6455E43004436446C44A244D84439
:104650000E454445B045E6454C3A252E3475000DCF
:1046600019133D23312F3B370B27331B211D3905F0
:1046700011091772666C425C4E504448745F465F85
:10468000465F465F465F465F465F465F4669465FF8
:1046900046694669465F465F46694669465F4669C0
:1046A000465F465F466946694669465F465F4669BA
:1046B000465F465F46694669465F46694669465FAA
:1046C000465F4669465F466946694669465F465F9A
:1046D000465F4669465F4669465F4669465F46698A
:1046E000465F46694669465F465F46694669465F7A
:1046F0004669465F460000FFFC0000001FFFFFE028
:1047000000003FFFFFF80001FFFFFFFF0003FFFF76
:10471000FFFFC003FFFFFFFFC00FFFFFFFFFC00F42
:10472000FFFFFFFFC01F87FFFFFFC03F01FFF0FF3C
:10473000C07C00FF0007C07C307E0000C07C787C1D
:10474000000040F8FC38000000F8FE38001FFFF8B9
:10475000FC30001FFFF8FC30001FFFF8F87000036A
:10476000F8F0C0F00003F8F0C0F00003F8F0C3F078
:104770000003F8F0FFF00003F8F0FFF80003F8780A
:10478000FFF800000078FFFC00004078FFFE00000A
:10479000C078FFFF0007C03CFFFFF0FFC01CFFFF19
:1047A000FFFFC00FFFFFFFFFC00FFFFFFFFFC003B2
:1047B000FFFFFFFFC003FFFFFFFFC000FFFFFFFE83
:1047C00000003FFFFFF800001FFFFFE0000000FFB8
:1047D000FC0000000000FC000000001C03FF0000C3
:1047E000000033E7EFC0000000207FCFF0000000A2
:1047F000231D4B3C00000013885E7600000019C2A8
:10480000DE678000000D0014CCE0000002E084D9D7
:10481000D0000001E1A4B9D8000003C109B3B80079
:104820000007F113277300000E1232677300001E99
:104830000A444E6720001FCA44CC4720003FEC9931
:10484000988470003C243B998CE000383B333398CB
:10485000D8004D3B663318D800FB546C677B900141
:10486000F6551CEC731001CD551DC8F3340790C1EB
:1048700059C1E7360FC85353CF8C4C0FEC49D39F27
:1048800088881FE529D79F992831F427173E39409A
:104890003E3C27D73C7AC0719CAC763C7AC0F1DDB7
:1048A000F82638F680F3F3C01F79E480FEFB800F12
:1048B00071E400FFF8000771ED007FC0000773C9C5
:1048C000001F80000367DA000F8000034794000098
:1048D0000000030CB400000000016CA00000000008
:1048E00000F9E8000000000073B800000000003389
:1048F000B000000000003F6000000000001E6000EB
:10490000000000000E40000000000006C000000093
:10491000000003C000000000000180000000000053
:104920000080000000000000000000500040003047
:10493000002000180014001200110010000E000DDD
:10494000000C800B000B800A000A50055005500532
:10495000400530050005E004A004600420040004C4
:10496000E003A0034003200300020001D3CFC0CA2C
:10497000CEC2C0CDCEC3CEC4C5CD2020C2C5D120AD
:104980002020D620C520CD20C02020D120D320CC6F
:1049900020CC20C025362E336620EAE3004E3A258F
:1049A0002E327500CACECFC8DF00C8D2CEC30028D1
:1049B000252E347529005425362E3366EAE300256A
:1049C000327520F8F2000025347520F8F200002539
:1049D0002E32783A252E32783A252E327800252E3E
:1049E00032783A252E32783A252E3278414D0025FC
:1049F0002E32783A252E32783A252E3278504D00D4
:104A0000252E32782E252E32782E252E327800CA89
:104A1000CEC43A252E366C7500CFCBD33A252E3531
:104A20007500DDD2C8CAC5D2CECA3A25327500D2C9
:104A3000C0D0C02020202020202020CEC1D9C8C92D
:104A400020CED2D7C5D2000000000000000000C870
:104A5000D2CEC3CE20CFCE20C2D1C5CC20CFCBD397
:104A60003A0000000000000000000000000000000C
:104A70000000000000000000000000000000000036
:104A8000002020202020CED2D7C5D220CFCE20CFCC
:104A9000CBD32025356400000000000000CFD0CE2D
:104AA000D7C8C520C2C5D1CEC2DBC520D2CEC2C0B8
:104AB000D0DB3A0000000000000000000000000011
:104AC000000000000000000000000000000000CF17
:104AD000D0CED7C8C520D8D2D3D7CDDBC520D2CE33
:104AE000C2C0D0DB3A00000000000000000000005F
:104AF00000000000000000000000000000000000B6
:104B000000D1D3CCCCC03A0000000000000000006F
:104B10000000000000000000000000000000000095
:104B20000000000000000000000000000000000085
:104B3000000000C2C5D12FD8D23A0000000000000A
:104B40000000000000000000000000000000000065
:104B50000000000000000000000000000000000055
:104B60000000000000CFD0CEC4C0C63A0000000054
:104B70000000000000000000000000000000000035
:104B80000000000000000000000000000000000025
:104B90000000000000000000000000000000000015
:104BA00000000000000000A85FCA5F00000000D7FE
:104BB0004BB74B974BE74BA85FDB5F00000000A7AC
:104BC0004BC74B974BD752A85FEB5F00000000B775
:104BD0004BD74B974B0753A85FB75FD073D073C7C2
:104BE0004BA74B974B0000CA5F00600000000047D6
:104BF0004CF74BA74B574CCA5F106000000000E712
:104C00004B074CA74BF74DCA5F256000000000F72B
:104C10004B174CA74BA751CA5F3A60000000000732
:104C20004C274CA74B5752CA5F07650C520C5217C2
:104C30004C374CA74B0000CA5F4E603E563E56278D
:104C40004C474CA74B0000CA5F5F600761076137A4
:104C50004CE74BA74B00000060936000000000D7BA
:104C60004C674CE74BE74C0060A560D061D06157C2
:104C70004C774CE74B00000060BA603762376267E0
:104C80004C874CE74B00000060C960DD56DD56776D
:104C90004C974CE74B00000060DC60000000008790
:104CA0004CA74CE74B574D0060EC60CD56CD569766
:104CB0004CB74CE74B00000060FC60C256C256A7E0
:104CC0004CC74CE74B000000604B61CE4CCE4CB75C
:104CD0004CD74CE74B000000600F61604B604BC746
:104CE0004C574CE74B000093605B61F456F456F769
:104CF0004CF74C574C000093606F6102570257E726
:104D00004CE74C574C00005B6183612F5B2F5B17B6
:104D10004D174DE74C00005B6197614B5B4B5B07A8
:104D20004D074DE74C00006F611C65295B295B470F
:104D30004D374DF74C00006F613065225B225B27D9
:104D40004D474DF74C00006F614465045B045B37D1
:104D50004D274DF74C0000DC60AB61685B685B770A
:104D60004D674D974C0000DC60C1617F5B7F5B57F6
:104D70004D774D974C0000DC60D761DD5BDD5B67F4
:104D80004D574D974C0000FC602461D25DD755977C
:104D90004D974DB74C0000FC603761D25DD7558709
:104DA0004D874DB74C0000C960D065765DD755C7BB
:104DB0004DB74D874C0000C960C265765DD755A7D9
:104DC0004DC74D874C0000C960DE65765DD755B78D
:104DD0004DA74D874C0000EC60C265BE5DD755E71E
:104DE0004DE74DA74C0000EC60D065BE5DD755D7B0
:104DF0004DD74DA74C00001060E66100000000A7F1
:104E00004E074EF74BD74E1060F6614B564B56F798
:104E10004D174EF74B000010600862E45DE45D073B
:104E20004E274EF74B000010601C62000000001778
:104E30004E374EF74B174F106041620000000027BD
:104E40004E474EF74BB74F1060BC62000000003772
:104E50004E574EF74B374F1060D062A256A25647BE
:104E60004E674EF74B0000106022633A563A565791
:104E70004E774EF74B00001060E7629456945667E9
:104E80004E874EF74B00001060FE628956895677B8
:104E90004E974EF74B00001060C964AB4EAB4E8787
:104EA0004EA74EF74B000010601163000000009702
:104EB0004EF74DF74BB74E1163B464714E714EC748
:104EC0004EC74EA74E000011636C64054F054FB7E7
:104ED0004EB74EA74E0000E66153621D4D1D4DE7D3
:104EE0004EE74EF74D0000E66164627C4D7C4DD785
:104EF0004ED74EF74D0000F66175627762D75507C1
:104F00004F074F074E0000F66186627B62D755F768
:104F10004EF74E074E00001C629562AD56AD562707
:104F20004F274F274E00001C62A9625E5E5E5E172F
:104F30004F174F274E0000BC6258651C571C57A7DF
:104F40004F474F474E0000BC6267652A572A5737C4
:104F50004F574F474E0000BC6243633457345747A6
:104F60004F674F474E0000BC624B613E573E57575C
:104F70004F774F474E0000BC62556348574857670C
:104F80004F874F474E0000BC6264635257525777B9
:104F90004F974F474E0000BC6277635C575C578762
:104FA0004FA74F474E0000BC628C63665766579709
:104FB0004F374F474E000041621E64FE4DFE4DD7F5
:104FC0004FC74F374E000041623264254E254EB721
:104FD0004FD74F374E000041624664494E494EC795
:104FE0004FB74F374E000095624B61C45ED75507EF
:104FF00050F74F174F000095627665C45ED755E7AE
:105000004F0750174F000095628965C45ED755F76A
:105010004FE74F174F00005865C265DE5FD7552731
:10502000502750374F00005865D065DE5FD75517C1
:10503000501750374F00006765C265F65FD7554778
:10504000504750474F00006765D065F65FD755372A
:10505000503750474F00004363C2650660D755671D
:10506000506750574F00004363D0650660D75557CF
:10507000505750574F00004B61C2651660D7558797
:10508000508750674F00004B61D0651660D7557749
:10509000507750674F00005563C2652660D755A70B
:1050A00050A750774F00005563D0652660D75597BD
:1050B000509750774F00006463C2653660D755C77C
:1050C00050C750874F00006463D0653660D755B72E
:1050D00050B750874F00007763C2654660D755E7E9
:1050E00050E750974F00007763D0654660D755D79B
:1050F00050D750974F00008C63C2655660D7550754
:10510000510751A74F00008C63D0655660D755F703
:1051100050F750A74F0000E762C2657360D755276C
:10512000512751774E0000E762D0657760D7551759
:10513000511751774E0000FE62C2657A60D755471D
:10514000514751874E0000FE62D0657E60D75537CB
:10515000513751874E0000F3631566EA67D75567EC
:10516000516751D7510000F3632666EE67D7555754
:10517000515751D7510000D06231676660D75587CB
:10518000518751574E0000D06220676C60D7557729
:10519000517751574E000022633363E967D7559723
:1051A000519751674E00002560CA637D567D56E7D2
:1051B00051B751074C00002560DC636F566F56A74E
:1051C00051C751074C0000256037665E565E56B7E2
:1051D00051D751074C00002560F3632F562F56C757
:1051E00051E751074C000025600764E355E355D7AC
:1051F00051A751074C0000CA63C265045FD7550729
:10520000520752A7510000CA63D065045FD755F713
:1052100051F751A7510000DC630466225FD7552780
:10522000522752B7510000DC634B66225FD75517F7
:10523000521752B7510000376604668260D755474F
:10524000524752C751000037664B668560D75537C5
:10525000523752C75100003A60B563886088606772
:10526000526752174C00003A609E63D14DD14D57A2
:10527000525752174C00004E607260CE65CE658763
:10528000528752374C97524E608260CE65CE65771A
:10529000527752374CB75272605B64485F485FA7E1
:1052A00052A7527752000072608164BB5FBB5F9768
:1052B000529752775200008260926456665666C7D3
:1052C00052C752875200008260A3646A676A67B758
:1052D00052B75287520000DB5FE66602630263F753
:1052E00052E752B74B0000DB5FF9667F627F62D7FF
:1052F00052F752B74B0000DB5F0B67B163B163E756
:1053000052D752B74B0000EB5FDE64CC4FCC4F3727
:10531000531753C74B0000EB5FF264154F154F074F
:10532000532753C74B0000EB5F9D65CF51CF5117FB
:10533000533753C74B0000EB5FAF654861486127A7
:10534000530753C74B000007646B69F267D755B723
:10535000535753E751000007647C69F667D75547F8
:10536000536753E751000007649069FB67D75557AF
:10537000537753E75100000764A469FD67D7556769
:10538000538753E75100000764B869FF67D7557723
:10539000539753E75100000764CC690168D75587DC
:1053A00053A753E75100000764E0690368D7559796
:1053B00053B753E75100000764F4690568D755A750
:1053C000534753E75100003230303200257300203C
:1053D000202020C2E2E5E4E8F2E520EFE0F0EEEB89
:1053E000FC0A00000000256400252E3232730025DF
:1053F0002E313273002533750025302E366C750042
:1054000025302E326C750025302E32750025362E53
:10541000336600CFD23A25362E33660025372E323A
:10542000660025372E306600252E326625632563FB
:105430002563252E3266256300252E3066256325DB
:10544000632563252E306625630025342E75F8F21A
:105450002025372E3066000025342E75F8F22025E1
:10546000372E3266000025362E3366EAE3202537D4
:105470002E30660025362E3366EAE32025372E329D
:105480006600CFEEE4EEE6E4E8F2E50A00CDE0E601
:10549000ECE8F2E520EAEBE0E2E8F8F3203CC2E2D7
:1054A000EEE43E0020202020C2FBEAEBFEF7E8F20B
:1054B000E520E2E5F1FB0A0000000020202020208A
:1054C0002020D1EFE0F1E8E1EE210A0000CDE0E795
:1054D000EDE0F7E8F2FC20EAEBE0E2E8F8F320CFB9
:1054E000CBD3200020CEE1EDEEE2EBE5EDE8E520C8
:1054F000F6E5EDFB20CFCBD3202000CDE0E7EDE0BB
:10550000F7E8F2FC20EAEBE0E2E8F8F320F6E5ED5C
:10551000E500C2F1E5E3EE3A0A0000CFEEEAF3EF70
:10552000EEEA3A0A0000000000D1F3ECECE020EAD9
:10553000EBE8E5EDF2E03A0A00D1E4E0F7E03A0A00
:1055400000CAEEEBE8F7E5F1F2E2EE20EAEEEFE872
:10555000E93A202020253275000000CDE0EFE5F784
:10556000E0F2E0EDEE3A20202020202025357500E5
:10557000000000000025327520F8F22000CFCBD3C8
:105580003A253575202020CAEEE43A25366C7500A0
:1055900000000000C2FBEFEEEBEDE5EDE020EEF2E7
:1055A000ECE5EDE0210A0000000000CFCBD320EFB6
:1055B000E5F0E5E7E0EFE8F1E0EDEE210A000000BC
:1055C0000000CDE5F220F4E8EAF1E0F6E8E820E2B8
:1055D000E5F1E0210A00000000CFEEE8F1EA20F258
:1055E000EEE2E0F0E02E2E2E0A00000000000000A7
:1055F000CFC5D0C5D5CEC420C220CCC5CDDE20D1EC
:10560000C5D0C2C8D1C000C0D6CF20EDE5E8F1EFCB
:10561000F0E0E2E5ED210A0000000000CEF8E8E14C
:10562000EAE020E4E8E0EFE0E7EEEDE020EDF3EB88
:10563000FF2100CEF8E8E1EAE020E2FBE1EEF0EA4B
:10564000E820EDF3EBFF210A0000CEF8E8E1EAE004
:1056500020E2FBE1EEF0EAE820F2E0F0FB210A00B4
:1056600000CFE5F0E5E3F0F3E7EAE020E2E5F1EE74
:10567000E2210A00000000CFE5F0E5EFEEEBEDE5FA
:10568000EDE8E520F1F3ECECFB210A00002D2D2DD7
:105690002D2D2D00D0E5F1F2E0F0F220EFEE20F21A
:1056A000E0E9ECE5F0F3210A000000CDE5E8F1EFD8
:1056B000F0E0E2EDFB20F7E0F1FB210A0000000042
:1056C0000000C2E5F1FB20EDE520EEF2E3F0E0E4BE
:1056D000F3E8F0EEE2E0EDFB00CDE5F220E1F3ECE3
:1056E000E0E3E8210A0000CDE520EDE0E9E4E5EDA6
:1056F000E020FDF2E8EAE5F2EAE0210A0000CEF25D
:10570000EAF0FBF2E020EFE5F72E20E3EEEBEEE22D
:10571000EAE0212000D1EDE8ECE8F2E520FDF2E836
:10572000EAE5F2EAF3210A0000CFE5F0E5E3F0E56F
:10573000E220EFF0E8EDF2E5F0E0210A000000CE13
:10574000F8E8E1EAE020E4E0F2FB2DE2F0E5ECE548
:10575000EDE8210A0000D1EEEEE1F9E5EDE8FF20E9
:10576000EDE5E4EEF1F2F3EFEDFB212000CEF8E8F9
:10577000E1EAE020F1EEE7E4E0EDE8FF20D8CA211D
:105780000A000000CDE5E2E5F0EDEEE520EAEEEB03
:10579000E8F7E5F1F2E2EE210A0000CDE5E2E5F0FE
:1057A000EDFBE920E2E5F1210A0000000000000025
:1057B0000000CDE5E2E5F0EDE0FF20F2E0F0E021D1
:1057C0000A00000000000000CDE5E2E5F0EDE0FF9A
:1057D00020F6E5EDE0210A0000000000000000CD09
:1057E000E5E2E5F0EDE0FF20F1F3ECECE0210A006A
:1057F000000000000000CDF3EBE5E2E0FF20F1F255
:10580000EEE8ECEEF1F2FC210A0000CEF8E8E1EA65
:10581000E020EDE0F1F2F0EEE9EAE82025750A007B
:105820000000CEF8E8E1EAE02025750A0000CDE5A9
:10583000E7E0E2E5F0F8E5EDEDE0FF20EFE5F7E089
:10584000F2FC212000202020CDE5E2E5F0EDFBE98F
:1058500020EFE0F0EEEBFC2120202000CFEEE2F282
:10586000EEF020EDE5E2EEE7ECEEE6E5ED210A00F4
:10587000000000CDE5E2E5F0EDFBE920EAEEE420F2
:10588000CFCBD3210A0000000000CDE5E2E5F0ED2A
:10589000FBE920EAEEE420F2EEE2E0F0E0210A008B
:1058A00000D2EEE2E0F020EDE5E4EEF1F2F3EFE518
:1058B000ED210A0000000000CFF3F1F2EEE520CF69
:1058C000CBD32025750A00000000CEEFE5F0E0F60E
:1058D000E8FF20E7E0EFF0E5F9E5EDE0210A000060
:1058E00000546FE2E0F020EDE520E2FBE1F0E0EDB6
:1058F000210A000000000000C4EEE1E0E2EBE5ED6B
:10590000E8E520EDE5E2EEE7ECEEE6EDEE2100CE97
:10591000F2ECE5EDE020EDE5E2EEE7ECEEE6EDE0C1
:10592000210A00000000D1F3ECECE0F2EEF020EDF3
:10593000E520EFF3F1F2210A0000000000D1F3ECC2
:10594000ECE0F2EEF020EFF3F1F2210A00000000AB
:105950000000D3F1F2E0EDEEE2E8F2E520E2F0E55E
:10596000ECFF2FE4E0F2F32100CEF8E8E1EAE020DA
:10597000F1E8ECE2EEEBE020E2E0EBFEF2FB2100EE
:10598000D2E0F0E020EDE520F3F1F2E0EDEEE2EB25
:10599000E5EDE021202000CDE5F220F3F1EFEEEA85
:1059A000EEE5EDE8FF20E2E5F1EEE2212000CAF3AA
:1059B000F0F120EDE520E7E0E4E0ED210A00000051
:1059C0000000000000CDE5E2E5F0EDFBE520E4E0BD
:1059D000EDEDFBE520CFCBD3210A0000435338394E
:1059E000303020EDE520EDE0E9E4E5ED210A0000AE
:1059F000000000CEF8E8E1EAE020F1F2F0F3EAF28C
:105A0000F3F0FB20E1E0E7FB21002020D1E8F1F2F8
:105A1000E5ECEDE0FF20EEF8E8E1EAE021202020CF
:105A200000D2EEE2E0F020EDE520EDE0E9E4E5ED86
:105A3000210A000000000000CDE5F220E8EDE8F6C4
:105A4000E8E0EBE8E7E0F6E8E8205352414D00D407
:105A5000F3EDEAF6E8FF20EDE520E2FBEFEEEBEDFB
:105A6000E5EDE0212000CFE5F7E0F2FC20E1FBEBE3
:105A7000E020EFF0E5F0E2E0EDE0212000CFEEE203
:105A8000F2EEF0E8F2E520EEEFE5F0E0F6E8FE2ECB
:105A900020202000CDE0E9E4E5EDE020EDE5E7E0C1
:105AA000E2E5F0F8E5EDEDE0FF2000EEEFE5F0E0F7
:105AB000F6E8FF20F3F7E5F2E02120202020202067
:105AC0002000CDE520E7E0E4E0ED20E72FED20E247
:105AD000E5F1EEE2210A00C2CC31303020EDE520C4
:105AE000EDE0E9E4E5ED210A0025750A00253375AE
:105AF0002E2533752E2533752E2533750A002D2D51
:105B00002E2D2D2E2D2D00252B2E316400252E31EE
:105B10007500252E327500252E337500252E34751F
:105B20000025302E347500252E35750025302E3594
:105B3000750025357500253131750025356C7500EA
:105B40002531316C7500252E316C7500252E326C97
:105B50007500252E336C7500252E346C7500252EAE
:105B6000356C7500252E366C7500252E376C75004A
:105B7000252E386C750025362E32660025392E32DA
:105B8000660025392E306600523A257520483A25A0
:105B90007520503A25752050453A25752F25332E0E
:105BA0003166560A004C3A25752F25332E3166563C
:105BB00020543A25752F257525630A00C2E5F0F1BA
:105BC000E8FF2025752E25750A0025642025730021
:105BD000252E32783A252E32783A252E32780A0050
:105BE000252E32782E252E32782E252E32780A0058
:105BF000252E32752E252E32752E252E3275002536
:105C00002E327800504D0A00414D0A0025630A00EB
:105C1000CAEBE0E22DF0E020E7E0E1EBEEEAE8F0AD
:105C2000EEE2E0EDE020002020D1F0EEF7EDEEE531
:105C30002020F1EEEEE1F9E5EDE8E520200020205E
:105C4000202020C3F0E0E4F3E8F0EEE2EAE02020D8
:105C50002020202000CFEEE4EEE6E4E8F2E5203557
:105C600020ECE8EDF3F22E2E2E202000CEF1F2E013
:105C7000EBEEF1FC3A257520ECE8ED20257520F1DE
:105C8000E5EA0A00CDE0E3F0F3E7E8F2E50A000018
:105C90000000000000000000000020EAE30A00000D
:105CA00000000000000000000000000000000000F4
:105CB000C6E4E8F2E520F3F1EFEEEAEEE5EDE8FF09
:105CC0000A0000000000CDEEE2FBE920EFE0F0EE7C
:105CD000EBFC3A0A000000000000000000CFEEE4F8
:105CE000F2E2E5F0E6E4E5EDE8E53A0A000000005E
:105CF00000000000CDEEE2FBE920EFE0F0EEEBFC6F
:105D000020F3F1EFE5F8EDEE0A0000F3F1F2E0ED3B
:105D1000EEE2EBE5ED2E0A000000000000000000BE
:105D20000000CDEEE2FBE920EFE0F0EEEBFC20ED31
:105D3000E520F1EEE2EFE02D00E4E0E5F220F120D5
:105D4000EFEEE4F2E2E5F0E6E4E5EDE8E5EC210073
:105D5000CFF3EDEAF220ECE5EDFE20EDE5E4EEF127
:105D6000F2F3EFE5ED2100CFF0E8EDFFF2EE3A209F
:105D7000202020CFEEF1EBE0EDEE3A20200028E2EB
:105D800020E4EDFFF5290A000000CAF3F0F13A0A19
:105D900000000000C0E2F2EEEFE5F7E0F2FC3A0AA4
:105DA0000000C2E2E5E4E8F2E520F2E0F0F33A0AAE
:105DB0000000202020202020202020CDE5F20A0015
:105DC00000202020CEF2E4E5EBFFE5F2203220E7D0
:105DD000EDE0EAE00A000000CFEEE4F2E2E5F0E4F4
:105DE000E8F2FC2FCEF2ECE5EDE8F2FC203F00D12A
:105DF000F2E0F2F3F13A2531752C20EAEEEBEBE814
:105E0000E7E8E83A25337500C7E0E2EEE4F1EAEEB0
:105E1000E920EDEEECE5F020E7E0E4E0ED2E00C84F
:105E2000E4E5F220E7E0EFE8F1FC20E220CEC7D382
:105E30000A00C8E4E5F220F7F2E5EDE8E520E8E73E
:105E400020CEC7D30A00C0E4F0E5F13A256C7820F3
:105E5000C7EDE0F73A25780A00C0E4F0E5F13A250D
:105E6000780A005B205D20F2EEEBFCEAEE20F7F210
:105E7000E5EDE8E50A005B205D20EFF0EEF1ECEEE9
:105E8000F2F020E7EDE0F7E5EDE8E92000D2EEE200
:105E9000E0F0EDE0FF20E1E0E7E020E820E8F2EECE
:105EA000E3E82000EFF0EEE4E0E620E1F3E4F3F2D3
:105EB00020EEE1EDF3EBE5EDFB2100D0E5E6E8ECCB
:105EC00020E1FBF1F2F0EEE920E7E0E3F0F3E7EAAE
:105ED000E800D0E5EFE5F0EDE0FF20F2EEF7EAE0D4
:105EE00020256420EAE30A00CFF0EEE8E7E2EEE4E2
:105EF000E8F2F1FF20EEE1F0E0E1EEF2EAE000C3CB
:105F0000F0E0E4F3E8F0EEE2EAE020F3F1EFE5F8A8
:105F1000EDEE0A00E2FBEFEEEBEDE5EDE0210A002D
:105F2000C3F0E0E4F3E8F0EEE2EAE020E1FBEBE0CE
:105F300020EFF0E5F02D00E2E0EDE020EFEEEBFCED
:105F4000E7EEE2E0F2E5EBE5EC210A00C3F0E0E485
:105F5000F3E8F0EEE2EAE020EDE520E2FBEFEEEB25
:105F60002D2000EDE5EDE02028EEF8E8E1EAE02064
:105F7000256429210A00EDE5EDE0210A00D3F1F2C4
:105F8000E0EDEEE2EAE020EDE0F1F2F0EEE5EA0A23
:105F900000E2E5F1EEE220EFEE20F3ECEEEBF7E0CD
:105FA000EDE8FE2E2E2E2000202020202020202074
:105FB00020CCC5CDDE0A002020202020D2E5F1F241
:105FC000E8F0EEE2E0EDE8E50A00202020202020C5
:105FD000CDE0F1F2F0EEE9EAE80A002020202020EE
:105FE000202020CEF2F7E5F2FB0A00202020D0E5A9
:105FF000E4E0EAF2EEF020F2EEE2E0F0EEE20A0097
:1060000020202020202020D1E8F1F2E5ECE00A0059
:10601000202020CFE0F0E0ECE5F2F0FB20EFE5F708
:10602000E0F2E80A002020D0E0E1EEF2E020F120EA
:10603000F2EEE2E0F0E0ECE80A0020202020D1F2CD
:10604000F0F3EAF2F3F0E020E1E0E7FB0A002020C1
:1060500020202020C8EDF2E5F0F4E5E9F10A002067
:1060600020202020C2EEF1F1F2E0EDEEE2E8F2FCB9
:106070000A0020202020202020205253323332D109
:106080000A002020202020202045746865726E655B
:10609000740A00202020202020C4E0F2E02FC2F06B
:1060A000E5ECFF0A0020202020CFEEEBEEE6E5ED48
:1060B000E8E520F2EEF7EAE80A0020202020202080
:1060C000202020C7E2F3EA0A002020202020D0E58B
:1060D000E6E8EC20EFE5F7E0F2E80A0020202020D7
:1060E00020202020C2E0EBFEF2E00A002020202049
:1060F000202020D4E0F1EEE2EAE00A002020202077
:1061000020C4EEF1F2F3EF20EA20CFCBD30A002037
:106110002020C8E7ECE5EDE5EDE8E520EFE0F0EE66
:10612000EBFF0A0020202020CFEE20EDEEECE5F082
:10613000F320CFCBD30A0020202020CFEE20EAEEA0
:10614000E4F320F2EEE2E0F0E00A0020202020203C
:106150002020B920E2E5F1EEE20A00202020D3F170
:10616000F2E0EDEEE2EAE020F7E0F1EEE20A0020F4
:10617000202020D3F1F2E0EDEEE2EAE020E4E0F2CC
:10618000FB0A00202020D0E5E6E8EC20F7E0F1EE65
:10619000E2203234F70A00202020D0E5E6E8EC20A7
:1061A000F7E0F1EEE2203132F70A002020D1E8ECEE
:1061B000E2EEEB20EEF1ED2E20E2E0EBFEF2FB0A48
:1061C000002020D1E8ECE2EEEB20E4EEEF2E20E21E
:1061D000E0EBFEF2FB0A00202020202020202020DF
:1061E000CAF3F0F10A0020202020202020CFF0E880
:1061F000EDF2E5F00A00202020202020D2E8EF2058
:10620000EFE5F7E0F2E80A00202020D4EEF0ECE021
:10621000F220FDF2E8EAE5F2EAE80A002020202078
:106220002020D8F2F0E8F52DEAEEE40A0020202044
:1062300020C2E5F120E0E2F2EEEFE5F7E0F2E80A55
:10624000002020202020CFF0E5F4E8EAF1FB20D860
:10625000CA0A0020202020202020CAEEEDF2F0E023
:10626000F1F20A0020202020202020D1ECE5F9E5E1
:10627000EDE8E50A0020202020202020DDF2E8EAD9
:10628000E5F2EAE00A002020202020202020CBE5B3
:10629000EDF2E00A00202020D2E8EF20EFF0E5F454
:1062A000E8EAF1E020D8CA0A002020202020D1F21C
:1062B000F0F3EAF2F3F0E020D8CA0A00202020CF61
:1062C000E5F7E0F2E0E5ECFBE520EFEEEBFF0A009E
:1062D000202020C4E0F2F7E8EA20FDF2E8EAE5F247
:1062E000EAE8202020200020D1E1F0EEF120CFCB01
:1062F000D320EFEEF1EBE520EFE5F72E2000202094
:10630000202020CFE5F7E0F2FC20EFEE20CF2B0A93
:1063100000202020202020C7E0E3EEEBEEE2EAE8B8
:106320000A00202020202020CFEEE4ECEEF2F7E857
:10633000EA0A0020202020202020CEE1FBF7EDFB00
:10634000E90A00202020202020B920FDF2E8EAE51B
:10635000F2EAE80A00202020202020202020D2E09D
:10636000F0E00A0020202020D1F0EEEA20E3EEE465
:10637000EDEEF1F2E80A00202020D6E5EDE020E87D
:1063800020F1F2EEE8ECEEF1F2FC0A0020202020F1
:1063900020C7EDE0EAE820E2E0EBFEF20A0020D1BF
:1063A000F2F0EEEA20E220EDE0E7E22E20F2EEE26B
:1063B000E0F0E02000202020D2EEE2E0F0FB2FF120
:1063C000EEEEE1F9E5EDE8FF0A002020202020D3E1
:1063D000F7E5F220EFEE20CFCBD30A002020C8E76C
:1063E000ECE5EDE5EDE8E520F6E5EDFB20CFCBD3E0
:1063F00020200020202020D1E2EEE1EEE4EDE0FFBD
:1064000020F6E5EDE00A0020D1E1F0EEF120CFCB5F
:10641000D320EFEE20F2E0E9ECE5F0F320002020BD
:1064200020C2E5F1EEE2EEE920EFF0E5F4E8EAF172
:106430000A00202020D8F2F3F7EDFBE920EFF0E589
:10644000F4E8EAF10A00202020C8F2EEE3EEE2FBD5
:10645000E920EFF0E5F4E8EAF10A0020202020200E
:106460002020D1EAEEF0EEF1F2FC0A002020C8F282
:10647000EEE3EEE2E0FF20FDF2E8EAE5F2EAE00A10
:106480000020202020202020CFF0EEF2EEEAEEEBDC
:106490000A0020202020202020495020E0E4F0E5C0
:1064A000F10A002020202020202055445020EFEE2B
:1064B000F0F20A00202020CEE1FBF7EDE0FF20FD06
:1064C000F2E8EAE5F2EAE00A002020CDE0E7E2E0C7
:1064D000EDE8E520ECE0E3E0E7E8EDE00A0020206D
:1064E00020D2E0E1EBE8F6E020F2EEE2E0F0EEE2CE
:1064F0000A002020D2E0E1EBE8F6E020F1EEEEE148
:10650000F9E5EDE8E90A00202020D0E5EAEBE0EC2F
:10651000EDE0FF20F1F2F0EEEAE00A00202020D4C6
:10652000EEF0ECE0F220E4E42EECEC2EE3E30A00E3
:10653000202020D4EEF0ECE0F220ECEC2EE4E42E6F
:10654000E3E30A00202020D4EEF0ECE0F220E3E3C5
:106550002EECEC2EE4E40A00202020202020202035
:1065600020C4E0F2E00A002020202020202020C2C9
:10657000F0E5ECFF0A0020202020C3F0F3EFEFEE5F
:10658000E2EEE920EAEEE40A0020202020C2E5F154
:106590002FF8F220EFF0E5F4E8EAF10A00202020DD
:1065A0002020CEF7E8F1F2EAE020CFCBD30A00209A
:1065B00020202020CEF7E8F1F2EAE020E1E0E7FB3E
:1065C0000A0020202020202020202020C4E00A00D3
:1065D000202020202020202020CDE5F20A002020AD
:1065E00020202020202020C0E2F2EE0A002020CF30
:1065F000F0EEF1ECEEF2F020F1E8ECE2EEEBE03A56
:1066000025630A00202020202020C7E0EFF0E5F9D4
:10661000E5EDEE0A00202020202020D0E0E7F0E584
:10662000F8E5EDE00A00202020202020C7E0EFF070
:10663000E5F9E5EDE00A00202020C7E0EFE8F1FCF5
:1066400020F6E5EDFB20CFCBD30A00202020202030
:1066500020D0E0E7F0E5F8E5EDEE0A00202020206C
:106660002020203234303020E1EEE40A00202020C7
:10667000202020203438303020E1EEE40A002020B1
:1066800020202020203936303020E1EEE40A00209E
:106690002020202020313932303020E1EEE40A0081
:1066A000202020202020333834303020E1EEE40A4E
:1066B00000202020202020353736303020E1EEE445
:1066C0000A0020202020202031313532303020E1D6
:1066D000EEE40A002020202020D8F2F0E8F52DCFAB
:1066E000F0E8EDF20A002020202020CEF2F7E5F2BB
:1066F00020EFEE20CFCBD30A002020202020CEE1B7
:10670000F9E8E920EEF2F7E5F20A00202020CEE1D8
:10671000EDF3EBE5EDE8E520E8F2EEE3EEE20A006A
:1067200020202020202020C2FBEAEBFEF7E5ED0A26
:106730000020202020202020C2EAEBFEF7E5ED0A11
:10674000002020202020202035387833302CD8CA53
:106750000A002020202020202035387834302CD802
:10676000CA0A002020202020202035387835302CFF
:10677000D8CA0A0020202020202020353878363042
:106780002CD8CA0A002035387834302CD8CA2CF1DD
:1067900020F0E0E7ECE5F2EAEEE920002035387879
:1067A00036302CD8CA2CF120F0E0E7ECE5F2EAEE26
:1067B000E920002020353878333020F120F0E0E760
:1067C000ECE5F2EAEEE90A00202035387834302092
:1067D000F120F0E0E7ECE5F2EAEEE90A00202035EE
:1067E0003878353020F120F0E0E7ECE5F2EAEEE928
:1067F0000A002020353878363020F120F0E0E7EC30
:10680000E5F2EAEEE90A0020202020202020D4EE44
:10681000F0ECE0F220310A0020202020202020D4BB
:10682000EEF0ECE0F220320A002020202020202090
:10683000D4EEF0ECE0F220330A00202030202D20AE
:10684000D8CA20EEF2EAEBFEF7E5ED0A002020318F
:10685000202D20CFCFD2D2D2D2D2EAD1D1D1D1CA1B
:106860000A00202032202D20CFCFD2D2D2D2EAD19E
:10687000D1D1D1D1CA0A00202033202D20CFCFD2B0
:10688000D2D2D2D2D2D1D1D1D1CA0A002020342042
:106890002D20CFCFD2D2D2D2D2D1D1D1D1D1CA0A0A
:1068A00000202035202D20CFCFD2D2D2D2D1D1D1AD
:1068B000D1D1D1CA0A00202036202D20CFCFD2D26C
:1068C000D2D2D2D2C2C2C2C2CA0A00202037202DE0
:1068D00020CFCFD2D2D2D2D2C2C2C2C2C2CA0A0042
:1068E000D1EEEEE1F9E5EDE8E53A0A00D1F2F03A51
:1068F0000A00CFCBD33A0A003C202020202020D809
:10690000F2F3F7EDFBE9202020202020203E003C80
:10691000202020202020C2E5F1EEE2EEE920202018
:10692000202020203E00202020202020202035353F
:1069300030302F3020202020202020200020203424
:106940003430302F35303020283420F1F2F0EEEAA8
:10695000E82920002020333330302F3530302028F4
:106960003820F1F2F0EEEA2920200020202020201B
:106970002020CEF2EAEBFEF7E5ED0A0020202020F1
:10698000F7E5F0E5E7203520F1E5EAF3EDE40A006C
:10699000202020F7E5F0E5E720313520F1E5EAF3A6
:1069A000EDE40A00202020F7E5F0E5E72033302071
:1069B000F1E5EAF3EDE40A00202020F7E5F0E5E751
:1069C00020343520F1E5EAF3EDE40A002020202010
:1069D000F7E5F0E5E7203120ECE8EDF3F2F30A000B
:1069E00020202020F7E5F0E5E7203220ECE8EDF369
:1069F000F2FB0A0020202020F7E5F0E5E720332015
:106A0000ECE8EDF3F2FB0A0020202020D1C5D0C233
:106A1000C8D1CDCEC520CCC5CDDE20202020002081
:106A200020202020C3F0E0E4F3E8F0EEE2EAE020EA
:106A30002020202020002020202020C2EEF1F1F292
:106A4000E0EDEEE2E8F2FC202020202000202020D3
:106A50002020D2E5F1F2E8F0EEE2E0EDE8E52020DA
:106A60002020200020202020D1F7E5F2F7E8EAE8F6
:106A700020F1E1EEE5E22020202000202020C7E0E8
:106A8000E4E0F2FC20E72FED20E2E5F1EEE2202049
:106A90002000202020C4E0F2F7E8EAE820EFF0E848
:106AA000EDF2E5F0E020202000202020D2E5F1F2F8
:106AB000EEE2E0FF20EFE5F7E0F2FC2020202000EE
:106AC00020202020C2E5F1EEE2EEE920ECEEE4F336
:106AD000EBFC2020202000202020C8EDF2E5F0F47F
:106AE000E5E9F120525332333220202020002020CB
:106AF000C8EDF2E5F0F4E5E9F12045746865726EE1
:106B000065742020002020202020D2E5F1F220EF23
:106B1000E0ECFFF2E820202020202000202020D2DE
:106B2000E5F1F220EAEBE0E2E8E0F2F3F0FB20200E
:106B3000202000202020D2E5F1F220506F776572EE
:106B4000204661756C74202020002020C2FBE1E506
:106B5000F0E8F2E520F2E8EF20EFE5F7E0F2E820D8
:106B60000028202920EBE5EDF2E02028202920FD57
:106B7000F2E8EAE5F2EAE0002020C2FBE1E5F0E815
:106B8000F2E520F2E8EF20F2E5F1F2E0202000202B
:106B900020205B205D20E1E5F1EAEEEDE5F7EDFB7D
:106BA000E92020202000C4E0F2F7E8EA20F1EDFF20
:106BB000F2EEE920FDF2E8EAE5F2EAE80020202022
:106BC00020205B205D20E2EAEBFEF7E5ED202020AF
:106BD0002020200020202020202020204545505229
:106BE0004F4D202020202020202000202020202069
:106BF00020205254432052414D202020202020208C
:106C000020002020202020202020205352414D20F1
:106C10002020202020202020002020202020D2E51D
:106C2000F1F220454550524F4D0A0000000000008F
:106C30002020202020D2E5F1F2205254432052415E
:106C40004D0A0000000000202020202020D2E5F185
:106C5000F2205352414D0A000000000000002020A5
:106C60002020C8EDE8F6E8E0EBE8E7E0F6E8FF20F2
:106C7000202020200020CFF0EEF1ECEEF2F020F00A
:106C8000E5E7F3EBFCF2E0F2EEE22000C2F0E5EC27
:106C9000FF2050464F3A25756D730A000000000032
:106CA0000000002020CFF0EEF1ECEEF2F020F1F742
:106CB000E5F2F7E8EAEEE22020002020CEE1EDF355
:106CC000EBE5EDE8E520F1F7E5F2F7E8EAEEE220A2
:106CD00000D1E1EEE5E220E4E8F1EFEBE5FF3A2553
:106CE000750A000000000000D0E5F1F2E0F0F2EEDD
:106CF000E220EFEE205744543A25750A000000D1F7
:106D0000E1EEE5E2205352414D3A25750A000000BC
:106D1000000000000000D1E1EEE5E22043533839E5
:106D200030303A25750A00000000000000D1E1EE85
:106D3000E5E2205254433A25750A000000000000A5
:106D400000000000D1E1EEE5E220574D3130303A4D
:106D500025750A0000000000000000C2E2E5E4E83A
:106D6000F2E520E7E0E2EEE4F1EAEEE90A000000F5
:106D70000000EDEEECE5F020E2E5F1EEE23A0A008B
:106D8000000000000000000000CDEEE2FBE920E77B
:106D90002FED20E2E5F1EEE23A25750A0000000051
:106DA000CEF8E8E1EEEA20EDE5F20A00000000008E
:106DB000CEF8E8E1EAE020EEF7E8F1F2EAE820E1D7
:106DC000E0E7FB21202000C0E2F2EEEFE5F7E0F281
:106DD000FC20E2FBEAEBFEF7E5EDE0212000CEF837
:106DE000E8E1EAE020EEF7E8F1F2EAE820CFCBD3E1
:106DF0002120202000C0E2F2EEE2EEF1F1F2E0ED1F
:106E0000EEE2EBE5EDE8E52E2E2E2000CEF8E8E1EF
:106E1000EAE020EEE1EDF3EBE5EDE8FF210A00000A
:106E2000000000CDE520E7E0E4E0ED20E72FED20D5
:106E3000E2E5F1EEE2210A000000CEF8E8E1EAE046
:106E40002028E0E4F0E5F13A257829210A00CEF87F
:106E5000E8E1EAE02028E0E4F0E5F13A256C782961
:106E6000210A00C3F0E0E4F3E8F0EEE2EAE020ED0E
:106E7000E5E2EEE7ECEEE6EDE000CEF8E8E1EAE090
:106E800020C2CC313030204E202564210A00CEF8BB
:106E9000E8E1EAE02050464F210A0020CAEEE42053
:106EA000F2EEE2E0F0E00020CDE0E7E2E0EDE8E540
:106EB00020310020CDE0E7E2E0EDE8E5203200D629
:106EC000E5EDE020F2EEE2E0F0E00020D1F0EEEAC5
:106ED00020E3EEE4ED2E00202020C2E5F120F2E0D8
:106EE000F0FB0020CAEEE420E3F0F3EFEFFB00B983
:106EF00020F1EEEEE1F9E5EDE8FF002020B920E316
:106F0000F0E0F4E8EAE8002020B920D0CED1D2C5E4
:106F1000D1D20020D2E8EF20F2EEE2E0F0E0002053
:106F2000D0E5E0EBE8E7E0F6E8FF0040650000E0D0
:106F3000EB0100807203007C153011E40C0000F4BA
:106F400001F40100040800FF01FE02FD03FC04FB44
:106F500005FA06F907F83031323334353637383927
:106F600041424344454600303132333435363738B8
:106F70003961626364656600286E756C6C20706FA1
:0B6F8000696E74657229003F3F3F00FE
:106F8C0000017D43874301A64301BB4301DE43015E
:106F9C00EF4301FA43010244010B44206E440213F7
:106FAC00441E5444026444032B4425844408314455
:106FBC00023D440237440843447A9C43FB000101E0
:106FCC0087469D4601AC46019D4601A546019D465E
:106FDC0001A546019D46019D4601A546079D46011A
:106FEC00A546019D46FB000044510C0049505A50E7
:106FFC0062506A5081509350B150BB50D150ED50FB
:10700C00F6502F5100002D5E0D00055E085E0B5EE4
:10701C000E5E115E145E175E1A5E1D5E205E235EB0
:10702C00265E295E0000975E08007E5E815E845EAF
:10703C00875E8A5E8D5E905E935E0100ED62140049
:10704C0096629B629E62A162A462A462ED62ED6292
:10705C00ED62CF62D262D562ED62D862DB62DE6233
:10706C00E162E462E762EA6201009D631400476337
:10707C004C634F635263556355639D639D639D637E
:10708C007F63826385639D6388638B638E63916387
:10709C00946397639A6301004E69080098699E692E
:1070AC00A269A669AA69AE69B269B66901000273E0
:1070BC001B00B072B472B772BA72BD72C072C37276
:1070CC00C672C972CC72CF72D272D572D872DB72A0
:1070DC00DE72E172E472E772EA72ED72F072F372D0
:1070EC00F672F972FC72FF72000004740800EB7304
:1070FC00EF73F273F573F873FB73FE730174000096
:10710C00D1730800D3731474167418741A741C7425
:10711C001E7420740000B3AF080087AF8CAF91AF22
:10712C0096AF9BAFA0AFA5AFAAAF0100D5C214001C
:10713C00A8C2ABC2AEC2B1C2B4C2B4C2D5C2D5C26F
:10714C00D5C2B7C2BAC2BDC2D5C2C0C2C3C2C6C202
:10715C00C9C2CCC2CFC2D2C25A0106C6CCC2010629
:10716C00C401E8C50123C402FAC5013DBE01FDC539
:10717C000100C601D2C26503C60115C2013DBEFBAA
:10718C0001006AC714004AC74EC750C752C754C73C
:10719C0054C76AC76AC76AC756C758C75AC76AC7A7
:1071AC005CC75EC760C762C764C766C768C70100B3
:1071BC006DCA14004FCA51CA53CA55CA57CA57CAC6
:1071CC006DCA6DCA6DCA59CA5BCA5DCA6DCA5FCA3F
:1071DC0061CA63CA65CA67CA69CA6BCA0100DDCBDA
:1071EC001400BDCBC1CBC3CBC5CBC7CBC7CBDDCB81
:1071FC00DDCBDDCBC9CBCBCBCDCBDDCBCFCBD1CB93
:10720C00D3CBD5CBD7CBD9CBDBCB84E503E88AE585
:10721C0090E596E59CE503E803E803E803E803E85A
:10722C00A2E5A8E5AEE5B4E5BAE5C0E5C6E5CCE572
:10723C00D2E503E803E803E803E803E803E8D8E54C
:10724C00DEE5E4E5EAE5F0E5F6E503E8FCE502E673
:10725C0008E60EE614E61AE603E803E820E626E65E
:10726C002CE632E638E63EE644E64AE650E656E6DA
:10727C005CE662E603E803E803E803E803E868E693
:10728C006EE674E67AE680E686E68CE692E698E6AA
:10729C009EE6A4E603E803E803E8AAE6B0E66CE59C
:1072AC0072E578E57EE5B6E660E5BCE65AE566E5AE
:1072BC0003E803E803E803E803E803E803E8C2E6AD
:1072CC00C8E603E803E803E803E803E803E803E897
:1072DC0003E803E803E803E803E803E803E8CEE681
:1072EC00D4E6DAE6E0E6E6E6ECE6F2E6F8E6FEE61A
:1072FC0004E70AE710E716E71CE722E728E72EE782
:10730C0034E73AE740E746E74CE752E758E75EE7F1
:10731C0063E703E803E803E803E803E803E868E746
:10732C006DE772E777E77CE781E786E78BE790E725
:10733C0003E803E803E803E803E803E803E895E758
:10734C009AE703E803E803E803E803E803E803E843
:10735C0003E803E803E803E803E803E803E89FE72E
:10736C00A4E7A9E7AEE703E803E803E803E803E8CA
:10737C0003E803E803E803E803E803E803E8B3E7FA
:10738C00B8E7BDE7C2E7C7E7CCE703E803E803E8E3
:10739C0003E803E803E803E803E803E803E8D1E7BC
:1073AC00D6E7DBE7E0E7E5E703E803E803E803E813
:1073BC0003E803E803E803E803E803E803E8EAE783
:1073CC00EFE7F4E7F9E703E803E803E803E803E889
:1073DC0003E803E803E803E803E803E803E803E849
:1073EC0003E803E803E803E803E803E803E803E839
:1073FC0003E803E803E8FEE7070170EE7CEE0B768A
:10740C00EE1E7AEE017AEE0182EE087AEE387AEE12
:10741C00017AEE017AEE017AEE7384EE1476EEFBCD
:10742C000001A5F9A0F9456DF90262F911C6F80B36
:10743C0088F801E6F8016DF9016CF90162F902E6D0
:10744C00F8056DF801BCF801C6F80394F802C6F80B
:10745C0003C3F8FB40D051F19E0100810E94F13C26
:10746C00002311F400E535C03DD010F404E531C023
:10747C0054D049D057D0E5E8FFE040815181652FC9
:10748C00660F660B041715072607360710F405E57B
:10749C0020C0288539852F3F3F4F11F407E519C0CF
:1074AC0037D001F31FD0A0F401E513C000918D0F6C
:1074BC0000238E0129F00E94A03E002329F4D2CF94
:1074CC000E947F3E002371F20DD010F402E501C042
:1074DC0000E02A9608952A97E3E8FFE000811181E5
:1074EC00012B08951AD0488159816A817B811AD069
:1074FC00E9E8FFE04081518162817381041715072F
:10750C002607370708954C815D816E817F81089530
:10751C008E010E94BE3E002308950FEF1FEF2FEF48
:10752C003FEF0895041B150B260B370B089548816C
:10753C0059816A817B81401B510B620B730B488311
:10754C0059836A837B830895C6DFE9E8FFE060D046
:10755C0022813381088319832A833B8341F1E5E837
:10756C00FFE056D0212F220F220B0C831D832E837C
:10757C002F8301E010E0088719879E0147D00E94F5
:10758C006C3D002311F400E536C047D00E94D13E7B
:10759C000023C9F340D046D00C811D812E813F8140
:1075AC0004831583268337830885198516C00091BB
:1075BC008D0F002332D029F00E94B33E002329F412
:1075CC00E2CF0E94923E0023F1F225D02BD000E0B6
:1075DC0010E004830583068307830087118716D088
:1075EC0026D00083118300918D0F0093AD0F01E025
:1075FC000093AE0F00E02A960895E1EAFFE00081C7
:10760C0011812281338193DF8E010895E3E8FFE03D
:10761C00008111810895E1EAFFE0088119812A8136
:10762C003B81089500831183228333830895EBEA11
:10763C00FFE00895BA93AA932A970091AE0F002306
:10764C0011F408E569C0F3DFE3DF012BB9F19E010A
:10765C00DFDF0E94F13C002329F400E00093AE0F21
:10766C0009E55AC0A1EABFE05BD013975ED014962F
:10767C0057D0179748DF401B510B620B730B4C8391
:10768C005D836E837F8318960D911C9119972885C5
:10769C003985201B310B288739879E01C8DFB8DF5D
:1076AC000E945B3D0023C9F233DFB9F239D03DD0E3
:1076BC008E010E94C83E0023D9F4CFCF0091AD0FAC
:1076CC0000238E0151F00E94A03E002331F295DF81
:1076DC000E94AA3E002361F4C0CF0E947F3E00238B
:1076EC0009F4BBCF8ADF0E94893E002309F4B5CF91
:1076FC0000E00093AE0FA1EABFE00D930D930D9344
:10770C000D930D930D930D930D930D930C938FDFA0
:10771C00008301830093AD0F2A96A991B991089526
:10772C000D911D912D913C91089501CF0E9477F4FC
:10773C0080E013D000E00D930C931197FD010283B0
:10774C00038304830583068307830087018783955E
:10775C00823078F3E4E00C9488F4A1E2B0E1082FD5
:10776C0010E04AE050E00E9479F1A00FB11F08959B
:10777C003B2F6A2FD801223010F000E01EC0022FE0
:10778C001FD0E1E2F0E1E00FF11F1FD01197008351
:10779C00118312961AD0139702831383149615D063
:1077AC00159704831583169610D0179706831783A5
:1077BC0018960BD00087118701E0A62FB32F0895E0
:1077CC0010E04AE050E00C9479F10D911C91089571
:1077DC000E9475F4D801290180E0082FF1DF21E225
:1077EC0030E1200F311FF90106811781FD0146811F
:1077FC00578104171507F1F4F90100851185FD0176
:10780C004085518504171507A9F4F90100811181F0
:10781C000D931C93119702811381FD010283138335
:10782C00F90104811581FD0104831583F201808324
:10783C0001E004C08395823080F200E0E6E00C9415
:10784C0086F40E9477F480E003C08395823060F464
:10785C0084DFFD0106811781012BB9F700851185A5
:10786C00012B99F7082F01C001E0E4E00C9488F497
:10787C000E9474F42B9700E6402E0AE0502E7CD028
:10788C00268537852130304009F070C02089318938
:10789C002030384009F06AC02289338924303640C0
:1078AC0009F064C006A117A16BD02681378102179D
:1078BC00130749F461D000A511A562D0208531854C
:1078CC000217130709F052C057D02489358921308B
:1078DC0000E0304031F0248935892230304009F005
:1078EC0046C0048D158D0F831887068D178D09875B
:1078FC001A879E018E010F5F1F4F6ADF602E3CD0EE
:10790C00248935892130304089F506E010E0F201F8
:10791C003696DE0111960E94A4F4662019F491DFCC
:10792C00202F01C028818E010F5F1F4F21DF06E041
:10793C0022D0369628D00E94A4F40AE01CD0769669
:10794C0022D090960E94A4F406E019D01CD0169672
:10795C000E94A4F40AE013D016D056960E94A4F408
:10796C0002E009D0048B158B01E001C000E02B96DE
:10797C00E7E00C9485F410E0E0E6FAE0089510E0FE
:10798C00E8EFFFE00895A0E6BAE008955B2F4A2FD8
:10799C00E7E3FFE609D0000F111FE00FF11F05917F
:1079AC001491A42FB52F0895A3ECBFE00D911D9158
:1079BC002D913C9108955B2F4A2FEDE3FFE6EACF22
:1079CC005B2F4A2FE3E4FFE6EFDFE00FF11F04919A
:1079DC00A42FB52F089513D011F400E00CC01BD0C8
:1079EC00E1F31DD0D1F31ED0C0F327D034D036D064
:1079FC000E94EDB801E02496EAE00C9482F40E9417
:107A0C0071F424974801290100912B0F002308954C
:107A1C009A938A93C8010091790E00230895082D3A
:107A2C0009290895B3DF0815190508951BD08201A3
:107A3C0020D00E94CAF128D033C014D0840120E099
:107A4C0030E001501040204030404AE522D070E038
:107A5C000E94CAF119C0005B1FD022C04AE09201FB
:107A6C008E010895ECE2FFE080819181A281B381C7
:107A7C00089520E030E001501040204030404AE5AD
:107A8C0050E060E070E00895080F191F2A1F3B1F9B
:107A9C00089550E060E008951F4F2F4F3F4F089519
:107AAC00088319832A833B830895A9DF11F400E02E
:107ABC00A2CFB1DFE1F3B3DFD1F3B4DFC0F3BDDFAD
:107ACC00CADFCCDF0E94A2B801E095CF0E9473F40C
:107ADC006297C801D90157D011F400E037C09BDF81
:107AEC00E1F355D0D1F356D0C0F3ECE2FFE0408087
:107AFC0051806280738052D05CD0ADDF5BD02AD0D5
:107B0C000E94EDB85FD0488559856A857B855DD02C
:107B1C00488759876A877B87FD01048115812681F7
:107B2C0037814C855D856E857F854FD04C875D8711
:107B3C006E877F870085118528893989200F311F31
:107B4C00288B398B07D00C5F1F4F0ED06296E8E064
:107B5C000C9484F44AE09E01285F3F4F8E010895F7
:107B6C009E012C5F3F4F8E010E94A2B801E0089548
:107B7C000E9477F430D0D90114E09E0108950E9440
:107B8C0075F42897280140CF1BDF402E5524082F71
:107B9C00092B0895FBDE0817190708958C0169DF7E
:107BAC000C94CAF170E00E94CAF118D01CD020D0FD
:107BBC0024C014C00C831D832E833F830895BA9375
:107BCC00AA93D801F3DE1397089512C0200F311F2A
:107BDC002883398308952497C8010895040D151D31
:107BEC00261D371D0895488159816A817B8108952E
:107BFC00400F511F621F731F0895488359836A8376
:107C0C007B8308950E9475F42E97BCDF11F400E07D
:107C1C0015C001DFE1F317D0D1F318D0C0F300E0A9
:107C2C001DD020D0088709870A870B870C870D8702
:107C3C0009D0820116D00FDF4AE092DF2E96E6E0E3
:107C4C000C9486F40FCF042D052908959FDE04159E
:107C5C00150508950C9102950F7010E020E030E0AE
:107C6C000895EFCE0C830D830E830F830895980136
:107C7C0012E005D011F400E0089501E0089508E049
:107C8C000E94434B00230895980112E005D011F493
:107C9C0000E0089501E0089508E00E94274B0023BE
:107CAC000895229712E09E01EADF11F400E012C061
:107CBC00288139812F30374218F000E010E003C0E2
:107CCC0014D00F5F1F4F0883198312E09E01E4DF6D
:107CDC0069F301E022960895088119812A813B817C
:107CEC00D3DEDEDE14E09E0108950881198108952B
:107CFC00B4CE980114E005D011F400E0089501E031
:107D0C0008950AE0BDCF980114E00AE0C6DF11F433
:107D1C0000E0089501E008952BDFF3DF11F400E09B
:107D2C0005C0DADF0AE0B9DFD1F301E02496E4E024
:107D3C000C9488F4980114E005D011F400E0089537
:107D4C0001E008950EE09CCF980114E00EE0A5DF51
:107D5C0011F400E0089501E008950ADFF3DF11F457
:107D6C0000E0E4CFB9DF0EE098DFD1F301E0DECF25
:107D7C00980114E005D011F400E0089501E0089595
:107D8C0002E17ECF980114E002E187DF11F400E0FC
:107D9C00089501E00895ECDEF3DF11F400E0C6CFA6
:107DAC009BDF02E17ADFD1F3E1CF32DE11F400E0A8
:107DBC0008C00BD0E1F3EBDED1F3FDDDECDEB8F364
:107DCC0001E08991999108951296F5DD012B0895A2
:107DDC008A93802F20DE11F400E008C0F6DFE1F377
:107DEC008823D1F3EDDD0817B8F301E089910895EC
:107DFC0028D011F400E0FFCD0EDEE1F3E6DFD1F385
:107E0C00C3DEC1F3D8DDC7DEA8F3AA2399F3820140
:107E1C000A1780F302D01DD057CE20E030E0AC0121
:107E2C0060E070E020D04A2F34DE70E0E1DE8A01A1
:107E3C009B0142E32EDE70E00FD032DE42E3940170
:107E4C0008950E9471F4C7DE4901A42FDDCD2C5F8B
:107E5C003F4F8E010C94EDB80E94CAF1025F1A4993
:107E6C002F4F3F4F089541505040604070400C944C
:107E7C00CAF1E7DF11F400E0BECDCDDDE1F3A5DF03
:107E8C00D1F382DEC1F397DD86DEA8F3AA2399F342
:107E9C0082010A1780F3C1DF01D016CE8E010C943B
:107EAC00A2B80E9474F424972801622E6CDE11F49F
:107EBC0000E020C0B0DDE1F388DFD1F381DD802F5D
:107ECC0090E0C1DEA9F377DDC2DE90F3662081F38A
:107EDC008C01061568F3C2DEA20116D0C4DF462D54
:107EEC0012D073DE8A019B0142E30DD0B5DF00DFB7
:107EFC0005D001E02496E7E00C9485F420E08E0197
:107F0C000C9446B840E050E060E070E0089580DDED
:107F1C0011F400E005C03BDEE1F33CDED0F301E000
:107F2C008991999108952BDE11F400E00EC073DD58
:107F3C00E1F389DED1F38ADEC0F378DD44E09E0103
:107F4C0086DF07D00CD089F701E02896E6E00C9488
:107F5C0086F40C811D812E813F81089504D0012B64
:107F6C00022B032B08950081118122813381089506
:107F7C000E9473F42497380106DE11F400E05DC012
:107F8C004ADDE1F3062D0729C9F300DD06151705B7
:107F9C00A8F358DE830162DE64DEAADE00E3402E25
:107FAC000FE0502E59D080819181A281B38144E0A1
:107FBC0056DD47D0D3DF29F480839183A283B3832A
:107FCC00DDCF4CE1920143DF4CE192012F5D40DFAC
:107FDC0041E120E33FE0225C3BDF43E020E33FE074
:107FEC00205B3F4F8E012DD0ED5AFF4F6082718286
:107FFC0033D0E65BFF4F008107FF02C001E001C0F8
:10800C0000E02AD0E35AFF4F008326D0E65BFF4FF7
:10801C0000810F7700830091800E023069F000E040
:10802C001BD001A30091800E002321F00091800E43
:10803C00033010F000E0048301E02496E8E00C9497
:10804C0084F40E94EDB808C0E0E3FFE08CDF00345C
:10805C0012442F4030400895E0E3FFE00895E5E836
:10806C00FFE027D020D019F410918D0F01C010E043
:10807C0040918E0FF1DF03E650E051930A95E1F742
:10808C00E5E8FFE02083318310938D0F40938E0F32
:10809C000895E2E7FFE00DD00FC0E4E7FFE009D060
:1080AC00293B3B400895E3E8FFE000811181012B5F
:1080BC0008952081318108952031374208950E941E
:1080CC0075F424975FDD11F400E02AC0A4DCE1F321
:1080DC0032D009F036D0B7DDB9F3B8DDA8F3A6DCA1
:1080EC0044E020E33FE0DADE4CE124E33FE0D6DE7F
:1080FC004CE121E53FE018D029F0EAE7FFE00081F0
:10810C000068008341E12EE63FE00ED029F0EAE75B
:10811C00FFE000810F77008343E020E83FE023DDA0
:10812C002496E6E00C9486F48E010E94A2B800918D
:10813C008D0F0023089544EA50E00E9437F10F3F61
:10814C0008950FEF44EA50E00C9451F10E9475F43D
:10815C0042DD290118DD11F400E0E2CF5CDCE1F333
:10816C00EADF09F0EEDF13DDB9F314DDA8F316DD59
:10817C00C801D90113D0BCDD4DE471DC0E94A2B85A
:10818C000DD0035B0FD083E0B9DEAFDD2A813B81DC
:10819C000F5F08D08A95C1F701E0C2CFECE2FFE097
:1081AC00E2DE58CC79DC59CC0E9473F42497280178
:1081BC003901E9DC11F400E040CF2DDCE1F3BBDF49
:1081CC0009F0BFDF40DDB9F341DDA8F32FDC40E55A
:1081DC00930164DE01E031CF12DC11F400E00BCC32
:1081EC001ADCE1F31CDCD1F31DDCC0F326DC80DDF2
:1081FC004DE4920110CE03DC11F400E0FCCB0BDC5F
:10820C00E1F30DDCD1F30EDCC0F317DC71DD40E5DE
:10821C00F0CF1ADF10F000E008952AD010F000E043
:10822C00089537DF10F000E0089537DF10F000E01C
:10823C000895E6E7FFE02FDF10F000E00895C5DDBC
:10824C0021F00FD010F400E0089500917A0F04365D
:10825C0010F000E008950FD011F400E0089501E053
:10826C000895A9DBE8E7FFE024DF02171307089560
:10827C00EEE6FFE0EBCE00E81FE00E94EF480023A3
:10828C000895E2DE10F002E80895F2DF10F003E842
:10829C000895FFDE10F004E80895FFDE10F005E805
:1082AC000895E6E7FFE0F7DE10F006E808958DDDAF
:1082BC0021F0D7DF10F407E8089500917A0F043607
:1082CC0010F008E80895D7DF11F40EE8089500E0E7
:1082DC00089575DC44DE11F402E825C073DC2BD064
:1082EC00D8F7DC966FDC27D010F003E81CC024D044
:1082FC0010F004E818C023D0293B3B4010F005E8EF
:10830C0012C01DD0D9DE10F006E80DC05DDD21F0E5
:10831C000DD010F407E807C012960C91043610F03B
:10832C0008E801C000E0A991B991089544DB08D098
:10833C000217130708958BCE149602D0BDCE129659
:10834C002D913C91119708953ADC09DE11F402E865
:10835C002EC038DCF0DFD8F7DC9634DCECDF10F024
:10836C0003E825C0E9DF10F004E821C0E8DF293B71
:10837C003B4010F005E81BC0E2DF9EDE10F006E883
:10838C0016C022DD21F0D2DF10F407E810C01296DF
:10839C000C910F77043610F008E809C015968D0182
:1083AC000E94EF48002311F40EE801C000E0A991EF
:1083BC00B9910895E4DB11F400E0C7CD2CDB00E0AB
:1083CC0041F050DC40DCC1F341DCB0F32FDB44E086
:1083DC00C7DBBBCD0E9471F4FEDB94DDCDD031F058
:1083EC002A95E1F0225009F440C004C0F801A081A4
:1083FC00A43610F000E0FFCA0A2FC8D01AE0019F83
:10840C00A019A883E82F0081C1D0E82F0083A02FEA
:10841C00BDD0019FA0D0E82F008356CBFC0100817A
:10842C001181003127E2120728F7A02F4AE00E94A1
:10843C0095F1ABD0A019A8837CD09AD0A02F7CD07A
:10844C0089D077D095D0DE011196402E75D09DD075
:10845C0040184C926ED08CD0402E6ED071D01197AB
:10846C000D911C91FC0185D02FCBFC018BD00030E1
:10847C0041EE140745EF240745E0340708F0BACF66
:10848C00A02F4AE080D0A019A8834CD06BD0A02F8D
:10849C004BD060D047D066D0DE011196402E44D030
:1084AC0074D040184C923ED05DD0402E3DD048D078
:1084BC00FC0139D0402E56D037D0480166D0401838
:1084CC0011964C92E82F808291822283338384010F
:1084DC002BD02801622E282D58D020192295207FD0
:1084EC000C91022B0C93E82F4082518262823383D1
:1084FC0011968201262D18D0502F4AE0549F401817
:10850C004C9230D0402EFFDC3ED0042D0019029549
:10851C00007FFD011081102B1C93139747DAFC018F
:10852C0022D0D2CAE82F1FDD4AE0B3DA70E00C94F7
:10853C00EEF1E82F008111814AE050E00C9495F1A6
:10854C0028D04018429400EF4022FD0100810429FC
:10855C000C9308951ED0A019A295A07F08810A2B18
:10856C0008830895E82F00831183228333830895B1
:10857C00E82F008311830895488349834A834B83F2
:10858C002A950895F0CC0E94EEF103C04AE00C94B9
:10859C006BF1102F0AE0109F08950E9473F424973A
:1085AC00D801F80100E002C031960395021760F47F
:1085BC00108112951F701A3010F000E03ECD108122
:1085CC001F701A3088F3F9CF9DDCD6DF29F02A957D
:1085DC0081F0225099F1F1CF0C910A3970F7202FCC
:1085EC0022952F701AE0219F0F70000D08830C93B9
:1085FC00F1CDA6DE2A39394900F70C9102950F709E
:10860C0010E04AE00E9479F12C912F7030E0DEDA14
:10861C0053D048EE53E00E9479F12801082F0F70D7
:10862C0010E044E650E00E9479F1040D151D2881FC
:10863C003981CCDA11972D933C93CCCDC3DA0A391E
:10864C0019492949394908F0B8CF04DB4AE00E949E
:10865C00CAF14C914F701DDA660F660B762F2AD03B
:10866C00FDDA48EE53E060E022D044E612DA9ADA02
:10867C001196F0DA40EA56E861E026D00C912AD047
:10868C0040E157E241DC0E94CAF193DAACDA12D035
:10869C00E5DA40E856E968E90AD040E452E46FE0D4
:1086AC0081DA13974D935D936D937C9393CD0CD09E
:1086BC00082F10C09DDAA1DA1196FD018081082FD8
:1086CC0002950F7010E0089570E00E94CAF1280125
:1086DC00390108950F7010E020E0220F220B322F89
:1086EC0008950E9477F42697802F8A3510F00EE5B6
:1086FC000EC129D110D10E9437F1ECE8FFE60C94A1
:10870C0018F42CD118DED0F40E94ECEDA8DC26D1A4
:10871C00EEE6FFE028DFF89400E0E7E2FEE0038BF2
:10872C00048B058B068B78940093630E1AD10E94F0
:10873C0037F1033008F4EAC000E6E9C00AE5E7C007
:10874C000DD1E5DB002311F40BE5E1C007D1EBDB28
:10875C00002311F00CE5DBC00E94ECEDFFD008DC2F
:10876C00002321F77CDC0DE5D2C0F8D0003442E4C4
:10877C0014074FE0240740E03407C0F40A831B833E
:10878C002C833D839E018E010E5F1F4F64D100230D
:10879C0011F401E6BCC0A9DAC6DB0023D9F60E94AD
:1087AC00ECEDA3DAE5DB002309F6DCCF02E6AFC083
:1087BC00BED010F00FE5ABC0D2DB39F001E00E9467
:1087CC00945B002311F408ECA2C0C8D000938E0F68
:1087DC00ADCFB2D019F4CBD000FF02C00AEC97C0D9
:1087EC009ED00E7F0083A2CFA7D0C1F7C0D000FDD2
:1087FC00F5CF95D00160F6CF9FD081F7B8D000FDB2
:10880C00EDCFB9D011601183EDCF96D039F7AFD041
:10881C0000FDE4CFB0D00064F6CFE8E4FEE09EDBD0
:10882C0011F009EC74C083D028F699DBA5D021F0A7
:10883C000E9437F1006203C00E9437F10F7D9CD07B
:10884C000E9451F10E94B97771CF88D0013098D035
:10885C0009F46CCFAFCF6ED008F0ACCF46E451E04A
:10886C00EFCF68D008F0A6CF47E451E0E9CF62D053
:10887C0008F0A0CF45E451E0E3CF59D008F09ACFEF
:10888C006EDB4AEC50E021F00E9437F1086003C027
:10889C000E9437F1077F4AEC50E0D2CF5FD0002E18
:1088AC0008E06DD008F086CF6FD00F70102D1295A8
:1088BC00107F102B012F44E451E0C2CF4FD0002E7B
:1088CC0000E15DD008F076CF5FD0007F102DF1CFA6
:1088DC0045D0033040E033D008F06CCF02302FD0BD
:1088EC0021F44AD037D00860AACF013028D044D028
:1088FC0019F430D00460A3CF2DD0A1CF2FD00D30E0
:10890C003FD008F057CF43E451E09ACF00E02696D1
:10891C00E4E00C9488F420EF31E090E024C038D0EF
:10892C00006211830083E8E7FEE00081089535D0F2
:10893C0040E005C032D024C0E0E5FEE0B6CB140721
:10894C00240734070895AAE4B2E004E0809FA00D48
:10895C00B11D08950E9437F1037F0895AD010C9469
:10896C003FF120EF31E0280F391FA9010895E2E60D
:10897C00FEE0008108950CC043EC50E00895001611
:10898C00104020403040089544E451E00C9437F1FD
:10899C00E0E5FEE0008111810895AD010E943FF1F8
:1089AC00023008950E9475F4802F8A3510F000E093
:1089BC002BC0C9DF78DBC9F04080518047D9B8F3B0
:1089CC000091640E0071059505950595059539F492
:1089DC0001E0A1DF0E9451F1820140D911C002E0F7
:1089EC009ADF0E9451F138DB0AC000E020EF31E041
:1089FC00280F301FA9010E9451F1EEE6FFE0C2DD05
:108A0C00AD010E945CF101E0E6E00C9486F40E945A
:108A1C0077F480E090E0A0E0B0E00FEFA2DF0E94DE
:108A2C0051F100E01AD96AE472E0AC01440F551F11
:108A3C00440F551F640F751FAB010E945CF18F5FD3
:108A4C009F4FAF4FBF4F8A359007A007B00728F351
:108A5C00E4E00C9488F40E9473F4289728013901FF
:108A6C00ECE2FFE08FDDA6D80E94CC3CD80181E07F
:108A7C0090E005C06EDA0A5A0FD89CD80196A81758
:108A8C00B907C8F044E09E018E010C5F1F4F0E9495
:108A9C00EDB82BD92A813B81F20140815181628151
:108AAC007381041715072607370721F7F301808315
:108ABC00918301E001C000E02896E8E00C9484F476
:108ACC0006D011F400E001C001E021960895219731
:108ADC009E0100E00E94F04A00230895F8DF11F493
:108AEC0000E004C0088107FDFBCF01E0219608954A
:108AFC008A93802F21D011F400E019C010E021D00E
:108B0C00D9F3882321F412E521D021F4F5CF10E01C
:108B1C001DD091F311E01FD079F311E021D061F356
:108B2C0010E021D049F310E022D031F301E089911B
:108B3C000895BA93AA93D80110E819C014961C9101
:108B4C00149701E015C013961C91139702E010C006
:108B5C0012961C91129704E00BC011961C91119760
:108B6C0005E006C01C9106E003C015961C9100E0C0
:108B7C000E94144B00230895F8012081243610F034
:108B8C0000E0089520E0F8013081332311F401E076
:108B9C00089530E008C02395422F4F704A3010F0F2
:108BAC00207F205F3395F80140813417A0F3208398
:108BBC0001E00895037011F401E0089500E00895B8
:108BCC00F801238126FF15C023812F7B18D061F07B
:108BDC001CD079F00FD018F0207F205F2383F80190
:108BEC000381005F03830895223119F020E0F8011E
:108BFC00238308952E5F33813E5F33830CC0338112
:108C0C003F7B3383322F307208952F7D33813F7D2C
:108C1C00338322310895322F3F703A300895BA933E
:108C2C00AA93D80198012B5F3F4F26D011F400E096
:108C3C0025C015960C91159707FDF9CF9D012C5F5A
:108C4C003F4F01E01AD099F39D012D5F3F4F02E099
:108C5C0014D069F39D012E5F3F4F04E00ED039F321
:108C6C009D012F5F3F4F05E008D009F39D0106E001
:108C7C0004D0E9F201E002C000E02CCFA991B99137
:108C8C00089557DF11F400E00DC058DFE1F35BDF0E
:108C9C00D1F35EDFC1F361DFB1F364DFA1F365DF14
:108CAC0091F301E0EBDF0895BA93AA932197D801D1
:108CBC009E01E2DF11F400E00CC03EDFE1F348DF7F
:108CCC00D1F34BDFC1F34EDFB1F3188150DF99F3D1
:108CDC0001E02196D3DF08952CDF11F400E007C0EA
:108CEC002DDFE1F330DFD1F340DFC1F301E0C6DF6C
:108CFC0008950E9476F42197D801F801058107FFA9
:108D0C0002C000E036C04C90042D007F0139C8F73A
:108D1C00042D0F700A30A8F7FD018281882389F396
:108D2C00982F9F700181EAECFFE60C9418F48233C3
:108D3C0040F780738033E1F09A30D0F0E2CF81338A
:108D4C0000F78033A9F09A3098F0DBCF8A32C8F65E
:108D5C009A30B8F6488221E08E010E94D34200235B
:108D6C0081F208810CD021F4FD010281093248F610
:108D7C0001E02196E5E00C9487F4F20100811ADF02
:108D8C0000230895F8012581322F307811F000E08E
:108D9C00089541DF10F000E00895207F213510F098
:108DAC0000E00895F801248136DF10F000E008950A
:108DBC00207F213510F000E00895F8013381232F36
:108DCC002F70432F407479F0432F4F7111F400E052
:108DDC000895307121F02330A8F000E008952A3076
:108DEC0088F000E008953073313210F000E00895FF
:108DFC00303221F4243030F000E008952A3010F0A5
:108E0C0000E0089501E008952223F8012381F1F098
:108E1C00223190F0223161F0213211F0203221F414
:108E2C00F8013381385103C0F80133813251338357
:108E3C00F8012381206204C0222319F422E1F801F5
:108E4C002383F80103810064038308952F7BF801C9
:108E5C00D6DE41F0DADE59F0CDDE18F0207F205F4F
:108E6C002383BDCE223119F420E0F8012383089529
:108E7C000E946FF4C801D901F901428099D05524A0
:108E8C00028175D0FC0197D0238344240AC00CE8DE
:108E9C0010E0E42DF0E0319792D07ED0611F711F6D
:108EAC0094D04394FD016180562C52940FE05022D3
:108EBC009924062D0F7010E05801052D87D00A0D4E
:108ECC001B1D401691061CF30FE060220AE0509E19
:108EDC00002D060D033060F00C910F701C91129553
:108EEC001F702AE0129F000E002D49DF09F055D0AB
:108EFC0044240BC003591E4F2F4F3F4F5CD033837C
:108F0C00042D3DDF09F049D0439455246C900FE0BB
:108F1C0060220C9102950F7010E058D0060D151DB3
:108F2C0040165106FC0156D02CF355D070D0E82FCA
:108F3C0042D03383FD0143803BD0038118D0322FC4
:108F4C0040E15EE021D0448033D0048110D0322F38
:108F5C004CE350E019D045802BD0058108D01CD0B3
:108F6C00621F721F32D001E0ECE00C9480F4029589
:108F7C000F7010E04AE050E00E9479F1040D151DCD
:108F8C00212F220F220B089560E041D033D0621FB5
:108F9C00731F40D0FD0108952DC0FC0133D00F5F2D
:108FAC001F4F2F4F3F4F008311832283338308952C
:108FBC000FE04022089500831183228308950E0F41
:108FCC001F1FF801049110E0089524C04AE050E0FE
:108FDC000C9479F117C040E851E561E0089517D081
:108FEC00801A910AA20AB30A08954CE350E060E09B
:108FFC0070E00895FC014081518162817381400FC2
:10900C00511F08950081118122813381089570E0F0
:10901C000C94CAF1408351836283738308950E9438
:10902C006BF4602E2901F801D5DFD5DF70E00E94CA
:10903C00EEF1C801D901E62D80809180A280B38029
:10904C00CADFCDDF6C017D018401950140E15EE05A
:10905C0060E070E00E94EEF1802F40E15EE060E0A5
:10906C00BEDFF201838382010D5F7FD011F400E03B
:10907C0078C084019501B9DF0E94EEF1802FB5DF35
:10908C000E94CAF1801AF201848382010C5F6DD0B8
:10909C0071F3F201858282010B5F67D041F380E0AE
:1090AC0065D083599E4FAF4FBF4F062D68DE09F038
:1090BC0062D066D090F0F20160828D569140A04053
:1090CC00B040062D5CDE21F081509040A040B040B5
:1090DC00C81AD90AEA0AFB0A04C0639404E66016AB
:1090EC0000F3ECE8F0E0849141D04AD0B8F0062DC2
:1090FC000395F2010183820137D009F4B8CFECE873
:10910C00F0E07724E60DF71D0491801B36DE21F08C
:10911C0001E0601609F48150C81A17C00CE810E081
:10912C00E62DF0E031964BDF800F911FA11FB11F90
:10913C0024DE39F0E62DF0E03196E130F04009F410
:10914C001AD063940CE0601680F2F201C2828201A4
:10915C000E5F0BD009F48BCF820118D009F487CFA6
:10916C0001E0E0E10C947CF40F5F0FC090E0A0E014
:10917C00B0E0662408958F5F9F4FAF4FBF4F0895A7
:10918C008C159D05AE05BF0508951F4FF5DC00231A
:10919C000895BA93FA2FD801203107E2300710F066
:1091AC0000E014C070E0890120E030E014DF0E9480
:1091BC00CAF14D915D916D917C91400F511F621FD1
:1091CC00731F7C936E935E934E9301E0AF2FB99116
:1091DC0008952697F8012281288321812983008113
:1091EC000A8300E00B830C830D830881002331F488
:1091FC000981002319F40A81002381F08E010E5F8E
:10920C00C4DF11F400E00BC08E01AEDFD9F38E0188
:10921C00BDDFC1F38E016DDD0023A1F301E02696C5
:10922C0008959A938A93C801A7DC8C010F5F1F4F96
:10923C00A3DC02968C01A0DC8991999108959A93F4
:10924C008A93C80121E00E94D34221E08C010F5F78
:10925C001F4F0E94D34221E002968C010E94D34200
:10926C0089919991089520E0E8ECF0E00DD06EE53D
:10927C0071E00CD0E8E9F0E013D06EE871E006D0B4
:10928C002395203388F3089530E00AC0620F731FD2
:10929C00AB010C9451F1E20FF31FAF010C9451F19F
:1092AC00E20FF31F04910895392F082EF80160E0A6
:1092BC00222319F48EE591E002C08EE891E009D0EA
:1092CC000E9437F101936395603390F3802D932FB7
:1092DC00089570E0860F971FAC010895392F282E42
:1092EC00F801223010F000E011C060E02223008170
:1092FC0019F48EE591E002C08EE891E0EADF0E945D
:10930C0051F131966395603388F301E0822D932FF0
:10931C00089520E068EF70E0FB013796B5DFEEEBC7
:10932C00F1E0B9DFFB01BCDFE5ECF1E0B4DF239544
:10933C00273080F320E0FB01B096B2DFECECF1E0DB
:10934C00AADFFB013E96ACDFEEEDF1E0A4DF239546
:10935C00223188F308950E9477F4802F0E9441B740
:10936C00002311F400E028C00DE10E941CB7082F67
:10937C000E941CB7805039F08A9551F08A9559F0AB
:10938C008A9569F0EFCF8EEB91E0A7E0B0E011C0C9
:10939C0085EC91E0FACF8CEC91E0A2E1F7CF8EED69
:1093AC0091E0FBCFAC010E9437F10E941CB70196F3
:1093BC00B395BA17B8F301E0E4E00C9488F43B2FB2
:1093CC006A2FD801205039F02A9551F02A9559F07E
:1093DC002A9569F00FC0EEEBF1E017E020E012C027
:1093EC00E5ECF1E0FACFECECF1E012E1F7CFEEEDC9
:1093FC00F1E0FBCF00E009C00D91AF010E9451F1EB
:10940C00319623952117C0F301E0A62FB32F0895B1
:10941C0023978E0158D010E000E00E945FB206E363
:10942C0011E0065F1F4F48D010E00CE00E945FB2C5
:10943C0000E114E045D007E31FE6E3ECFFE04081D8
:10944C00518162817381440F551F040F151FF80160
:10945C000591149135D00AEC1BE52ED0249611E021
:10946C0000E00E945FB2E6E3F1E03196049127D070
:10947C00E6E3F1E0049124D00CEB1BE51DD024961F
:10948C0011E00BE00E945FB20A8119D00B8118D059
:10949C000C8116D000EF1BE50FD026960E94FEB271
:1094AC00F89400E717E1E7E2FEE004831583789473
:1094BC000E940FEA2396089520E00C94B4F410E077
:1094CC001A930A9308953B2F2A2FD80100E00C938E
:1094DC00FD0101830283EAE2F1E00491015421F1E0
:1094EC00035089F1025039F1045049F00350A9F0AE
:1094FC000A9539F10A9519F10450F9F026C0319604
:10950C0004913197013611F401E020C044D00C369F
:10951C0011F407E01BC006E019C03DD0023711F46E
:10952C0003E014C005E012C036D0023711F404E099
:10953C000DC008E00BC002E009C009E007C00AE05A
:10954C0005C00BE003C00CE001C000E011960C93C9
:10955C001197349604913497003271F0349614912B
:10956C0034971053110F110F110F34960491349737
:10957C000053000F010F0C9335960491359700534F
:10958C001C91100F1C933A9604910053FD01028319
:10959C00A22FB32F089532960491329708958A938F
:1095AC00802F04E10093280E0E9408760091280E6B
:1095BC00002321F40E941D7600E005C00E940C7669
:1095CC0004D0A1F701E089910895082F0E944276FA
:1095DC00002308950E9477F4802FD9011BD069F0E5
:1095EC00F4DF49F412D039F40E946F760C930E9488
:1095FC00367607D003C00E941D7600E0E4E00C94A0
:10960C0088F40E941D7601E008950E940C7601ED0D
:10961C00DDCF812F00EDC3DF002308959A938A9349
:10962C00902FF7DF41F00BD021F4CFDF11F4E9DFFD
:10963C0003C00E941D7600E0899199910895092F2D
:10964C00C5CF16D021F0FBDF39F00E941D7600E06B
:10965C00E4E00C9488F41196082F8A95002331F0DD
:10966C000C910E9442760023B1F3EFCFCADFF0CF0A
:10967C000E9477F4902FD901CCCFFADF31F0DFDFE5
:10968C0011F4C3DF49F00E941D7600E0E4E00C9475
:10969C0088F40E9436761196082F8A95002341F0A3
:1096AC000E946F760C938823A1F30E942C76F3CF43
:1096BC00A8DFECCFFED02F9780E05CD190E05ED19C
:1096CC00FE013A965BD1FE0159D183958530A8F302
:1096DC0080E004C0FDD08430E8F384E00E94A2B2A4
:1096EC0003C00DD10E94FEB215D106EC1CE51CD1B5
:1096FC0010E002E113D119D1A9F3843049F41AD145
:10970C00B9F480E000E0E5D08530E0F380E045C0BE
:10971C00843070F400915E0E003350F000915E0EB8
:10972C000A3330F410915E0ED7D01083D1D0DACF3B
:10973C0000915E0E063009F4BAC000915E0E053041
:10974C0051F4882309F08A95C7D00081002309F4CD
:10975C00D6D0B2D0C7CF843070F400915E0E0931F0
:10976C0051F400E308D1B1D0843008F0BBCF00E352
:10977C00B3D00083DBCF00915E0E023009F0B1CF85
:10978C00882339F080E098D083958530E0F380E031
:10979C00A9CFA7CFB4D00E94FEB2D3D00DED1CE55B
:1097AC00C3D011E002E1BAD0C0D0A9F3843001F5E6
:1097BC00C1D071F580E090D0108190D0008110174D
:1097CC0009F45AC0A7D002E21DE5AED0BAD009E325
:1097DC001DE5AAD00E94FEB2F894E7E2FEE000ED8F
:1097EC0017E0028313837894F89400EA1FE05EC0BC
:1097FC00843070F400915E0E003350F000915E0ED8
:10980C000A3330F410915E0E69D0108361D0C3CF4F
:10981C0000915E0E063009F44AC000915E0E0530D0
:10982C0059F4882309F457CF8A9558D00081002326
:10983C0009F465D043D0AFCF843078F400915E0E3C
:10984C00093159F400E3FE013A963FD0843008F018
:10985C00A2CF00E343D00083D9CF00915E0E02303B
:10986C0009F098CF882339F080E028D08395853093
:10987C00E0F380E090CF8ECF8395843008F49BCFBB
:10988C0080E02AD000812FE131E0280F391FA90197
:10989C000E9451F183958430A0F33CD004EF1CE579
:1098AC0043D04FD00BE01DE53FD04FD056D02F9674
:1098BC0059C09A938A9308955DD003C000E0FE01CD
:1098CC003A96E80FF91F008350C0E80FF91F008388
:1098DC000AE24BD0839508954ED002C0FE013A9611
:1098EC00E80FF91F089501E00E9441B211E000E079
:1098FC000E945FB201EA18E545D00E94FEB2F894CE
:10990C0000ED17E0E7E2FEE00283138378940895FC
:10991C000E9441B210E016C011E000E00E945FB25C
:10992C008E0133D00CEC13E52DC022960E946EB73D
:10993C000023089500915E0E0130089501E00E940D
:10994C0041B211E000E00C945FB20E94FEB2F894B8
:10995C0000EA1FE0E7E2FEE00895048315837894A3
:10996C000C94DAE9899199910895FE01E80FF91F99
:10997C000083089500E0FE0135960895E80FF01F6E
:10998C000083089520E00C94B4F41A930A9308957C
:10999C0041D00E94A2B20091B80F002321F0009197
:1099AC00B80F043620F001E044EC50E029D00091CF
:1099BC00B80F0883AFDF0BE411E6B6DF01C09FDF01
:1099CC000ED015D049F02CD0D1F308810436B8F75D
:1099DC00088144EC50E01AD020C00E94B4F420E07E
:1099EC0011E002E020D01BE00AE00C94366820E085
:1099FC008E010E943069802F0E946E688C3308950E
:109A0C000E9451F10C94DA5544E451E00E9451F15A
:109A1C000C94B9778A93219708952196899108958A
:109A2C000881002308950E94076821E0089541DF12
:109A3C00679700E03BD0F0F349D08F7029F488E0B1
:109A4C0003C05DDF0E94FEB204E8FE0190E0E80F67
:109A5C00F91F00835FDF03E512E666DF5DDF2FD0C1
:109A6C0008503CD007E01BE55FDF5FDF59F3009146
:109A7C005E0E033031F4823028F300E276DF8A95F3
:109A8C00E1CF00915E0E043029F48F30D8F600E25D
:109A9C0020DFD8CF00915E0E063031F04BDF89F617
:109AAC0021D0007F082BB0DF67965CCF20E2FE014F
:109ABC0010E0E00FF11F20830395073108952296E3
:109ACC0011E004E10E945FB2082F08951E8B0CE395
:109ADC0008830EE3088B8091BC0F0895102F110F93
:109AEC00110B53CF44E451E00C9437F10E9477F4FE
:109AFC0067970091BC0F02950F70083028F0F2DFC9
:109B0C000F7044E451E07CDF00E0D0DFF0F3DEDFE7
:109B1C0082958F7003C0F3DE0E94FEB2DE010FE06F
:109B2C0010E022E0829F00191109A00FB11F04E878
:109B3C000C93F0DE04E612E6F7DEEEDEC0DF0195F4
:109B4C00CDDF06EE13E5F0DEF0DE31F300915E0EB4
:109B5C00033031F4873000F700E20C938395DCCFAF
:109B6C0000915E0E043031F48823B1F200E20C93C4
:109B7C008A95D2CF00915E0E063049F0DBDE59F6A5
:109B8C00B1DF0F708295807F802B082F3DDF6796A9
:109B9C00E4E00C9488F43EDF0E94A2B20091800EA7
:109BAC00033020F002E042E451E02ADF0091800E05
:109BBC00088301C0A4DEAEDE0EE913E6B5DE20E0BC
:109BCC0011E001E030DF1BE00AE00E9436680FDF95
:109BDC0039F00881033070F704D042E451E016DF0D
:109BEC001CCF0E94FEB2088108951DDF15E1089577
:109BFC0011DF0091B90F002321F00091B90F043649
:109C0C0020F004E14FE351E0FBDE0091B90F13D0DB
:109C1C0001C075DE7FDE0EE114E620E0DEDEE7DE5D
:109C2C0049F0FEDEB1F30881043698F7DADF4FE332
:109C3C0051E0ECDEF2CE088301E00C9441B2EADE96
:109C4C000091BA0F002321F00091BA0F043620F0D6
:109C5C0005E140E451E0D4DE0091BA0FECDF01C025
:109C6C004EDE58DE02E314E620E0B7DEC0DE49F03B
:109C7C00D7DEB1F30881043698F7B3DF40E451E046
:109C8C00C5DECBDE0895C6DE00917F0E002361F0A9
:109C9C0000917F0E002321F000917F0E043620F0FE
:109CAC0000E041E451E0ACDE00917F0EC4DF01C066
:109CBC0026DE30DE06E414E620E08FDE98DE49F086
:109CCC00AFDE19F00881043698F78BDF41E451E0E0
:109CDC009DDEA3DE0895EDDD28D02CD0F1F71BD04E
:109CEC0004EB14E605D019F020D019D0F1F73ACED8
:109CFC0049DE20E010E00CE196DE15E100E00E9468
:109D0C00366820E007EF1EE074CE1BD0048F20E0F5
:109D1C0010E00CE16ACF15D0048F0C94A2B2008134
:109D2C00AC010E9451F1319609C08BEC90E00AD045
:109D3C001CE10895AC010E9437F1019301961A952C
:109D4C00089500E0E7EFFEE00895B3DD80E00E94A7
:109D5C00A2B209EC14E6E8DD882389F44CD001E0CA
:109D6C002AD03ED035D0F1F7D0DF1DD03CD0D1F089
:109D7C0081E09D3361F334D025D049F3FDCF8130A0
:109D8C0089F439D002E017D033D022D0F1F7BDDFFF
:109D9C000AD029D039F082E09D33C1F229D012D0FB
:109DAC00B1F2FDCFDFCD00E00E94366821E007EF75
:109DBC001EE00C94306910E0E8DD0DE01BE5E2DDFF
:109DCC00229608950081A9010E9451F1319604C098
:109DDC00A9010E9437F101932F5F3F4F1A95089507
:109DEC0027EE30E0A4CF902F0E946E689C3308952C
:109DFC0023E031E09CCF10E004E10C945FB259DD1C
:109E0C000BD098DFF1F787DF0CE614E671DF19F061
:109E1C0003D085DFF1F7A6CD83E291E088CF0E94D5
:109E2C0077F4A3D069F46BDD8CDD03EF19E57CDDF1
:109E3C000E94FEB20E941CEA2296E4E00C9488F484
:109E4C000E94E13C012B21F40E942DB2F5CF57DD8D
:109E5C0000E010E0088319830E94A2B202EF14E61E
:109E6C0063DD6FDD00EE18E620E06AD075D082D09D
:109E7C0019F3088119810E94DB3E002341F3A1E014
:109E8C0001C0A39500E044DD00EE18E64DDD10E0C6
:109E9C000AE066D007E11BE547DD229610E001E100
:109EAC000E945FB20CEE18E63FDD10E005E10E9467
:109EBC005FB2B0E0BA93AA930DE01BE535DD2296B4
:109ECC0000E020E010E0F801E950F14F2083039509
:109EDC000333B8F355D00E94FE3E002329F42EDD47
:109EEC0006E517E509DDA6CF20E010E002E37DDEF4
:109EFC005ADF40D009F4ACCF8D3331F40E94E63CEC
:109F0C00A01708F4BECFBBCF3BD00E943F3F00232D
:109F1C0031F30E94E63CA01708F4B3CF2CD00E947A
:109F2C00DB3E002309F498CF26D094CF20E012E03A
:109F3C0004E079DD15E102E10E94366821E0089524
:109F4C000E94B4F40E94FEB220E012E005E06BDD4A
:109F5C0015E101E10C94366821E08E010C94306916
:109F6C000E945FB20881198110CD22970091790E61
:109F7C000023089540CD088119810F5F1F4F08956C
:109F8C004A2F27EF3EE00881198108950E946FF453
:109F9C00ECDF69F4B4DCD5DC03EF19E5C5DC0E9419
:109FAC00FEB20E941CEA2296ECE00C9480F400E0D5
:109FBC0008830983E3E8FFE060807180062D0729A0
:109FCC0011F466247724EEE6FFE080819181A28172
:109FDC00B38180908D0F05C092DC00E010E0088307
:109FEC0019830E94A2B20EED14E69EDCAADC02EFED
:109FFC0018E620E0A5DFB0DF402EB3D159F40E9463
:10A00C003540062D072921F083010E94BE3FCBCF9E
:10A01C009BD1C9CF93D101F3088119810E94993F3B
:10A02C00002321F00E94354055240BC00881198172
:10A03C000E94BE3F0023C1F756DC0E941CEACDCF24
:10A04C00539401E065DC02EF18E66EDC10E004E0EE
:10A05C0087DF0CE11BE568DC229610E00BE00E9428
:10A06C005FB20BE91EE65801052D10E04CE050E004
:10A07C000E9479F1A00EB11E850156DC052DE2EF90
:10A08C00FFE60C9418F449D171D140F43FD14CD176
:10A09C0000E31FE00E943069402EF0C05ED10083C7
:10A0AC00018302830383E7C00091800E002341F2F9
:10A0BC0026D104E31FE0EECF0091800E023000F2B7
:10A0CC001ED101E51FE0E6CFEEE6FFE028D14ED130
:10A0DC0028F700917D0E005019F0025019F002C0C3
:10A0EC0015D105C024E013E006E07FDD0FE01CD1A4
:10A0FC000EE61FE0CFCFE2E7FFE03FD12031374241
:10A10C0040F41FDC0EE71DE50FDC10DF02E71FE05B
:10A11C00C1CF23D100830183AEC02DD1293B3B405D
:10A12C00C0F722E012E005E060DD00E1FDD004E7BD
:10A13C001FE026D109F0A2C01ED1293B3B4008F4F8
:10A14C009DC023D110E0E4E7FFE000831183D7DB4F
:10A15C000E941CEA76CFE6E7FFE00FD120313742B0
:10A16C00C0F6E4DE06E71FE095CF0E94E13C012B30
:10A17C0009F466CFDAD068F2E7DE21E008E71FE0E9
:10A18C00FFD009F07BC0D1D008F078C0FED010E031
:10A19C00E8E7FFE0DACF00917A0F0436A0F420E074
:10A1AC0011E002E022DD04E1BFD00AE71FE0E8D0B5
:10A1BC0009F064C000917A0F043608F45FC0E5D052
:10A1CC0000937A0FC4CFC9D000937A0F54C020E00B
:10A1DC0010E004E00ADD02E1A7D00BE71FE05ACF44
:10A1EC0000918D0F023050F0B8D000938D0F43C00A
:10A1FC0001E0EDE8FFE0108110271083A2DB009155
:10A20C008D0F002319F008EF18E602C00FE019E6D5
:10A21C008BDB0E94FEB20E946EB7002379F3009193
:10A22C005E0E043029F300915E0E033009F30091A9
:10A23C005E0E063011F40CE32FCF00915E0E07304A
:10A24C0011F40DE329CF76DB11F4442417C057DB4E
:10A25C00D5CF00E81FE00E94EF48002329F000E86A
:10A26C001FE00E94475A18CF78D00093800F0093BC
:10A27C00810F0093820F43DB0E941CEA72D069F4B9
:10A28C00062D072941F083010E94BE3F002321F4D3
:10A29C000E943540A6CE58D0A0CE0DE3401669F4EE
:10A2AC00552031F43AD0012B022B032B09F44FCF5C
:10A2BC000BE0501608F4C4CEB7CE0EE3401609F4EA
:10A2CC00C0CE552031F429D0012B022B032B09F4DD
:10A2DC003ECF088119810E946540002321F403DBE5
:10A2EC000E941CEA7ECE0BE0501608F4A9CE43DE89
:10A2FC000E948D3F002309F474CE3DDE70CE20E029
:10A30C0010E00CE190DB15E100E016CE20E013E04C
:10A31C0006E089DB15E100E10895E0E3FFE0008150
:10A32C00118122813381089507CE0E94E13CE8E738
:10A33C00FFE02081318102171307089508811981EC
:10A34C000E948D3F00230895EEE6FFE08083918309
:10A35C00A283B38380928D0F08950EE3402E00E00C
:10A36C0008950E946E680CE3401608950034124460
:10A37C002F4030400895E4E7FFE0208131810895BB
:10A38C000E943069402E002308950E946E6800E000
:10A39C0008958A93229700E0088309830E94A2B251
:10A3AC000DE915E6C1DACDDA02EF18E6BDDA0E9446
:10A3BC00FEB201C0A4DAC8DD1ADB29F1BFDFD1F38C
:10A3CC000E9487550023F9F0E3E8FFE0008111813A
:10A3DC00288139810217130721F40E94ECED0E94A9
:10A3EC003540ACDA088119810E94E041002331F438
:10A3FC000EED1DE681DA0E941CEA05C000EA1DE69E
:10A40C0093DAA3DAAADA22968991089552DA12D055
:10A41C0091DCF1F796DC068B0E94A2B207E015E600
:10A42C0083DA20E010E006E167DC19F003D077DC7A
:10A43C00F1F798CA85EA90E085DC16E1089505D01D
:10A44C0011F400E0089501E0089542E551E00E9406
:10A45C003AF10F3F1F4F0895BA93AA93949804E1D1
:10A46C005DD060D001C0000061D0E9F700E410E0DD
:10A47C0063D067D069D060D00081118106FF05C020
:10A48C0055D0C9F7949A00E041C006E358D04AD0A1
:10A49C0001C000004BD0E9F757D04ED0008111819C
:10A4AC0007FD03C043D0C9F7EDCFCFDF59F302E16D
:10A4BC0046D003ED18E03ED002E041D000E03AD0A7
:10A4CC0004E03ED000E01DE235D006E038D007E0D5
:10A4DC0031D008E535D0E8EFFFE00181308138D08C
:10A4EC000AE53BD00381328133D00CE536D00581AF
:10A4FC0010E0348121D0008331830CE221D0ECE0D8
:10A50C001083118301E000931D10949AA991B991C5
:10A51C000895F89400ED17E025D008E311E0EAE087
:10A52C00F3E10FC0F89402E010E01CC00E944DEA69
:10A53C00012B0895ECE005C0ECE0F3E1089511E087
:10A54C00EAE0008311830895F89400ED17E00AC047
:10A55C00ACE0B3E10D933C930895AAE0B3E10D9305
:10A56C001C930895E7E2FEE0068317837894089520
:10A57C000E9477F42297D801C90126D02083318319
:10A58C00022F032B19F4949A00E01AC0C2DFD4DF17
:10A59C000081018100FD03C0C9DFC9F7F4CFE0E001
:10A5AC00F0E009C02D913D9128833983309300133D
:10A5BC00209301133296E817F907A0F3949A01E05F
:10A5CC002296E4E00C9488F4949800EC10E0E4E01B
:10A5DC00F3E100831183E6E008950E9473F423975E
:10A5EC00C80129013A01DB010EE0400E00E0501ECB
:10A5FC009E018B010E94EE3B002311F402E036C059
:10A60C0006E010E0FD01DC010E94A4F406E010E07D
:10A61C00E8EFFFE0DC0116960E94A4F4FC016486CE
:10A62C007586D2DF40825182042D052919F4949A43
:10A63C0000E01CC06EDF80DF0081018100FD03C0E3
:10A64C0075DFC9F7F4CFA0E0B0E00BC0FC010191BD
:10A65C001191CF0109831A831093001300930113F6
:10A66C001296A415B50590F3949A01E02396E8E0B0
:10A67C000C9484F49A938A932297202F949802E056
:10A68C0014E0EAE0F3E15DDFE0E031813983308111
:10A69C003883432F59814432524030F03FDF00E47D
:10A6AC0010E048DF949A44C080E69AE040E050E025
:10A6BC0003C002964E5F5F4F68817981461757073A
:10A6CC0000F5BA016C5F7B4FEAE0F3E160837183C4
:10A6DC00E0E03081FC013183E0E0F3E13181FC0109
:10A6EC0030834C3030E0530721F7222311F33091A3
:10A6FC0018103323F1F66081718160307840C9F60F
:10A70C00CDCF949A8B010E50104008831983E0E64C
:10A71C00FAE044855585463008E0584071F40E94B3
:10A72C003E3C002329F02AE230E000E61AE020DF6C
:10A73C0000E0229689919991089544855585403081
:10A74C005007B1F708810E94227C023089F701E0A2
:10A75C00F0CFBA93AA939A938A93FA93EA933A9284
:10A76C002A921A920A927A936A935A934A933A9338
:10A77C002A931A930A93AFB7BBB700E00BBF22978B
:10A78C00A8950091F40F002309F06BC0109165009F
:10A79C0014FF67C001E000931D1000931E109498E5
:10A7AC0004E179D00081118106FF07C000E000931D
:10A7BC001D1000931E10949A54C004E370D00081B5
:10A7CC00118107FD02C000E0F4CF0CE268D00081DB
:10A7DC00018102FF04C000E363D00081118108E213
:10A7EC005ED08081918192FF06C020E030E000E0D5
:10A7FC0010E00E94BE5291FF0CC04CD08081918120
:10A80C00009120100F3F29F0E0E2F0E10081039568
:10A81C00008397FF0CC03ED00081118100911F1066
:10A82C000F3F29F0EFE1F0E100810395008304E292
:10A83C0032D00081018100FF12C029D00091011398
:10A84C000983009100130883098100FF08C003FFEE
:10A85C0003C02AD00860008327D001600083949A3B
:10A86C00A8952296BBBFAFBF099119912991399137
:10A87C004991599169917991099019902990399040
:10A88C00E991F99189919991A991B991189500E063
:10A89C0014E00EC002E311E0EAE0F3E102C011E0C3
:10A8AC00EAE007D0ECE00895E4EFFFE000810895C2
:10A8BC00EAE0008311830895BA93AA93229700913A
:10A8CC00F40F002309F4EAC0EFDF0260008300817B
:10A8DC0003FF02C001E001C000E01081167F10836D
:10A8EC000E944053002309F4D6C0A2E0B0E10091CD
:10A8FC00F50F005039F0025009F485C00A9509F49F
:10A90C00AEC0C6C00C91053041F406E0D3D0F1D0F6
:10A91C00E0D0E3D00E94F2ECBEC00C91023031F4D6
:10A92C00D8D0008511850330104010F405E1EECF2E
:10A93C000285002311F402E001C003E00093E50C52
:10A94C00378147EE5CE020918B0A0CE81AE00E94FC
:10A95C00D6E410E0BED0008711870093E60C0E5FA2
:10A96C001F4F008711870781002329F450E06BEB00
:10A97C007CE04085A6D0ADD00285002309F48BC0C5
:10A98C0001811281ADD001831283A3D00381148184
:10A99C00A7D0038314839DD0A0D0A2D005831683A7
:10A9AC0098D0008511859CD00087118794980EC093
:10A9BC0002E0AAE0B3E10D931C930181008102E057
:10A9CC0011E076DF00E410E0ECE073DF04E263DF1B
:10A9DC00008111810883198310FF08C058DFE0E063
:10A9EC00018109830081018100FDE2CF949A02E08C
:10A9FC000093F50FF89400ED17E0E7E2FEE0068314
:10AA0C001783789448C04ED079F460D06AD061F442
:10AA1C0063D05FD069D041F40C910630C9F105E1E7
:10AA2C0049D04FD003E035C00BE000938A0A58D0D0
:10AA3C0001811281E0E6FAE003A714A751D003814B
:10AA4C001481E0E6FAE005A716A746D0E0E6FAE0A6
:10AA5C0007A710AB50E060E67AE047E058CF22D071
:10AA6C0019F734D03ED001F737D033D03DD0E1F6D2
:10AA7C000C910530A1F651E06BEB7CE031D04085B8
:10AA8C002DE030E12F5F3F4F28D00E94F2ECAFCF8A
:10AA9C0000E00093F50F08DF0D7F00832296A9914B
:10AAAC00B99108952BD001811281E2E0F0E121816E
:10AABC0032811CC000938A0A50E060E67AE041E0E3
:10AACC00089517D0058116810C94F2EC17D00381F0
:10AADC001481E2E0F0E1089511D00581168108950A
:10AAEC000DC02381348102C02581368102171307E2
:10AAFC00089522E030E12F5F3F4F0895EDE0F0E143
:10AB0C00089513D008ED1DE525D001C028D029D01B
:10AB1C00F1F32DD011F401E008952DD021F0009126
:10AB2C005E0E063099F700E0089529D02BD00C94D6
:10AB3C005FB228D00E945FB228D020E00E94B4F40B
:10AB4C000E94FEB225D00C941CEA1CD00E945FB26D
:10AB5C000EE218E520E00C94B4F40E94FEB218C08A
:10AB6C0022960E94FEB20E946EB7002308950091B7
:10AB7C005E0E0130089500915E0E0530089501E0DF
:10AB8C000C9441B211E000E008950BEA16E508952B
:10AB9C00F89400ED17E0E7E2FEE00283138378946B
:10ABAC000895DDDF0C941CEA0E94B977BEDF05EF37
:10ABBC001DE6D0DF0E94FEB2F4CF35D00091C20F5B
:10ABCC00083020F000E040E551E031D00091C20F98
:10ABDC000A9569F00A9571F00A9579F00A9581F059
:10ABEC000A9589F00A9591F00A9599F015C007E538
:10ABFC0013E514C007E613E511C007E713E50EC013
:10AC0C0007E813E50BC007E913E508C007EA13E5ED
:10AC1C0005C007EB13E502C007E413E5E6E9FFE026
:10AC2C000083118308950E9425B20CC00FD00E949E
:10AC3C0051F1BACF03D00091640E0895E4E9FFE01E
:10AC4C000083118301E00093990F089549E451E0CA
:10AC5C000895E9DF0091840E002319F007E611E551
:10AC6C00DDCF07E511E5DACFDEDF07E911E5D6CF59
:10AC7C00DADF07D019F007E712E5D0CF07E812E5C5
:10AC8C00CDCF0091650E00230895CDDF0091810E8C
:10AC9C00023020F000E045E451E0C9DF0091810E64
:10ACAC00002319F007E01FE4B9CF07EF1EE4B6CF7D
:10ACBC00BADF00917E0E07D019F007E412E5AECF93
:10ACCC0007E312E5ABCF0071059505950595059544
:10ACDC000895A9DF07D019F007E212E59FCF07E12D
:10ACEC0012E59CCF00917E0E0670059508959BDFB2
:10ACFC00EEE7FEE0008100FF03C007EF11E58ECF09
:10AD0C0007E012E58BCF8FDF0091820E002319F044
:10AD1C0007E311E583CF07E411E580CF84DF0091D1
:10AD2C007E0E087005950595059519F007E111E55E
:10AD3C0075CF07E211E572CF76DF0091830E002309
:10AD4C0019F007E711E56ACF07E811E567CF07E1CE
:10AD5C001FE474DF0DD019F407EE1FE45FCF08D0A9
:10AD6C00013019F407EF1FE459CF07E010E556CF77
:10AD7C000091BE0F0370089507EB1CE45BDFA3DFAB
:10AD8C0019F007E91DE44ACF07E81DE447CF07EAAD
:10AD9C001CE450DF09D019F007ED1DE43FCF07EE9E
:10ADAC001DE43CCF0091640E007205958DCF07E831
:10ADBC001CE440DF0FD0013019F407EB1DE42ECF5B
:10ADCC0007D019F407EA1DE429CF07EC1DE426CFC0
:10ADDC000091640E0C7005950595089524DF07D03D
:10ADEC0019F007E01DE41ACF07E11DE417CF00911D
:10ADFC00640E02700595089516DF13D0112019F416
:10AE0C0007E21DE40BCF07D019F407E41DE406CFCD
:10AE1C0007E31DE403CF1091640E109F01E01016A0
:10AE2C0008951091640E04E0109F0895FCDE08D084
:10AE3C0000FF03C007E110E5F1CE07E210E5EECE0E
:10AE4C00EDEBFFE000810895EEDEFADF01FF03C0B9
:10AE5C0007E310E5E3CE07E410E5E0CEE4DEF0DF37
:10AE6C0002FF03C007E510E5D9CE07E610E5D6CE04
:10AE7C00DADEE6DF03FF03C007E710E5CFCE07E815
:10AE8C0010E5CCCED0DEDCDF04FF03C007E910E513
:10AE9C00C5CE07EA10E5C2CEC6DED2DF05FF03C081
:10AEAC0007EB10E5BBCE07EC10E5B8CEBCDEC8DF77
:10AEBC0006FF03C007ED10E5B1CE07EE10E5AECEF0
:10AECC00B2DEBEDF07FF03C007EF10E5A7CE07E039
:10AEDC0011E5A4CE033011F0043011F401E0089513
:10AEEC00003320F00A3310F401E0089500E00895D7
:10AEFC0012D0902F002369F0802F8A5F112309F064
:10AF0C008A95933008F0839509D0953011F48D5FB4
:10AF1C0005D008C090E09A938A930895182F01E009
:10AF2C000C9467B3899199910895002359F0102FCF
:10AF3C001A5F033008F01395053008F0139501E003
:10AF4C000E9467B3089524D0822F26D0805029F018
:10AF5C008A9539F08A9559F018C023D024D01296CE
:10AF6C000CC012960C91129726D01DD006C019D089
:10AF7C0012960C91129723D011960C9120D000EEC2
:10AF8C001BE5E8DD26960E94FEB2E4E00C9488F402
:10AF9C000E9477F4D8010895F2DD11E007E00C94DB
:10AFAC005FB20C9108C011960C91119708C00E94C9
:10AFBC005FB2FD01058110E002C03A932A931A9307
:10AFCC000A930895E5DFC901E7DF0C91002351F4E2
:10AFDC00FD010181002331F40281002319F499232E
:10AFEC0009F483E0805039F08A9589F08A95A9F0AC
:10AFFC008A95D1F01EC0FD010281DDDF0181DFDF0A
:10B00C000C91DDDF00EE1BE5A5DD269610C0C9DF37
:10B01C00FD010181D4DF0281F4CFFD010281CBDF80
:10B02C000C91CDDF0181EDCF0EEF1AE593DD0E947F
:10B03C00FEB2E4E00C9488F4ABDF922F832F9FDDFB
:10B04C00992311E0C1F006E0B2DF0481B8DF03817F
:10B05C000F71B5DF00ED1BE57DDD269611E00EE0EE
:10B06C000E945FB2882321F004E01CE573DD0DC063
:10B07C0008E01CE5FBCF07E09ADF0481A0DF038129
:10B08C009EDF00ED1BE566DD26960E94FEB2E4E035
:10B09C000C9488F40E9477F415D141F027D11AD181
:10B0AC0011F01DD121F40BD121D101C008D167DDE4
:10B0BC0080E0DE01139605C052DD1B811074082F51
:10B0CC0017DFF8D004FD07C0DCDD19F00E945FB477
:10B0DC0002C00E946254882309F408D13C9130725A
:10B0EC002B8120748E01A8DF08D159F3D7D039F009
:10B0FC00882329F43CDD19F000E00D8381E00091F8
:10B10C005E0E003308F458C000915E0E0A3308F04E
:10B11C0053C0EFD049F00A9521F10A9551F10A95E7
:10B12C0099F10A95C1F146C00B81102F1074109142
:10B13C005E0E59F0123300F60F7EC6D009F0BDCF6B
:10B14C000B81007F02600B83B8CF133308F0B4CFB0
:10B15C000F7CBAD009F0B1CF02DD0B81007F036008
:10B16C00F2CF9B81CBD00B83B5D009F0A6CF9B83BC
:10B17C00A4CF9C81192F98D0012B0C83ABD009F054
:10B18C009CCFEDDC9C8399CF9C81B8D00C83A2D052
:10B19C0009F093CFF6CF00915E0E003319F40B81BA
:10B1AC000F7DD1CF00915E0E013319F40B8100623B
:10B1BC00CACF82CF81E081CF00915E0E063021F4A0
:10B1CC0079D004FD2BC078CFD6DC21F473D004FFEA
:10B1DC0025C072CF00915E0E043051F40B8106FF36
:10B1EC0004C0853038F7839568CF8430E0F3E2CF24
:10B1FC0000915E0E033059F4823010F08A955DCFC9
:10B20C00882309F084E00B8106FF57CFECCFAFDC2D
:10B21C0061F4882319F05ED039F077D00E9481B3A5
:10B22C002696E4E00C9488F447CF00915E0E01342E
:10B23C00A1F000915E0E013681F000915E0E003C93
:10B24C0061F000915E0E003E41F000915E0E003800
:10B25C0021F000915E0E0D3A21F4853009F49FCF58
:10B26C002BCF00915E0E0035A9F000915E0E0037D9
:10B27C0089F000915E0E0F3C69F000915E0E0F3E5E
:10B28C0049F000915E0E0F3829F000915E0E0C3BD8
:10B29C0009F012CF853009F489CF0ECF00915E0EE4
:10B2AC0019DE002308951A811F7000915E0E02951D
:10B2BC00007F0895E0E5FEE000810181089597DDAF
:10B2CC000C947E45269724C010915E0E1295107F2B
:10B2DC00102B1B838E010E94C846002308958E01FB
:10B2EC000E947F46002308950E947E458E010C9497
:10B2FC001546082F0A950895249635CC192F0CD095
:10B30C00012B08958E010E940A478E010C9447462A
:10B31C000E94744500230895107F00915E0E005327
:10B32C0008958A93CFDF41F0E1DFD4DF11F0D7DF4E
:10B33C0021F4C5DFDBDF01C0C2DF21DC80E003C00C
:10B34C000EDC082FF2DDB6DF04FD07C09ADC19F025
:10B35C000E945FB402C00E946254882309F4C6DFC5
:10B36C0060DD212D8E01EFDDC8DF69F397DF39F049
:10B37C00882329F4FCDB11F081E001C080E000910E
:10B38C005E0E003308F448C000915E0E0A3308F0DC
:10B39C0043C047DD112019F5ACDF59F00A9569F06F
:10B3AC000A9569F00A9581F00A9581F00A9599F051
:10B3BC0014C079DF012B0A83C4CF5DD0FBCF198178
:10B3CC0073DF012B0983BDCF58D0FBCF18816CDF05
:10B3DC00012B0883B6CF53D0FBCF81E0B2CF1BDD5E
:10B3EC00082F69F40A9591F30A95A9F30A9539F394
:10B3FC000A9551F30A95E9F20A95F9F2EECF0A95FE
:10B40C00F1F20A9509F30A95A1F20A95B1F20A959F
:10B41C00E9F20A9501F3E1CF00915E0E033029F4B5
:10B42C00823008F48ECF8A958CCF00915E0E04305A
:10B43C0021F4863090F6839584CF00915E0E063011
:10B44C0021F438DF04FD11C07BCF95DB21F432DF12
:10B45C0004FF0BC075CF8BDB09F072CF882329F06A
:10B46C003EDF41F08E010E945A460E9481B326961F
:10B47C008991089565CF1A814FCF19814DCF1881CD
:10B48C004BCF0E9477F42397D80179DB80E00C91A5
:10B49C000883FD010181098302810A838E010E94C8
:10B4AC00174903C05CDB082F40DD382FBADC212D97
:10B4BC008E0188DD22DFC9F3F1DE39F0882329F40F
:10B4CC0056DB11F081E001C080E000915E0E00338C
:10B4DC0008F448C000915E0E0A3308F043C0A1DCAA
:10B4EC00112019F506DF59F00A9571F00A9571F0E3
:10B4FC000A9589F00A9589F00A9599F014C018817B
:10B50C00D3DE012B0883CFCFBADFFBCF1981CCDE82
:10B51C00012B0983C8CFB1DFFBCFC5DE012B0A831A
:10B52C00C2CFA9DFFBCF81E0BECF75DC082F69F459
:10B53C000A9599F30A95A9F30A9541F30A9559F3DB
:10B54C000A95E9F20A9501F3EECF0A95F9F20A95FC
:10B55C0011F30A95A1F20A95B9F20A95F1F20A953E
:10B56C0001F3E1CF00915E0E033029F4823008F430
:10B57C009ACF8A9598CF00915E0E043021F48630D4
:10B58C0090F6839590CF00915E0E063041F40E94A8
:10B59C0081B30CE310E02396E4E00C9488F4009162
:10B5AC005E0E073021F40E9481B30DE3F3CFE3DA92
:10B5BC0021F000915E0E023011F419D074CFD7DA5D
:10B5CC0009F070CF8E010E9425498E010E94EF4830
:10B5DC00002359F008810C930981FD0101830A8134
:10B5EC0002830E9481B300E0D5CF01D05BCF00E095
:10B5FC00088309830A8380E00C9481B313D019F477
:10B60C000CD0C3DAD6CA12D00F73006401D089CE25
:10B61C0010D00E9451F10C94B97711E000E00C9419
:10B62C005FB226970E9466450023089502D00C94C1
:10B63C0037F143EC50E00895F5DF09F4E1CFF6DF84
:10B64C000F730068E3CFEEDF09F4DACFEFDF0F738F
:10B65C00DDCFE7DF11F46DDA16C05ADE69F046DE95
:10B66C0039DE11F03CDE11F401E03EDE0B8106FF09
:10B67C0006C020E047DE03C001E00E947E45D6DF15
:10B68C000260C6DF07DD26960895CBDF11F451DA90
:10B69C0017C03EDE71F02ADE1DDE11F020DE19F43B
:10B6AC005EDA00E021DE0B8106FD06C021E02ADE19
:10B6BC0003C000E00E947E45B9DF0D7FA9DFEADC04
:10B6CC002696089501C04BDA12D00BEA11E642DA45
:10B6DC00A4DF00E870DC0DEE15E63CDA41DAA1F3EC
:10B6EC0046DA21F000915E0E063069F7089510E0FD
:10B6FC0095CF01C034DAFBDF01EC11E62BDA8DDFDC
:10B70C0001E859DC0DEE15E625DA2ADAA1F32FDA79
:10B71C0021F000915E0E063069F70895002329F0A0
:10B72C0027D030D011F400E0089522D02BD010F4A3
:10B73C0000E008952DD019F0025061F011C0ECE436
:10B74C0019D041EF53E264E779E40E94EEF370F014
:10B75C0000E00895ECE40ED01FD040F000E0089516
:10B76C00ECE408D019D010F000E0089501E0089541
:10B77C00ECE4FEE017C00E945BF240E050E068ECA5
:10B78C0072E4089540E050E060E070E00C94EEF359
:10B79C0000917D0E0050089547EF5FE36CE176E475
:10B7AC000C94EEF3008111812281338108950E9463
:10B7BC0073F4269700E0B3D0F0F300E0AFDF002382
:10B7CC0021F400E0D8D0D3D0EFD9E2DF19F0025049
:10B7DC0019F002C0CDDF04C0CBDFCFDF0E9422F313
:10B7EC000E945DF2C801D901BA93AA9394DB4EE58D
:10B7FC005BE560E08E010C5F1F4F0E9407F52496FD
:10B80C0059DD04FF04C073DF07ED11E6A3D9B7D9E6
:10B81C0003C0A5D90E94FEB24DDD04FD0EC031DA85
:10B82C0019F00E945FB402C00E946254F6DE0AE86E
:10B83C001DE590D911E000E102C011E007E00E9483
:10B84C005FB28C019D0197DF0E9480F328013901C2
:10B85C009FDF19F0025049F008C00E9423B4BA933C
:10B86C00AA9359DB0BE31BE506C07A926A925A92B3
:10B87C004A9206E71BE56ED93FDD61F200915E0E40
:10B88C00003348F000915E0E0A3328F45ED04FD09E
:10B89C00C801D901BFCF00915E0E093119F45DD0FA
:10B8AC000B83F5CF00915E0E023011F45BD0F8CF14
:10B8BC0000915E0E063021F4FDDC04FD17C0A9CF0B
:10B8CC005AD921F4F7DC04FF11C0A3CF50D909F0E9
:10B8DC00A0CF5EDF19F0025031F005C08C019D0144
:10B8EC000E945BF202C08201930141D00E94B977A1
:10B8FC002696E8E00C9484F40E945FB28C013CD054
:10B90C000E945BF240E050E06AE774E40E9480F32E
:10B91C003A932A931A930A930DE014E5089520E0C4
:10B92C00FE01E00FF21F20830395063008950C836F
:10B93C0000E00D834AE050E01FD08E010C9427F5F7
:10B94C001AD04AED56E00C945CF119D00B810A83A5
:10B95C000C810B8300915E0E089516D00C810A8326
:10B96C0000E3089500E3088309830A83089546ECF5
:10B97C0050E00C945CF110E020E030E00895098177
:10B98C0008830A81098308950A8108830B8109833E
:10B99C0008950E9477F426971BDA023029F03DDED9
:10B9AC0007EC1DE6CAD83CCC00E0B9DFF0F382DC32
:10B9BC0004FF04C09CDE0DE212E6CCD8E0D8E2E530
:10B9CC00FEE075D0012B81F0A2E5BEE0ED91FC917B
:10B9DC00B89734F0E2E5FEE079D029393A4324F007
:10B9EC0000E010E074D0E0D8E2E5FEE080819181C7
:10B9FC0092DA4CE25BE560D003C0B1D80E94FEB293
:10BA0C0059DC04FD0EC03DD919F00E945FB402C090
:10BA1C000E94625402DE04E91DE59CD811E000E1AD
:10BA2C0002C011E008E068DF95D866DC39F30091BC
:10BA3C005E0E003340F000915E0E0A3320F485DF79
:10BA4C0076DFC801DBCF00915E0E093119F485DF7A
:10BA5C000B83F6CF00915E0E023011F483DFF8CF2A
:10BA6C0000915E0E063021F425DC04FD17C0C5CF15
:10BA7C0082D821F41FDC04FF11C0BFCF78D809F0A5
:10BA8C00BCCF082F092B41F0883200E0900760F002
:10BA9C0089390AE3900740F48C0119D00E94B977D8
:10BAAC0002E000937A0EBCCBA8CFE3E8FFE0008164
:10BABC001181089547E15BE560E08E010E5F1F4F39
:10BACC000E9407F522960895E3E7FEE006C04AE4DB
:10BADC0051E00C9455F1E3E7FEE0208131810895AB
:10BAEC0077D9033028F0A2DD037F0460A2DD9FD854
:10BAFC006FD9005029F00A9589F00A95E9F025C014
:10BB0C002FD019F11DE4273B3107D9F01DE4273C58
:10BB1C00310769F48BDD037F086016C021D019F45E
:10BB2C0085DD037F11C01DE4273B310771F01DE457
:10BB3C00273C310719F4EECF13D091F3273B3D444A
:10BB4C0021F474DD037F046010D00E94B97701E00A
:10BB5C000093980FB9DF273C3D4409F41ADF089590
:10BB6C00BADF1DE4273A3107089563DD0C9451F1D7
:10BB7C0019D9AADF31F0273D3D4449F057DD0F7D3F
:10BB8C0005C0273E3D4419F051DD0062EEDF01E0B7
:10BB9C000093980F0C94B9770091640E94D894DFAD
:10BBAC0031F027393D4449F041DD0F7E05C027387F
:10BBBC003D4419F03BDD0061D8DFE9CF8A93009159
:10BBCC00BB0F0D3010F005E005C00091BB0F0D3020
:10BBDC0020F001E043E451E02AD88091BB0F04C06F
:10BBEC000E94B5550E94FEB282DD08E012E60E946A
:10BBFC00B05513DD082FE0E1F0E70C9418F401E4E4
:10BC0C0017E623C002E517E620C003E617E61DC0C1
:10BC1C0004E717E61AC005E817E617C00CE917E6A3
:10BC2C0014C003EB17E611C008EC17E60EC00DEDBF
:10BC3C0017E60BC002EF17E608C007E018E605C0D0
:10BC4C0008E118E602C009E218E60E94B05526D0B9
:10BC5C0054DB41F200915E0E043029F483958D3053
:10BC6C0008F280E0BFCF00915E0E033031F48823E0
:10BC7C0011F08A95B7CF8CE0B5CF00915E0E0630EF
:10BC8C0049F00E94BD5509F0ABCF082F43E451E0B9
:10BC9C000E9451F10E94B977899108952CE310E02C
:10BCAC0001E00E9415B42EE315E101E00C9415B4EB
:10BCBC008A930091BE0F06950695083028F05AD04D
:10BCCC0003700C610E941C568091BE0F8695869560
:10BCDC0004C00E94B5550E94FEB209DD09EA12E6C5
:10BCEC000E94B0559ADC082FE0E3F0E70C9418F4AE
:10BCFC000AE318E614C00DE418E611C002E618E6D3
:10BD0C000EC007E718E60BC00CE818E608C001EAFD
:10BD1C0018E605C006EB18E602C00BEC18E60E940C
:10BD2C00B055BCDFEADAB9F200915E0E043029F4AA
:10BD3C008395883080F280E0CECF00915E0E033088
:10BD4C0031F4882311F08A95C6CF87E0C4CF0091D7
:10BD5C005E0E063071F00E94BD5509F0BACF0AD0C4
:10BD6C000370880F880F802B082F0E942C560E947E
:10BD7C0051F190CF0E942C560C9437F10E94BE5674
:10BD8C00033028F0F7DF0C7F02600E941C560E94E3
:10BD9C00BE56005029F00A9589F00A95E9F0F7CEC5
:10BDAC0028D031F11FE4273F3107D9F010E52730B7
:10BDBC00310769F4DFDF0C7F026016C01AD019F46A
:10BDCC00D9DF0C7F11C01FE4273F310789F010E544
:10BDDC002730310719F4EECF0CD091F3273F3F44B5
:10BDEC0039F4C8DF0C7F01600E942C560E9451F17F
:10BDFC00CECE71DE1FE4273E31070895EEE7FEE05C
:10BE0C0013D000FF06C0273F314559F00FD00E7FED
:10BE1C0005C02730324529F009D001600AD00E94B4
:10BE2C0051F1B5CEEDEBFFE0008155CE02D00C9474
:10BE3C0037F14AEC50E008950E947856023028F011
:10BE4C00F5DF097FF6DF0E941D560E9478560050E0
:10BE5C0019F00A9569F09BCE37DE12E527313107D0
:10BE6C0081F02732324521F4E1DF097F026006C000
:10BE7C002BDE2731324529F4D9DF097FDADF0E9426
:10BE8C0051F185CE8A930091BF0F0770073030F0C7
:10BE9C0066D002604DE451E00E941D568091BF0FA8
:10BEAC0087700E94A2B20BE514E60E94B05507C041
:10BEBC0002EC16E60E94B055F1DE0E94FEB21DDACD
:10BECC0051F100915E0E033031F4882311F08A9504
:10BEDC0022C086E020C000915E0E043031F4863022
:10BEEC0010F4839518C080E016C00E94BD5569F40B
:10BEFC00873078F434D0082B4DE451E08ADB10E025
:10BF0C00082F0E94B1798991089500915E0E063038
:10BF1C00D1F30E94B55581DB082F005071F00A95C2
:10BF2C0079F00A9581F00A9589F00A9591F00A95B5
:10BF3C0099F00A9509F4BCCFBFCF0CE516E6BACF41
:10BF4C000DE616E6B7CF0EE716E6B4CF0FE816E609
:10BF5C00B1CF00EA16E6AECF01EB16E6ABCF4DE45F
:10BF6C0051E00E9437F1007F08950E94A2B201E8CF
:10BF7C0014E60E94B0550AC00E94B5554EDB04ED84
:10BF8C0016E60E94B0558ADE0E94FEB2B6D9B1F315
:10BF9C0000915E0E033091F300915E0E043071F34C
:10BFAC000E94BD5521F000915E0E063029F70895D0
:10BFBC0039DF00FF06C02731304549F009D00E7F2C
:10BFCC0005C02732304519F003D0016005D0DFCD14
:10BFDC0048E451E00C9437F148E451E00C9451F1F1
:10BFEC0021DF01FF06C02733304549F0F1DF0D7F1B
:10BFFC0005C02734304519F0EBDF0260EDDFC7CD0B
:10C00C0011DF02FF06C02735304549F0E1DF0B7F19
:10C01C0005C02736304519F0DBDF0460DDDFB7CD16
:10C02C0001DF03FF06C02737304549F0D1DF077F1A
:10C03C0005C02738304519F0CBDF0860CDDFA7CD20
:10C04C00F1DE04FF06C02739304549F0C1DF0F7E11
:10C05C0005C0273A304519F0BBDF0061BDDF97CD35
:10C06C00E1DE05FF06C0273B304549F0B1DF0F7D0F
:10C07C0005C0273C304519F0ABDF0062ADDF87CD42
:10C08C00D1DE06FF06C0273D304549F0A1DF0F7B0E
:10C09C0005C0273E304519F09BDF00649DDF77CD4E
:10C0AC00C1DE07FF06C0273F304549F091DF0F770F
:10C0BC0005C02730314519F08BDF00688DDF67CD67
:10C0CC0001E047E451E00E9451F162CD00E047E409
:10C0DC0051E00E9451F101E05BCDA8DE0860A9DEC1
:10C0EC00F8CFA4DE077FFBCF01E046E451E0EBCFB5
:10C0FC0000E046E451E0EDCF99DE0F7EF0CF96DE06
:10C10C000061EDCF0E94915790E06FD033DB03308C
:10C11C0010402040304048F000E012DC91E00E94DA
:10C12C00DA5563D027DB0E9406775FD080811181BE
:10C13C002281338102C00E94B555D9DA05EB13E692
:10C14C000E94B0556ADA082F005029F00A9541F088
:10C15C000A9549F00BC006E219E60E94B05507C0DB
:10C16C000DE319E6FACF04E519E6F7CF80E096DD8A
:10C17C000E94B75511F30E94BD55C1F436D038D08A
:10C18C00481750406040704071F037D051F0082F84
:10C19C00D7DB0E94B97729D0EDDA0E94067772D0EE
:10C1AC00DAD20C9498579923E1F3F9CF0E94C15538
:10C1BC0021F000915E0E063019F4992391F3EFCF24
:10C1CC0000915E0E033031F4882311F08A95B5CFBF
:10C1DC0082E0B3CF00915E0E043009F0ACCF823018
:10C1EC0010F48395AACF80E0A8CFE3ECFFE008958C
:10C1FC00408151816281738108950E94875500238B
:10C20C00089538D000E00E945FB20FE510E60E945E
:10C21C00B055F3DFF9F00E949B5502E814E50E943B
:10C22C00B05523D00E94C5780E94475631F0E1E703
:10C23C00FEE03DDC0068118300830E94B9770E9408
:10C24C0081B30E949B5500EA1DE60E94B05503D0B5
:10C25C000E94DAE908950E94FEB2F89400EA1FE009
:10C26C000ED004831583789408950E94FEB219E0D1
:10C27C000C94955700E00E9441B210E00895E7E25B
:10C28C00FEE00895F7DF00E00E945FB20FEA15E6CA
:10C29C000E94B055B2DF11F10E949B5502E814E5E3
:10C2AC000E94B055E2DF01DC012B21F00E94ECED85
:10C2BC000E943540B2D90E942B77002349F00E948E
:10C2CC0081B300EA1DE60E94B055C5DF0C94DAE993
:10C2DC000E9481B300EB1DE60E94A35508950E94B5
:10C2EC009157269700E01BDBF0F30E94C55580E0C8
:10C2FC0090E000E00E94E1574CE25BE5DDDB04C01E
:10C30C000E94B5550E94FEB20E94605904FD08C0FF
:10C31C000E94475619F00E945FB402C00E946254FA
:10C32C007CD902EA1DE50E94B05511E000E1E4DA87
:10C33C000E94B0550E94825929F300915E0E003381
:10C34C0040F000915E0E0A3320F4FFDAF0DAC801F7
:10C35C00D9CF00915E0E093119F4FFDA0B83F6CFB9
:10C36C0000915E0E023011F4FDDAF8CF0E94C15537
:10C37C0069F00E94BD5521F68C010E9415EE002338
:10C38C0029F44BD900E819E50E94A35526960E9482
:10C39C00985708958A9300917D0E033020F40091F4
:10C3AC007D0E013029F402E045EC50E00E941D5650
:10C3BC0080917D0E04C00E94B5550E94FEB297D9A3
:10C3CC0005EA10E60E94B05528D9082F005019F044
:10C3DC00025021F007C002EB1DE502C001EC1DE587
:10C3EC000E94B0555BDC0E94835939F300915E0EBC
:10C3FC00043021F000915E0E033031F4882311F4E7
:10C40C0082E0DBCF80E0D9CF00915E0E063019F1CF
:10C41C000E94BD5581F621D00817D9F0082F005085
:10C42C0019F0025049F010C018D0023069F4A0D9AC
:10C43C00A4D90E9422F307C010D0002329F498D964
:10C44C009CD90E9480F393DA082F45EC50E00E94AF
:10C45C0051F10E94B9778991089545EC50E00C9404
:10C46C0037F18A930091B70F023028F001E041E5D3
:10C47C0051E00E941D568091B70F04C00E94B55523
:10C48C000E94FEB234D90AEB10E60E94B055C5D812
:10C49C00082F005019F00A9521F007C000E217E6AA
:10C4AC0002C001E317E60E94B055F8DB0E948359E5
:10C4BC0039F300915E0E043021F000915E0E0330D2
:10C4CC0019F401E08027DCCF00915E0E063039F0C4
:10C4DC000E94BD5599F6082F41E551E09AD88991F3
:10C4EC00089500E045E451E0F4CD01E045E451E06D
:10C4FC00EACD0E9491570E9446990023C1F576D04F
:10C50C00B1F18BD80E947F5959F00A9571F00A95B8
:10C51C0079F00A9581F00A9589F00A9579F011C0A5
:10C52C0009ED16E50E94B0551CC007EE16E5FACFD2
:10C53C000EEF16E5F7CF05E117E5F4CF09E217E5A5
:10C54C00F1CF843638F0883728F40E9490570BE0EE
:10C55C0018E504C00E94905702E218E50E94B055FD
:10C56C0022960E94B3550E941CEA0C94985700E046
:10C57C0000937B0E01DA01E00E940AAC3AD069F11B
:10C58C00893059F10E94135B082FE6E4F0E70C9414
:10C59C0018F40E94CB55C6CF0FE317E5C3CF06E5C1
:10C5AC0017E5C0CF0DE617E5BDCF04E817E5BACF08
:10C5BC000BE917E5B7CF02EB17E5B4CF08EC17E59D
:10C5CC00B1CF0FED17E5AECF06EF17E5ABCF843645
:10C5DC0008F2883708F4B9CFBDCF893029F40E940E
:10C5EC00AB5539DE0E94DAE90C94985701E00E94B1
:10C5FC0097AB802F002308950E949157229700E05B
:10C60C00088309830E94A2B206EE16E60E94B0557A
:10C61C000E94135B02EF18E60E94B0550E94FEB216
:10C62C0002C00E94B55520E012E005E00E940768A8
:10C63C0021E015E101E10E94366820E08E010E94A4
:10C64C003069802F0E946E688C3309F47DC008819C
:10C65C0019817DD031F30E9446990023C1F5C6DFC4
:10C66C00B1F10E94135B0E947F5959F00A9571F049
:10C67C000A9579F00A9581F00A9589F00A9579F076
:10C68C0011C009ED16E50E94B0551CC007EE16E569
:10C69C00FACF0EEF16E5F7CF05E117E5F4CF09E277
:10C6AC0017E5F1CF843638F0883728F40E9490577C
:10C6BC000BE018E504C00E94905702E218E50E94B6
:10C6CC00B05522960E94B3550E941CEA3DC000E072
:10C6DC0000937B0E288139810E940AAC8ADF69F1B4
:10C6EC00893059F10E94135B082FE4E7F0E70C94B2
:10C6FC0018F40E94CB55C7CF0FE317E5C4CF06E55E
:10C70C0017E5C1CF0DE617E5BECF04E817E5BBCFA3
:10C71C000BE917E5B8CF02EB17E5B5CF08EC17E539
:10C72C00B2CF0FED17E5AFCF06EF17E5ACCF8436E0
:10C73C0010F2883708F4BACFBECF893029F40E94A2
:10C74C00AB5589DD0E94DAE922960C9498570E9429
:10C75C008D3F002308950E94A2B20BE017E60E94C1
:10C76C00B0554BDDC1F00E949B5502E814E50E94C8
:10C77C00B0557BDD0E94135B0E947477002329F077
:10C78C000E949577002309F09ACD0E9481B30CE0AA
:10C79C001EE60E94A35508950E9491570E941CEA20
:10C7AC0025DF99F10E94135B0E947F5949F00A958D
:10C7BC0061F00A9569F0025071F00A9561F00EC0B3
:10C7CC0009ED16E50E94B05519C007EE16E5FACF33
:10C7DC000EEF16E5F7CF09E217E5F4CF843638F003
:10C7EC00883728F40E9490570BE018E504C00E948B
:10C7FC00905702E218E50E94B05522960E94B5555A
:10C80C000E94FEB20E941CEA09C0F89400ED17E0E9
:10C81C0036DD0483158378940E94DAE90E949857D8
:10C82C0008950E946FF42597882499244424552454
:10C83C0066247724B0E0BB24B394A0E020E0FE0192
:10C84C00EA0FF21F2083A395A530C0F32ED9202F19
:10C85C00212B19F04801C80108C0EEE6FFE040802A
:10C86C0051806280738081E090E0A0908D0F0E94D7
:10C87C00ECED7BD111F0A2E00FC07ED111F4A1E060
:10C88C000BC0A0E009C00E94915708EB18E50E946C
:10C89C00B05522960E94FEB20E94475619F00E9493
:10C8AC005FB402C00E9462540E941DED0E94835925
:10C8BC0009F4E4C00E947CEA002309F043D1009102
:10C8CC005E0E0A95C1F00A9509F48CC00A9509F41C
:10C8DC0056C00A9509F465C00A9569F00A9509F4E1
:10C8EC006DC00A9509F470C00A9509F49EC00151F7
:10C8FC0009F47DC09CC00E94BD55E1F5AA23D1F579
:10C90C000E940F410023E1F40E94135B05EC19E532
:10C91C000E94A35533D159F036D131F40E943540E1
:10C92C002596ECE00C9480F40E9417BCF9CFEEE64F
:10C93C00FFE04082518262827382A0928D0FF0CF11
:10C94C000E9417BC00918D0F002301E051F010E004
:10C95C00E5E8FFE000831183E2E6FEE0008102607F
:10C96C0006C00E9475EDE2E6FEE000810D7F0083BB
:10C97C00E9D0D6CF03D1D9F206D1B1F6CFCF8C0105
:10C98C0001501040E4DE61F0B0E00197EED011F000
:10C99C00A2E074C0F1D011F4A1E070C0A0E06EC0B0
:10C9AC006BC08C010F5F1F4FD2DE39F0B0E00196E7
:10C9BC00DCD071F7E1D091F7EFCF5EC0BB2311F063
:10C9CC00BA955CC0B2E05AC0BB2331F40091800E22
:10C9DC000230C1F7B1E052C0B13011F4B3954EC082
:10C9EC00B0E04CC080E090E00E943540D7CF0E9470
:10C9FC00915741E25BE50E94625D0E94CA5C00E3D4
:10CA0C000A830B8300E00C830E94A05CA9D051F038
:10CA1C00AED011F0A2E007C0AFD011F4A1E003C07A
:10CA2C00A0E001C0A3E0BB2429C0B6DE27C0009162
:10CA3C005E0E003308F100915E0E0A33E8F4BB2061
:10CA4C0021F000E30883098308C00E94915741E25A
:10CA5C005BE50E94625D82D00B810A8300915E0EC1
:10CA6C000B8300E00C830E94A05C7AD0D9F27FD0BB
:10CA7C0089F682D099F2D4CF0E94B5550E94A2B209
:10CA8C00E0E3FFE0B5DB403452446F4000E070401F
:10CA9C0090F00E94E1570E9491570DE715E50E9416
:10CAAC00B055249610E000E10E945FB20DE816E547
:10CABC000E94B0550BC00E94C05B0E94E3570E94BD
:10CACC0091570DE715E50E94B05526960E94135B11
:10CADC00AA2359F50091800E002309F4DBCEB13066
:10CAEC0039F401E51FE00E94E55709EE13E5CFCEBE
:10CAFC00B230C1F40FEB1EE60E94B05511E00CE011
:10CB0C000E945FB2EEE6FFE00E94C05B0E94C15B38
:10CB1C000E9480F30E94E3570CE114E50E94B0558B
:10CB2C002496B8CE04E31FE0DECFA13029F401EA4D
:10CB3C0018E50E94B055AECEA33009F0A4CE03E7A1
:10CB4C0018E5F7CFF894E0E4FEE00E94D85B97DBA1
:10CB5C00038B148B258B368B789408950C94C55CC1
:10CB6C00C8010E9435408C01F2CD0E9435408C01E9
:10CB7C000E94993F002308958C0106C00E94354005
:10CB8C00082D0929089584010E94BE3F00230895B1
:10CB9C000E946A5D12E52737310731F50E9447562E
:10CBAC0019F52BDBF1F1F89400E00AB900917D0046
:10CBBC000F7E00937D0000E100937C0000E0009369
:10CBCC008A000FEF61D010E00091BF0F07700E9438
:10CBDC00B17955DB00E05FD00093CC0F0093860E4B
:10CBEC000093C80F789408952738324509F04BC04C
:10CBFC000E94475609F447C00E942552002329F48D
:10CC0C000E949B5503E21EE60AC0F7DA51F00E941F
:10CC1C003252002361F40E949B550CED19E50E94E1
:10CC2C00A3550E9425B201E00093980F0895F89443
:10CC3C0000E00AB929D023DB2ED00093F40F009327
:10CC4C00F50F00931810E9E1F0E100830183EBE1AB
:10CC5C00F0E10083018300931F10009320100093D8
:10CC6C008B000093890000938800009387000AEFE3
:10CC7C00009386000DE000938A0000917D00006116
:10CC8C0000937D00789408954CE451E00E9451F19A
:10CC9C000093650E08950087018706830783089526
:10CCAC000E9473F4249790E020E0FE01E90FF21F3C
:10CCBC00208393959430C0F3E8EFFFE08781668082
:10CCCC00A185408490E0B0E001C0802F0E94A2B208
:10CCDC0002E914E60E94B05511E003E00E945FB235
:10CCEC0055245A924A920A2F0E94E15777247A923D
:10CCFC006A92082F0E94E5570DEE1AE50E94B05576
:10CD0C0028960E94FEB2092F005039F00A9571F056
:10CD1C000A95A1F00A95D9F024C0082F0E94E1577A
:10CD2C000E94605DBB23E9F015E018C07A926A920C
:10CD3C000E94605DBB23A9F019E010C00A2F0E946D
:10CD4C00E1570E94605DBB2361F01DE007C05A9261
:10CD5C004A920E94605DBB2321F011E101E00E9428
:10CD6C0067B30E94835909F4B1CFB1E00E94BD555D
:10CD7C0041F522E531E0182F00E09ED0AB010E9476
:10CD8C0055F19AD0AB010E943AF1600E711E94D00D
:10CD9C008301AB010E9455F11A2F00E088D00E944C
:10CDAC0055F185D00E943AF1400E511E285F3F4F3D
:10CDBC008201A90185D00E9481B32496E8E00C94ED
:10CDCC0084F400915E0E0630B1F30E94C15599F3C4
:10CDDC0000915E0E003318F100915E0E0A33F8F4E8
:10CDEC00BDDE00915E0E0A8300E00B830E94A05C06
:10CDFC000F3F104018F00E94B55500E0292F20502D
:10CE0C0009F463CF2A9529F02A9529F02A9529F05F
:10CE1C005DCF602E5BCFA02F59CF402E57CF009106
:10CE2C005E0E0931C9F40A81088300E30E94BA5CE2
:10CE3C0000E00B830E94A05C113018F00E94B555E5
:10CE4C0000E0292F205039F02A9519F32A9519F36F
:10CE5C002A9519F33BCF39CF00915E0E023091F435
:10CE6C00092F005039F00A9539F00A9539F00A95D6
:10CE7C0039F02CCF80E02ACF662428CFA0E026CF33
:10CE8C00442424CF00915E0E033029F4992309F435
:10CE9C001DCF9A951BCF00915E0E043029F4933070
:10CEAC0008F014CF939512CF0E94B5550FCFB9014E
:10CEBC00685F7F4FAB010895B9016A5F7F4F08959A
:10CECC000E9455F10C94B9770E9478F42697A0E053
:10CEDC0000E0FE01EA0FF01F0083A395A630C0F31B
:10CEEC00E6EFFFE080819181A0E00FC00E94AB5C77
:10CEFC000E949D5C0F3F4FEF14072040304020F004
:10CF0C000E94B55500E010E0C8010E94A2B203EAED
:10CF1C0014E60E94B05511E008E00E945FB20E9436
:10CF2C00915702E31BE50E94B05522960E94FEB277
:10CF3C000E94915747E25BE50E94625DAA2321F0B3
:10CF4C001CE001E00E9467B30E948359F1F2A1E05A
:10CF5C000E94BD5551F48C014CE551E0B1DF0E94AB
:10CF6C0081B32696E3E00C9489F400915E0E0630B2
:10CF7C00B1F30E94C15599F300915E0E003328F075
:10CF8C0000915E0E0A3308F4B1CF00915E0E0931A8
:10CF9C0081F40E94B35C0B830E949D5C003040E0E6
:10CFAC0014072140304020F00E94B55500E010E0FD
:10CFBC00ABCF00915E0E023019F480E090E0A5CF6B
:10CFCC000E94B555A2CF2FCE00E04EED56E081C8A1
:10CFDC0001E04EED56E077C800E040E551E079C83D
:10CFEC0001E040E551E00C94696002E0F6CF03E00B
:10CFFC00F4CF04E0F2CF05E0F0CF06E0EECF07E08F
:10D00C00ECCF302F002311F0333310F009E20895E8
:10D01C00143010F009E20895112351F0222341F04D
:10D02C0045EC50E00E9437F1031710F009E2089527
:10D03C00E4ECFEE000E040E0419303953017D8F7B4
:10D04C003093BE0E1093BF0E2093C00E4093600E13
:10D05C00112321F0032F0A950093600E00E0089530
:10D06C00392F282E602F012F161710F0063110F0D3
:10D07C000BE22BC02230E0F7402F50E0461B504013
:10D08C001091C00E11231091BF0E51F41123B1F069
:10D09C008091BE0E90E00197481759077CF4E8CFB9
:10D0AC00112331F00090BE0E11244015510504F3EC
:10D0BC000090C00E112404161506D4F66093C10E10
:10D0CC000093C20E2093C30E00E0822D932F08957F
:10D0DC0000E00093BE0E0093BF0E0093C00E0093B1
:10D0EC00600E0093C10E0093C20E0093C30E089500
:10D0FC003B2F6A2F0091C20E1091C10E011B03959C
:10D10C00212F1091C30E112309F02A5E1091600E8D
:10D11C00101720F0412F401B439501C040E0E4EC78
:10D12C00FEE050E0E40FF51FACE8BEE0A20FB51F27
:10D13C0010E005C020E22C93319611961395101730
:10D14C0068F42091C00E222329F0121719F42EE254
:10D15C002C93F3CF2081222369F3EDCFA62FB32F8D
:10D16C000895E4ECFEE000E003C010E01193039599
:10D17C0017D0D8F30091C10E1091C20E2091C30E9E
:10D18C00222359F00A5E1A5E08C040E2202F30E0DC
:10D19C00F901E457F14F408303951017B0F7089548
:10D1AC001091BE0E01170895202F30E02150304011
:10D1BC0004C000E32091600E30E0F90101C0F801D9
:10D1CC00EC53F14F08952AD011F00A9502C000914A
:10D1DC00BE0E20E004C010E220D01083239520174F
:10D1EC0040F4EADF10811033B1F317D01081103204
:10D1FC0091F314D011F40091BE0E0A95202F08C0A3
:10D20C00DBDF0081003219F400E307D000832395A3
:10D21C000091BE0E2017A0F30895CFCF0091C00E41
:10D22C00002308959A938A9320E009C0822F90E0FE
:10D23C000196FC01C5DF1081BFDF1083239510918F
:10D24C00600E211798F3212FB7DF0083BCDF899183
:10D25C00999108950E9476F4C801422ED80100914C
:10D26C00BF0E005041F00A9519F10A95E1F10A95AB
:10D27C0009F452C010C00C91002361F02D91009163
:10D28C00600EFED120831AD20081E7D106D298F726
:10D29C000CE2D8C1DBD10091BF0E002309F093DF63
:10D2AC0027DF0091BF0E002311F4ECD10AD270C01D
:10D2BC00FAD129F00A9559F00A9579F0E9CF0C9139
:10D2CC0010E004D24DE05BE504D22296E4CF0C9141
:10D2DC0010E0FCD142E15BE5F7CF0C9110E0F6D108
:10D2EC0047E15BE5F1CFDFD149F00A9549F00A95AA
:10D2FC0049F00A9549F00A9559F0CACF02D2E1CF0C
:10D30C0000D2E7CFFED1EBCFE0D14CE15BE5DCCF37
:10D31C00DCD147E25BE5D8CF0091BE0EE2EAF0E744
:10D32C000C9418F4C4D146E45BE5D3D12496B3CF66
:10D33C00BED14CE45BE5F9CFBAD142E55BE5F5CF64
:10D34C00B6D148E55BE5F1CFB2D14EE55BE5EDCF6B
:10D35C00AED144E65BE5E9CFAAD14AE65BE5E5CF81
:10D36C00A6D140E75BE5E1CFF894E7E2FEE000ED03
:10D37C0017E0028313837894F89400EA1FE0048387
:10D38C00158378940E94DAE90E9441B7002361F377
:10D39C000E94FEB20E946EB70023B1F300915E0EA4
:10D3AC000E3109F5DEDE52D10091BF0E002309F4D7
:10D3BC0020C179D10093600E00E004C020E260D15E
:10D3CC0020830395EDDED0F329DF11F00A9507C019
:10D3DC000091600E04C020E353D120830395E0DE5E
:10D3EC00D0F386DE06C10C3141F40091BF0E002350
:10D3FC0011F074D1CFCF2AD1F4CF0D3161F400915B
:10D40C00BF0E002311F0F5CF25D132D154F705DF33
:10D41C003FD1D1F7E6CF063019F469D10CE312C134
:10D42C000530D9F3073029F4442019F060D10DE30D
:10D43C0009C10230E9F50091BF0E00230091600E86
:10D44C0069F005C0B1DE20811BD120830A95002331
:10D45C00C9F700E20093C40EB6DEC3CF10E00F5F35
:10D46C001F4FADDE15D1B9F403D131F4D6DE10D196
:10D47C0019F0D3DE3083B5CF02D10AD131F4022FAB
:10D48C00222319F01BD10A95008300E02091600E35
:10D49C00C4DE0083A6CF0091600E05C00395F0D0CA
:10D4AC00108182DE1083ECD010811123B9F799CF53
:10D4BC00033069F40091BF0E002309F09ACF00915C
:10D4CC00600E002319F0FAD00A95E3CF91C0043016
:10D4DC0019F50091BF0E002309F08BCF15D12091C7
:10D4EC00600E30E00091BE0E10E051F405D13CF41A
:10D4FC0094DECED021F0E2D0022F0395CACF78C0B3
:10D50C00FBD04CF4BCD0C4D019F400E286DE00830E
:10D51C00D5D00081A2D065CF0130D9F497D0DC01F1
:10D52C000091BF0E005051F00A9509F47DC00A9588
:10D53C0009F47DC00A9509F47EC082C0AED008F40F
:10D54C007FC0012F9DD000810D93B8D0008185D074
:10D55C00F5CF0E3039F402E0EFE5FEE01081102734
:10D56C00108347C00B31B9F3093011F401E0F4CF4B
:10D57C00083019F40E94D2633CC01091600E2091C7
:10D58C00BE0E1217A8F51091BF0E112369F00033CF
:10D59C0020F00A3368F546DE24CF093149F500E363
:10D5AC0041DEA6DD00E3F7CF0931B9F402DE73D01A
:10D5BC0029F42091600E5FD00CF44CD099DDA4D0EE
:10D5CC00C1F40091600EECDDA0F4F3DD008320913A
:10D5DC00600E51D00CF43ED004CF003248F0EADD9E
:10D5EC005AD029F42091600E46D00CF433D0F9CEE9
:10D5FC0075D00E947DBB0E94FEB20091BF0E00232D
:10D60C0009F0C8CE2091C20E30E00091C10E201B53
:10D61C0030400091600E2017304024F41091C20E5F
:10D62C0050D0B8CE2FD0FCCF1BD00C9309C018D043
:10D63C000D931C9305C014D00D931D932D933C9307
:10D64C0056D000E010E0E5E00C9487F400E0009385
:10D65C00600E0895E0E6FEE0022F03950083089526
:10D66C004AE050E020E030E004EC1EE00C9427F59A
:10D67C002091600E30E00091BE0E10E03DC0022FF4
:10D68C0010E09DCD0091C10E1091600E100F089509
:10D69C00008100230895008337C00091BE0E1091C5
:10D6AC00600E011708950091BE0E0A9508950D9114
:10D6BC001D912D913C913A932A9308C0E0E6FEE02F
:10D6CC0008950091C30E0C9467B31BD01A930A9360
:10D6DC00089560E004EC1EE00C9407F5F89400ED5E
:10D6EC0017E0E7E2FEE002831383789408950E942A
:10D6FC0081B337DD0C94FEB2015010402017310776
:10D70C0008950D911C91089500918B0E002308959E
:10D71C00E2E6F4E01283018300E000830895E2E680
:10D72C00F4E01281011779F002830081002319F0D3
:10D73C000A95008308950181002329F00BE30083EF
:10D74C0001810A950183089500916204002331F44C
:10D75C0000916304002311F401E0089500E00895A2
:10D76C000E9478F44CD009E11CE64FD051D061F105
:10D77C00A0E052D002C0AA2331F454D058D009E50D
:10D78C001EE543D057D0AC010E9437F1102F0AE5AB
:10D79C00AC010E9451F1012FAC010E9451F14FD00C
:10D7AC0019F051D089F021D0A395A03208F0A0E057
:10D7BC000196903100F336D000EA1DE626D002C067
:10D7CC000E94FEB23CD0E1F3E3E00C9489F411E04A
:10D7DC0000E00E945FB2082F3AD002E218E520E088
:10D7EC000E94B4F422960E94FEB2F89400ED17E069
:10D7FC00E7E2FEE00283138378940895249710E007
:10D80C0012C02FD025D002ED1EE520E00C94B4F40C
:10D81C000E9487550023089580E090E0089501E070
:10D82C000E9441B211E000E00C945FB220D09A93B8
:10D83C008A93089522960C94FEB20E94FEB20E9426
:10D84C006EB70023089500915E0E0530089510E028
:10D85C001A930A930895E7E2FEE004831583789403
:10D86C00089509811A8148EE53E00C9495F1BA930E
:10D87C00AA9308950E9477F42297C1DF00E31CE677
:10D88C00C4DFC6DF81F180E0A8E0CCDF30D009E551
:10D89C001EE5BBDFCFDF9E012CD011F481E011C05F
:10D8AC001AE52CD0D9F39E012F5F3F4F22D0B1F354
:10D8BC0009810A3599F7188121D081F3A395A034F9
:10D8CC0020F3B0DF882339F0D2DF0AE31EE687DFCE
:10D8DC000E941CEA06C000EA1DE697DF02C00E9407
:10D8EC00FEB2ADDFE1F32296E4E00C9488F4B0E0F4
:10D8FC00BECF0A2F0E94F04A002308950A2F0E94DF
:10D90C00144B002308950E9473F478DF07E41CE69F
:10D91C007CDF12D1D9F05CD10023C1F0FBD0B1F087
:10D92C006EDF0DE81EE571DF7DDF04EA1EE56DDFBD
:10D93C000E94FEB207C038D109F4E5C084DF09F4B7
:10D94C00E2C053DF7CDFF1F333D1A9F758DF07E4F2
:10D95C001CE65BDF5DDF09F4D6C064DF03E61EE581
:10D96C0054DFA0E090E04424D5D081F05BDF06E7E3
:10D97C001EE54BDF25C067DF09F4C5C015D109F4DE
:10D98C00C2C033DF0E94FEB2AA2311F420E201C010
:10D99C0028E7BDD0B9F30CD149F30ED119F401E04D
:10D9AC00A027F0CF0DD139F7FACF4DDF09F4ABC07A
:10D9BC00FBD009F4A8C019DF0E94FEB2992311F420
:10D9CC0020E201C028E7A3D0B9F3F2D0B9F5AA231D
:10D9DC00A9F480E027DF0FE11EE517DF0E94FEB2FD
:10D9EC00C3D0843609F480E0C4D02491C8D095D03B
:10D9FC00C0F30AE544EA50E00E9451F113DF02E360
:10DA0C001EE503DFA9D0B0E0AFD0843609F480E086
:10DA1C008E010E9474B8602E992369F103DF77247C
:10DA2C007A926A920A811B812C813D81ACD006E4EA
:10DA3C001EE5EBDE26960E94FEB20AC0BDD019F49C
:10DA4C0001E09027B9CFBCD009F0AFCFF9CFCDDE34
:10DA5C00F6DEF1F3ADD079F0F6DE09F454C0A4D0C3
:10DA6C0009F451C0B1D099F790E0DCDE02E31EE579
:10DA7C00CCDE0E94FEB260D011F0AA2339F479D02A
:10DA8C000491601609F16CD0F9F421C07FD02A8181
:10DA9C003B81003F1F4F274040E0304050F4E7E40B
:10DAAC00F2E0E80FF41F0491601671F059D061F4A4
:10DABC000EC0E6E4FFE610E0EB0FF11F04916016D8
:10DACC0011F04ED021F0B39528D008F49ECFAADEE9
:10DADC00442079F000E000932B0F54D00EE41EE6A6
:10DAEC0094DE24962DD00E941CEA53D00E94DAE9D1
:10DAFC000AC00E94F27600EA1DE687DE25D00E945D
:10DB0C0048610E94B1632496E8E00C9484F411E01F
:10DB1C0048D095CE5DD00A35089583955DD00F5FC2
:10DB2C001F4F2F4F3F4F088319832A833B830030AD
:10DB3C00104028403040089500912B0F0023089589
:10DB4C000E94FEB24ED053C00E94FEB2F89400EA7E
:10DB5C001FE081DE0C94DAE90E94FEB280E00895A9
:10DB6C004424439499230895888389838A838B83DF
:10DB7C000895E7E4F2E010E0E80FF11F08958E013C
:10DB8C000C9446B829D03A932A9362CE0881198115
:10DB9C000895F89400EA1FE014960D931C93789462
:10DBAC00089501E00C9415B400915E0E06300895B2
:10DBBC0000915E0E0130089500915E0E03300895C1
:10DBCC0000915E0E0430089500915E0E07300895AA
:10DBDC0044EA50E00C9437F1088119812A813B8189
:10DBEC000895F894A7E2BEE000ED17E008951296B0
:10DBFC000D931C931397789408958A9380E001C039
:10DC0C00AFDDFDDD05E01BE600DE0CDE44D029F0C7
:10DC1C000A9539F00A9541F00AC004ED1BE6F5DDD2
:10DC2C0007C00BEE1BE6FBCF02E01CE6F8CF80E052
:10DC3C0029D039F3B9DF11F489910895B9DF11F0C6
:10DC4C00C3DF59F428D0E1F20A9519F00A9519F0BE
:10DC5C00D5CF10DED6CF57DED4CFAEDF31F488234C
:10DC6C0011F08A95CECF82E0CCCFAADF21F482309E
:10DC7C0028F68395C6CF12D019F40E94D263C1CF77
:10DC8C00B4DDBFCF2CE310E08CDF2EE315E189DF90
:10DC9C000E94FEB2D4CD082F0050089500915E0E64
:10DCAC00083008950E946FF400E00093930F02C0B7
:10DCBC000E94D26302E007B90FEC06B9F894009108
:10DCCC00930F0023A9F03398379800E00093930F3B
:10DCDC0007B1025029F0025029F00A9529F004C02E
:10DCEC0004E003C005E001C002E007B90FEC06B97F
:10DCFC0078940E94A2B20E94309A402E0E945B99A6
:10DD0C00C801D9010E942999A02E0E944699802E03
:10DD1C000E944299602E0E942F9988DDBB24BA92F2
:10DD2C00AA9286948694869499249A928A927724BD
:10DD3C007A926A9230D008E81BE567DD2C9672DD8A
:10DD4C000E944E9938010E948499C801D9010E9401
:10DD5C003B9922E830E03A932A9355245A924A92FE
:10DD6C007A926A9263DD17D005EA1BE54EDD2C969C
:10DD7C0064DD09F4A3CF1CDF21F016DF11F063DDA5
:10DD8C0029F433983798ECE00C9480F487DF09F48D
:10DD9C008FCF2BDD93CF10E05BCD0E9476F4442423
:10DDAC000E94A2B20AE41BE630DD3CDD01E61BE674
:10DDBC002CDD02C01BE00CD142DDD9F001DF11F0EB
:10DDCC00FBDE19F401E0402610C0EEDE11F03BDD65
:10DDDC0009F4F6C0EDDE19F44092810E11C05EDF3D
:10DDEC0019F40E94D26301C000DD1CDD01E61BE6C4
:10DDFC000CDD44202EE2F1F211E0DDCFFCD081F6F7
:10DE0C00FAD009F591E00E94A2B206EA1BE6FDDC0D
:10DE1C0009DD0DEB1BE6F9DC03C028E716E0D8D0D2
:10DE2C000EDD21F1CDDE11F0C7DE19F401E09027F3
:10DE3C0019C0BADE09F4B4CF06DD09F4B1CFB8DEEF
:10DE4C0059F49093830EC1D008E71BE6DEDCEADCC4
:10DE5C000FE81BE6DADC11C021DF19F40E94D26353
:10DE6C0001C0C3DCDFDC0DEB1BE6CFDC9923A9F68C
:10DE7C0020E2D4CF28E714E0ABD0E1DC19F1A0DE2E
:10DE8C0011F09ADE19F401E0802718C08DDE09F438
:10DE9C00B5CFD9DC09F4B2CF8BDE51F4982F0E94A8
:10DEAC00A2B209EA1AE6B1DC57DEA0E0B0E020C06D
:10DEBC00F5DE19F40E94D26301C097DCB3DC0FE8E5
:10DECC001BE6A3DC8823B1F620E2D5CF0A2F0B2B5F
:10DEDC0031F4A8DC05E117E598DC0E94FEB2F89459
:10DEEC0090D008EC10E086DCF89400EA1FE08CD0AF
:10DEFC00A6DC61F059DE11F0A6DC19F40E94B977AA
:10DF0C005FC056DE11F480E005C06FDC882311F091
:10DF1C00893071F770D041F40E943B99002321F0B5
:10DF2C000091830E002391F60E9446990023E1F4A0
:10DF3C0001E00E9497AB6FD049F0843021F047DCB0
:10DF4C000E941CEAD5CF47D007DED2CF54D061F463
:10DF5C000E943B99002341F00091830E002321F095
:10DF6C003AD00E94FEB2C4CF00E00E947DA253D0F2
:10DF7C0011F0893069F4119655DC79DC0BE515E567
:10DF8C0044DC58DCF89408EE13E03BD03DD003C0E1
:10DF9C001EDC0E941CEA992309F0AACF03C025DCE1
:10DFAC000E94FEB24CDCE1F34EDC21F0FDDD11F001
:10DFBC00FFDDA9F780E047DC19F0F6DD09F098CF1A
:10DFCC000E94B977E5E00C9487F480E00C94A2B23F
:10DFDC00E8DD0C94FEB201E00C9441B208DE0E9424
:10DFEC0039EAF89408EE13E014960D931C931597E8
:10DFFC0078940C940FEA0091810E00230895F89404
:10E00C0000E0E7E2FEE008950483158378940C9415
:10E01C00DAE90E9410EF802F002308950E9475F416
:10E02C00249780E0A0E000E010E09EDD0E945FB24B
:10E03C0000EC1AE6EADB0E941CEF03C080E00E94B1
:10E04C00FEB2F0DB823089F400E010E00883098333
:10E05C000A830B8305E70E9451EE002311F4A1E023
:10E06C0004C08E010E94FEEEA02FE9DBD9F09CDDEE
:10E07C0011F0E9DB31F40E9428EF2496E6E00C94D1
:10E08C0086F49ADD31F4882311F08A950BC082E076
:10E09C0009C096DD31F4823010F4839503C080E022
:10E0AC0001C0A3DB0091D30F002321F407ED1AE587
:10E0BC00ACDBC5CF90DFEFDD29F00A9591F00A9526
:10E0CC00C1F0BCCF0BEA402E02E0502E0091D40FD1
:10E0DC0010E047E150E00E9479F1400E511E8201A0
:10E0EC00E7CF07ED1FE058DE09EE13E58EDB229635
:10E0FC00A6CF48DDFCDB0CE413E087DB26969FCF34
:10E10C000E9477F46FD021F4F89470D0789402C008
:10E11C0000E00AB95ADF07ED1AE677DB83DB07E686
:10E12C001DE573DB12E086D00E94B17902C01D9A06
:10E13C008CB95E9B0DC05E9A11E004E10E945FB247
:10E14C0090E075DB0FEF1BE560DB229683951D9845
:10E15C005F9B0AC0ACB111E008E00E945FB2C7DB64
:10E16C000FEF1BE552DB229668DB19F321DDF9F288
:10E17C006ADB11F019DDE9F600E00AB933D051F58C
:10E18C0041D041F44CDB03E21EE63FDB2CDB0E946A
:10E19C001CEA23C00E943252002321F440DB0CED18
:10E1AC0019E5F3CF2CDF068307830093F40F00935C
:10E1BC00F50F00931810E9E1F0E100830183EBE126
:10E1CC00F0E10083018300931F10009320101ED0F8
:10E1DC00789403C005D00E94B179E4E00C9488F4E3
:10E1EC0010E028C00091650E0023089500917D0079
:10E1FC000F7E00937D0000E100937C0000E0009313
:10E20C008A0008950E9425520023089500938B00E4
:10E21C000093890000938800009387000AEF009315
:10E22C0086000DE000938A0000917D000061009350
:10E23C007D0008954DE451E00E9437F10770089578
:10E24C000E9477F42A97DBDA0EE31CE5DEDAE0DADB
:10E25C0009F410C171DC61F4E5DA08E31AE5D5DAEA
:10E26C006FDC97DC0E94DAE94EDB66DC21F402C13C
:10E27C0051DC09F448DBC6DF09F4B1D30E946645D2
:10E28C00CADE09F451C00E947445002339F443ECF2
:10E29C0050E00E9437F102700E947E45EFD01F4F74
:10E2AC000E94E645198505E033DAA9DA05E51CE597
:10E2BC00ACDA882389F0E2D01F4F0E94E64509852D
:10E2CC002EDAB0DA0091620466DD0091630464DD3D
:10E2DC000CE61CE59ADA2496B0DA49F069DCC9F050
:10E2EC00B2DA09F4C7C060DC09F4C4C07EDA2CDAF7
:10E2FC000023D9F276DC72DEF89408EC10E06EDEC6
:10E30C00F89408EC10E012960D931C9378940E94EC
:10E31C0039EA0E941CEF01E07CDE89F083DA81305F
:10E32C0059F407ED1AE5A0C07DDA0BEA16E56DDAB3
:10E33C005ADA0E941CEAB9CF03E61EE695C090E0BB
:10E34C0001C053DA8E010E942EEF65DE09F045C044
:10E35C000B81033008F060C00B81005029F00A9546
:10E36C00C1F00A95E9F023C04ADA04E81CE54DDA5D
:10E37C0010E00BE00E945FB274DA0EDD06EE13E5DE
:10E38C0044DA22960AE91CE540DA4CDA0DE814E589
:10E39C000DC035DA36DA229645DA00EB1CE506C0FC
:10E3AC002EDA2FDA22963EDA08EE1EE52EDA45DA60
:10E3BC0049F249DA31F40E9447EF2DDE71F491E015
:10E3CC000CC0F6DB09F0BDCF0B81002309F0B9CFEF
:10E3DC000E9450EF20DE09F4B5CF882389F005DACE
:10E3EC000EDA0CE41FE511DA1DDA90E020DA03E610
:10E3FC001FE50BDA22960E94FEB20E9439EA2BC06E
:10E40C00992351F0F2D9FBD900E21FE5FED90ADAC3
:10E41C0007E31FE5FAD9EFCF0B810330F89449F0ED
:10E42C00E5D9EDD90CE41FE5F0D9FCD906E71FE5D9
:10E43C00F1CFA7E2BEE008EE13E0D9DBAADBDFD90F
:10E44C000FEF1EE5E2D9EED904E11FE5DED90E94FB
:10E45C00FEB20E940FEA00E0DCDD51F0E3D981301E
:10E46C0009F46ACF0AE71EE6D0D9BDD90E941CEA8E
:10E47C000E9428EF2A96E4E00C9488F48E010C5F3D
:10E48C001F4F0E9415468E010C5F0895ABDEE9F01C
:10E49C00B9DE39F4C4D903E21EE6B7D9A4D90C9479
:10E4AC001CEA00E00AB90E943252002351F4B7D999
:10E4BC000CED19E5AAD997D90E941CEA91DE0C94AF
:10E4CC00B17900E0A3DE01C090D90E9462540E9491
:10E4DC00A2B20EEE1AE699D9A5D900911D1000230F
:10E4EC0059F000911F1057DC00911E1055DC0FEEF7
:10E4FC001DE58BD9249603C00CED19E586D99DD961
:10E50C0021F3A1D911F050DBF9F66CDE21F06EDEAF
:10E51C0067DE0E94B17908958A930E94A2B20CE141
:10E52C001BE673D90E94FEB280915F0EEFE5FEE010
:10E53C0000810E7F008300810460008384D07FD92A
:10E54C0009F474C080D06ED900915E0EE8EBF0E750
:10E55C000C9418F404E511E058D966C00AE511E0F2
:10E56C00FBCF01E611E0F8CF00E711E0F5CF00E8B2
:10E57C0011E0F2CF08E811E0EFCF07E911E0ECCFA2
:10E58C0005EA11E0E9CF0FEA11E0E6CF08EB11E064
:10E59C00E3CF02EC11E0E0CF0AEC11E0DDCF0FECA1
:10E5AC0011E0DACF06ED11E0D7CF0FED11E0D4CFAB
:10E5BC0003EE11E0D1CF09EE11E0CECF00EF11E068
:10E5CC00CBCF05EF11E0C8CF0AEF11E0C5CF0EEFAE
:10E5DC0011E0C2CF02E012E0BFCF0AE012E0BCCFE4
:10E5EC0006E112E0B9CF04E212E0B6CF08E212E085
:10E5FC00B3CF0FE312E0B0CF00915E0E003368F0A2
:10E60C0000915E0E0A3348F400915E0E10E0005348
:10E61C001040C2DB09EE1AE505C000915E0EBBDBB3
:10E62C000CE01CE5F2D822960E94FEB20E9446EA4B
:10E63C00012B09F084CFE3DC048305837894809369
:10E64C005F0E89910895F89400E117E204C9EFE593
:10E65C00FEE010811027108308950E9477F4CED825
:10E66C000EE51CE6D2D8D4D849F0B3990BC0BDD86E
:10E67C00C6D80EE81EE6C9D80E94FEB22496E4E085
:10E68C000C9488F4C9D8A0E0B0E088839983AA835D
:10E69C00AB8320E074DA0196883A01E6900798F390
:10E6AC0000E0A0937B0E11E00E945FB204EA14E537
:10E6BC00ACD80E94FEB2B0D8B399FECF0FE91FE0E0
:10E6CC0001501040E9F700C00000893803E19007C1
:10E6DC0098F788839983AA83BB8325EA50DA01963D
:10E6EC00EBCF0E9474F4249797D8442455246624C5
:10E6FC00488259826A826B828E010E9474B8053AF4
:10E70C0049F4019601E0400E561C08E8401603E15E
:10E71C00500668F374D805E71CE677D883D887D8F9
:10E72C000CE81CE672D8229688D8F1F32496E7E020
:10E73C000C9485F48A9380E001C08FDF60D803E3EA
:10E74C001BE663D86FD8A7DA19F00A9529F007C031
:10E75C000EE51CE65AD804C005E71CE6FBCF80E0AA
:10E76C0091DA61F321DA11F48991089521DA11F02B
:10E77C002BDA39F490DA09F30A9511F4B2DFDECF13
:10E78C00DACF1ADA11F01CDA19F401E08027D6CFAF
:10E79C002CD8D4CF8A9380E001C084DA76D021F0D3
:10E7AC006FD000E00093650E1DDD19F00E945FB480
:10E7BC0002C00E94625423D80DE41AE626D832D83F
:10E7CC00082FE4EFF0E70C9418F402E91AE61DD8D0
:10E7DC0016C009EA1AE6FBCF00EC1AE6F8CF07EDF3
:10E7EC001AE6F5CF0EEE1AE6F2CF05E01BE6EFCFF8
:10E7FC000CE11BE6ECCF03E31BE6E9CF80E042DA49
:10E80C0069F2D2D911F489910895D2D911F0DCD9D9
:10E81C0099F4082FEAE0F1E70C9418F4BEDABECFB5
:10E82C00FDDBBCCF6DDCBACF31DEB8CFE6D9B6CFCD
:10E83C0073DEB4CF7FDFB2CFBFD931F4882311F0B0
:10E84C008A95ACCF87E0AACFBBD929F4873010F4D6
:10E85C008395A4CFA0CF22DA19F40E94D2639ECF65
:10E86C0000915E0E0B3119F402E0F1DE97CF0091AE
:10E87C005E0E093011F401E0F8CF0E94FB6B8ECFD5
:10E88C0000E00093C90F0AB9C1CC0E947DBB009176
:10E89C00C90F002308958A9380E002C00E94FB6B8D
:10E8AC000E94056C03EA1CE60E940B6C0E94186C1B
:10E8BC00F2D959F00A9591F00A95B1F00A95D1F078
:10E8CC000A95F1F00A9511F127C040EE56E03CD0C4
:10E8DC0001ED1CE60E940B6C22961FC041EE56E027
:10E8EC0033D008EE1CE6F6CF42EE56E02DD00FEFFB
:10E8FC001CE6F0CF43EE56E027D006E11DE6EACF4A
:10E90C0044EE56E021D00DE21DE6E4CF45EE56E094
:10E91C001BD004E41DE6DECF80E00E94236C01F2E4
:10E92C0043D911F48991089547D931F4882311F012
:10E93C008A95B6CF85E0B4CF43D909F0AFCF8530F7
:10E94C0010F48395ADCFA8CF0E9437F10C942D6CA9
:10E95C008A9380E001C09FDF0091C90F002321F052
:10E96C008FDF00E00093650E3DDC19F00E945FB470
:10E97C0002C00E9462540E94056C04E61AE60E94D2
:10E98C000B6C0E94186C87D919F00A9531F008C0ED
:10E99C0003EA1CE60E940B6C04C00AEB1CE6FACFDF
:10E9AC0080E070D9C9F200D969F002D911F00CD904
:10E9BC0061F471D981F20A9539F40E940E6C61F2FE
:10E9CC000E94A37689910895C4CFF6D811F0F8D897
:10E9DC0019F401E08027C0CF0E94FB6BBDCF8A9356
:10E9EC00229700E0088309830DDC51F00E940E6C25
:10E9FC0009F45CC046E551E00E943AF108831983A2
:10EA0C000E94056C0BE51DE60E940B6C0E94186CB5
:10EA1C0002E71DE60E940B6C20E012E005E00E946C
:10EA2C00076821E015E101E10E94366820E08E01C3
:10EA3C000E943069802F0E946E688C33B9F10E945D
:10EA4C00056CA4D8A9D909E81DE60E940B6C229686
:10EA5C000E940E6C59F10E94056C0BE71AE60E949D
:10EA6C000B6C94D8012B11E000E069F40E945FB2AA
:10EA7C0002EC1AE50E940B6C22E531E00FEF1FEF60
:10EA8C0018D01AD00FC00E945FB208E01EE50E9499
:10EA9C000B6C22E531E008E010E00BD000E012E254
:10EAAC000BD074D82C5F3F4F04D04ED8229689914E
:10EABC000895A9010C9455F1B9016E5F7F4FAB011C
:10EACC000C9455F18A9381DA0E941D9943EA50E027
:10EADC000E9437F10C3329F40E94B97702C00E94CE
:10EAEC00D263D3DE21F0CCDE00E00093650E7ADB3E
:10EAFC0019F00E945FB402C00E946254CCD849F055
:10EB0C000A9599F00A95D9F00A9519F10A9559F1D7
:10EB1C0034C00E94056C73D00E940B6C0E94186C60
:10EB2C000FE11AE60E940B6C29C00E94056C67D09D
:10EB3C000E940B6C0E94186C06E31AE6F3CF0E943D
:10EB4C00056C5DD00E940B6C0E94186C0DE41AE6EB
:10EB5C00E9CF0E94056C53D00E940B6C0E94186C7C
:10EB6C0004E61AE6DFCF0E94056C49D00E940B6CBC
:10EB7C000E94186C0BE71AE6D5CF80E083D809F415
:10EB8C00B0CF00915E0E0A9589F0025039F10A95CA
:10EB9C0059F1035059F00A9509F4A1CF0A9569F17E
:10EBAC00075009F49ECF0B5029F115C0882311F49E
:10EBBC0047DB97CF813019F40E94076192CF8230E6
:10EBCC0011F4E8DD8ECF833011F4C2DE8ACF8430AD
:10EBDC0011F405DF86CF0E94FB6B83CF882311F0E5
:10EBEC008A957FCF84E07DCF843011F0839579CFE7
:10EBFC0080E077CF02E02BDD74CF01E0FCCF08E0A2
:10EC0C001AE60895919A899A909A0895919A909AF1
:10EC1C0008E00A95F1F708E00A95F1F7919808E0F9
:10EC2C000A95F1F708E00A95F1F79098089508E035
:10EC3C000A95F1F708E00A95F1F7909A08E00A9521
:10EC4C00F1F708E00A95F1F7919A0895919808E088
:10EC5C000A95F1F7909A00E10A95F1F790980895CA
:10EC6C00919A08E00A95F1F708E00A95F1F7909A65
:10EC7C0000E10A95F1F7EFCF18E007FB16F4919A33
:10EC8C0001C09198000F000000000000000000007F
:10EC9C00909A20E12A95F1F7909828E02A95F1F7BF
:10ECAC0028E02A95F1F71A9541F79198899808E090
:10ECBC000A95F1F708E00A95F1F7909A08E00A95A1
:10ECCC00F1F708E00A95F1F700B302709098899A71
:10ECDC0008959198899800E018E0000F20E12A959A
:10ECEC00F1F7909A28E02A95F1F728E02A95F1F7A8
:10ECFC008199016090981A9581F7899A0895BA9331
:10ED0C00AA93A0E6BAE093962C919397283011F031
:10ED1C0000E010C020E093962D932D932C939597A3
:10ED2C0098018D010E5D1F4F0E94B67C94960D9339
:10ED3C001C9301E0A991B991089500E011D00E94B3
:10ED4C0051F111D00E9451F111D00E9451F111D00A
:10ED5C000E9451F111D00E9451F111D00C9451F13B
:10ED6C0040EE56E0089541EE56E0089542EE56E02E
:10ED7C00089543EE56E0089544EE56E0089545EEAE
:10ED8C0056E008951AD023D00E94EDB800E010E0B0
:10ED9C00F801E950F14F2081E6E4FFE6E00FF11FA6
:10EDAC001491211711F000E004C00395003178F3A1
:10EDBC0001E000932B0F24960895249700EF1FEF8A
:10EDCC0027E030E0088319832A833B83089540E1D0
:10EDDC0027EF3EE08E010895F0DF00E0E6E4FFE669
:10EDEC0010E0E00FF11F2491F801E950F14F20835E
:10EDFC000395003198F3EBDF0E94A2B801E0D9CF64
:10EE0C0011E01093790EEBE2FFE614E0019FE00DA8
:10EE1C00F11D0591159125913491ECE2FFE003C0B1
:10EE2C0006D0E3ECFFE00ED02283338308954AED45
:10EE3C0056E00C943FF1E3ECFFE00081118122815C
:10EE4C00338108950083118308950E9475F4009115
:10EE5C00790E002311F400E036C03DD00E9437F14A
:10EE6C000A3519F437D00E9451F10E94CC3C28018C
:10EE7C0081E090E001C001964816590630F08C01F3
:10EE8C000E94E0410023B9F7E6CF0E94E13C280143
:10EE9C00012BB1F00E94E63CB02F81E090E001C064
:10EEAC0001964816590660F0A1E001C0A395BA1767
:10EEBC00B8F32A2F8C010E94573F0023B9F7CBCF10
:10EECC0000E009D003D0E6E00C9486F40E9451F1E6
:10EEDC0001E0089505EA44EA50E0089524970E9461
:10EEEC00B3EB00E0088309830A830B838E010E9435
:10EEFC004A3E002311F400E010C08E010E94893EAE
:10EF0C000023C9F38E010E94AA3E0023A1F38E01B7
:10EF1C000E94C83E002379F301E0249608950E94D4
:10EF2C0077F40091790E002311F400E019C0D3DFBF
:10EF3C000E9437F10A3519F4CDDF0E9451F10E947D
:10EF4C00CC3CD80181E090E001C00196A817B9072C
:10EF5C0030F08C010E94083E0023B9F7E6CF01E0A7
:10EF6C00E4E00C9488F44BEB50E00E943FF1EFEAA4
:10EF7C00FFE059DF4FEB50E00E943FF1E3EBFFE085
:10EF8C0052DF43EC50E00E9437F10093640E44ECE6
:10EF9C0050E00E9437F10093B80F45EC50E00E940E
:10EFAC0037F100937D0E46EC50E00E943FF1ECE40B
:10EFBC00FEE039DF4AEC50E00E9437F100937E0E00
:10EFCC004FE351E00E9437F10093B90F40E451E058
:10EFDC000E9437F10093BA0F41E451E00E9437F1DF
:10EFEC0000937F0E42E451E00E9437F10093800EB3
:10EFFC0043E451E00E9437F10093BB0F44E451E02D
:10F00C000E9437F10093BC0F45E451E00E9437F1A8
:10F01C000093810E46E451E00E9437F10093820E7A
:10F02C0047E451E00E9437F10093830E48E451E02D
:10F03C000E9437F10093BD0F49E451E00E9437F173
:10F04C000093BE0F4AE451E00E943AF1E2E5FEE083
:10F05C00F9DE89D00093650E8AD00093BF0F4EE481
:10F06C0051E00E943AF1E0ECFFE0ECDE40E551E0CB
:10F07C000E9437F10093C20F0091C20F0A9569F0FC
:10F08C000A9571F00A9579F00A9581F00A9591F03C
:10F09C000A9599F00A95A9F018C000E117E217C07B
:10F0AC0000E315E714C000E61AEE11C000E91FE5F5
:10F0BC0021E00EC000EC14EDFBCF00E819EA23E0D0
:10F0CC0007C000E41EE725E003C000E010E020E0EC
:10F0DC0030E0E0E4FEE0A7DEE8EFFFE022E531E01F
:10F0EC00A9010E943AF1AEDEB9016E5F44D00283F1
:10F0FC001383B9016C5F3FD004831583B9016A5F38
:10F10C003AD006831783285F3F4FA9010E943AF13A
:10F11C00008711874CE551E00E943AF1E6EFFFE0E1
:10F12C0091DE7EDE01E00093C70F4EED56E00E94AB
:10F13C0037F10093840E4FED56E00E9437F10093A7
:10F14C00850E41E551E00E9437F10093B70F00E0C6
:10F15C000E94B14901E00E94B14902E00E94B1490C
:10F16C0003E00C94B1494CE451E00C9437F14DE4BC
:10F17C0051E00C9437F17F4FAB010C943AF1269788
:10F18C0006E043EC50E0D4D045EC50E09FDE41E586
:10F19C0051E00E9451F144EC50E00E9451F100E02A
:10F1AC0010E020E030E04AED56E00E945CF146ECC5
:10F1BC0050E00E945CF14AEC50E00E9451F104E1F5
:10F1CC004FE351E00E9451F105E140E451E00E940F
:10F1DC0051F109E141E451E0ABD042E451E00E942D
:10F1EC0051F105E043E451E00E9451F108E044E4A0
:10F1FC0051E00E9451F10FE748E451E00E9451F1B7
:10F20C0006E149E451E00E9451F100E04AE451E08A
:10F21C000E9455F145E451E00E9451F146E451E061
:10F22C0055DE47E451E084D04DE451E00E9451F1A9
:10F23C0008EC4EE451E00E9455F100E040E551E04D
:10F24C000E9451F14EED56E00E9451F10FEF4FED3F
:10F25C0056E00E9451F1E8E5F3E073D06BEC70E0FE
:10F26C006BD023952C31B8F320E0E5E7F3E069D0BF
:10F27C0067EE70E061D0E2E9F3E063D063E071E047
:10F28C005BD023952C3188F320E0EFEAF3E059D0E2
:10F29C0065EA70E051D023952631B8F320E0E3EE17
:10F2AC00F3E04FD06FE171E047D023952430B8F3F1
:10F2BC0020E0E6ECF3E045D063E271E03DD023952D
:10F2CC002C31B8F30E946645002379F00E947445F6
:10F2DC00002359F08E010E941546002331F08E0157
:10F2EC000E94E6458E010E9447460E9439490E94C1
:10F2FC008F490E94F79C0E940D450E94DB9B08EAF7
:10F30C0010EC48E551E00E9455F10AEC10E04AE59A
:10F31C0051E00E9455F107E514E04CE551E00E94E4
:10F32C0055F10CE343EA50E00E9451F12696089502
:10F33C000E9451F102E00895620F731FAB010C940F
:10F34C0051F1E20FF31F0491089543EA50E00E943B
:10F35C0037F10C33089522E02BB9113031F40FEC56
:10F36C0009B900E02AD001E00895005069F00A952F
:10F37C0079F00A95C9F00A9579F00A9579F00A9511
:10F38C0079F00A9579F010C000E409B903E00FC0D8
:10F39C0000EA09B901E00BC007E607C003E305C0AA
:10F3AC0002E203C000E101C00FEC09B900E005D096
:10F3BC00112309F4579A01E008950093900008E195
:10F3CC000AB9089522E020939B00113029F40FEC28
:10F3DC0034D037D001E00895005069F00A9569F0F7
:10F3EC000A95A9F00A9559F00A9559F00A9559F021
:10F3FC000A9559F00CC017D00CC01AD00AC007E6F9
:10F40C0007C003E305C002E203C000E101C00FEC3A
:10F41C0014D017D0112329F400919A00006800939E
:10F42C009A0001E0089500E40093990003E0089528
:10F43C0000EA0093990001E008950093990000E020
:10F44C0008950093980008E100939A0008950050E5
:10F45C0069F00A9569F00A9569F00A9569F00A95C0
:10F46C0069F00A9569F00A9569F00EC0DCDF0EC0F0
:10F47C00DFDF0CC009C009C007E607C003E305C005
:10F48C0002E203C000E101C00FECD7DF009398004B
:10F49C0008958A930FEF0ABB0BBB04BB05BB07EBAC
:10F4AC0007BB0EE908BB0FEF01BB0CE102BB0FE67B
:10F4BC0002B903E403B908E8009361000093620009
:10F4CC00009165000061009365000FEF00936400EC
:10F4DC0007EF0093650000E00AB96E9804BD0DE7D4
:10F4EC0003BD0BE005BD07B7006807BF10E000E0E7
:10F4FC0069DF05B7006805BF00916D0002600093DD
:10F50C006D0000E000936C007894F89408EE13E022
:10F51C00E7E2FEE002831383789401E00093B70FD7
:10F52C000E941D9912DF21F482DC22D108F478DCD0
:10F53C0000E000938B0EF89400EA1FE0E7E2FEE097
:10F54C000483158378940E940FEA0E94E5B300238C
:10F55C0071F406DC0E9437F10F3F39F001DC0E9498
:10F56C0037F10395FDDB0E9451F101E3F7C00E94D6
:10F57C000E4A14B713FF0EC0F6DB0E9437F10F3F93
:10F58C0039F0F1DB0E9437F10395EDDB0E9451F16C
:10F59C0008E2E4C00E946645002371F4EDDB0E9492
:10F5AC0037F10F3F39F0E8DB0E9437F10395E4DBCC
:10F5BC000E9451F103E3D2C0C8DEC9F010E000E0B4
:10F5CC000E945FB20DE71FE520E00E94B4F411E049
:10F5DC0000E00E945FB201E91FE520E00E94B4F454
:10F5EC000E94FEB2CCDD01E00E947E45A6DBBBDCB6
:10F5FC0000E00093D30F80E010E00CEF0E9451EE7E
:10F60C00002341F001E00093D30F8093D40F0E94AC
:10F61C00DAEE06C0082F03951ADF8395873060F366
:10F62C000091D30F002399F402E00093D40F0FDF65
:10F63C0097D0A5DB0E9437F10F3F39F0A0DB0E9479
:10F64C0037F103959CDB0E9451F108E387C00E94BF
:10F65C00ABEF002311F084D0F8CF0E9459EF802F2C
:10F66C008DD0823029F489D0CBDB8CDB0DE276C0D7
:10F67C0000917D0E033020F400917D0E013039F4A1
:10F68C0002E045EC50E00E9451F100937D0E75D0E4
:10F69C006FD010F008EA62C00081118122813381A1
:10F6AC00AFDB0E942552002311F407E357C05BDD4A
:10F6BC00002329F010E05BDD07704DDE25C00E94B1
:10F6CC003252002369F455DB0E9437F10F3F39F0B9
:10F6DC0050DB0E9437F103954CDB0E9451F185E31E
:10F6EC0000E000938B000093890000938800009346
:10F6FC0087000AEF009386000DE000938A000091CA
:10F70C007D00006100937D003DDB002371F42EDB56
:10F71C000E9437F10F3F39F029DB0E9437F1039536
:10F72C0025DB0E9451F189EA02C0882311F0082FD1
:10F73C0015C00E947445002311F400E30FC000E0D3
:10F74C0013D049F001E010D031F002E00DD019F0E7
:10F75C0003E00AD011F404E301C000E0899108959C
:10F76C000DD069DB4DDB0ECB0E94B149002308950F
:10F77C00033010402040304008955DCB00E002BFC4
:10F78C0007E003BF07B7016007BF08950E9473F439
:10F79C002A97C80129013B014AD00F5F1F4F0083F4
:10F7AC00118304E1400E00E0501E15E4FC010687B5
:10F7BC001787408A518A3BD0FC01028B138B00E0E7
:10F7CC0010E4048B158B50E8468B578B10E0008FA0
:10F7DC00018F04E0FB01DC015E960E94A4F404E0BE
:10F7EC0010E0EEEFFFE0DC015A960E94A4F424E155
:10F7FC0030E08C01025F1F4FB3D0FC01008F118FE2
:10F80C0004E010E0F301DE0116960E94A4F4BE01A0
:10F81C0040E058E092018C010E94F352002311F455
:10F82C0000E001C001E02A96E8E00C9484F4E5E6DF
:10F83C00F4E00081118108950E9474F42B97D80193
:10F84C00622E8BD00785053409F082C00489158996
:10F85C001F73012B09F07CC024E130E000E61AE0B4
:10F86C00025F1F4F7DD00F3F1F4F09F071C0662004
:10F87C00A9F473D0068D178DE8EFFFE02681378150
:10F88C000217130751F469D000A111A1E8EFFFE0B2
:10F89C00208531850217130731F05AC000911810DA
:10F8AC00002309F455C059D0408851880EE2401607
:10F8BC0000E0500620F0A415B50509F04AC00CEE86
:10F8CC00400E0FEF501E028D138D0F831887048D81
:10F8DC00158D09871A879E018E010F5F1F4F0E949D
:10F8EC00EE3B002311F028810BC006E010E035D070
:10F8FC003696DE0111960E94A4F40E94273C202F1C
:10F90C008E010F5F1F4F0E94BE3B27D0068901302E
:10F91C0089F482010E9485760023D1F0BE01695FD3
:10F92C007F4F41E0920100E61AE030DF002381F0C6
:10F93C0001E00FC00689013159F4462D9E01295F63
:10F94C003F4F82010E947DEC002311F002E001C0C8
:10F95C0000E02B96E7E00C9485F4E0E6FAE00895DD
:10F96C009A938A93F80140E050E060E070E080E008
:10F97C0090E007C03324400D511D621D731D31965C
:10F98C0001968217930748F400801124222480FFEB
:10F99C00F1CF312C102C0024EECF8A0120E0AB01EA
:10F9AC0060E070E0400F511F621F721F8B01040F4B
:10F9BC00151F0F3F2FEF120711F00095109589912D
:10F9CC0099910895BA92AA929A928A927A926A928C
:10F9DC005A924A92BA93AA939A938A9367E674E0DE
:10F9EC00F8018380E7E6F4E026E330E031932A95D2
:10F9FC00E1F73B0126E0620E731E482C5524F801FA
:10FA0C002081243009F054C0D3014BEA55E020E0AA
:10FA1C00E22FF0E0E40FF51F0080002009F448C04D
:10FA2C00802D90E0E0E3AE2EBB24B89EB02CA99EB6
:10FA3C00B00CA89EB10C87E084199040880F991FD8
:10FA4C00800D9B1D0D013323E0E0F9E161F4E80F1B
:10FA5C00F91F94909D92E0E0F9E10196E80FF91FEF
:10FA6C0004900C921FC0E80FF91F94909294EFE051
:10FA7C009E22F0010080090C0D92E0E0F9E1E80F04
:10FA8C00F91F04900294E0EF0E220C92E0E0F9E1F1
:10FA9C000196E80FF91F849182958F70FD0100800B
:10FAAC00080E0D92E1E03E2723952C3108F4B0CFDF
:10FABC00F8012081253009F055C030E0D3014BEA24
:10FACC0055E020E0E22FF0E0E40FF51F008000206D
:10FADC0009F448C0802D90E0E0E3AE2EBB24B89E24
:10FAEC00B02CA99EB00CA89EB10C8FE0841990404C
:10FAFC00880F991F800D9B1D0D013323E0E0F9E168
:10FB0C0061F4E80FF91F94909D92E0E0F9E1019601
:10FB1C00E80FF91F04900C921FC0E80FF91F949086
:10FB2C009294EFE09E22F0010080090C0D92E0E02F
:10FB3C00F9E1E80FF91F04900294E0EF0E220C9209
:10FB4C00E0E0F9E10196E80FF91F849182958F703E
:10FB5C00FD010080080E0D92E1E03E2723952C312B
:10FB6C0008F4B0CFF8012081263009F055C030E000
:10FB7C00D3014BEA55E020E0E22FF0E0E40FF51F53
:10FB8C000080002009F448C0802D90E0E0E32E2E88
:10FB9C003324389E302C299E300C289E310C87E162
:10FBAC0084199040880F991F800D931D0D013323EC
:10FBBC00E0E0F9E161F4E80FF91F24902D92E0E008
:10FBCC00F9E10196E80FF91F04900C921FC0E80FA1
:10FBDC00F91F24902294EFE02E22F0010080020CF9
:10FBEC000D92E0E0F9E1E80FF91F04900294E0EFC8
:10FBFC000E220C92E0E0F9E10196E80FF91F8491D6
:10FC0C0082958F70FD010080080E0D92E1E03E2779
:10FC1C0023952C3108F4B0CFCB010396F801208149
:10FC2C002C30E9F4DC0146E057E020E0E22FF0E074
:10FC3C00E40FF51F6080662091F030EFA32E3AE0C0
:10FC4C00B32E30E1639EF0013F96E419F040AE0E06
:10FC5C00BF1EF50134913D932395223338F3F801FF
:10FC6C0020812B30E1F4DC0146E057E020E0E22F6C
:10FC7C00F0E0E40FF51F2080222089F0E0EFFAE09D
:10FC8C0030E1239E37E0030E30E0131E04181508F4
:10FC9C00E00DF11D34913D932395223340F3F8018F
:10FCAC0020812F30E1F4DC0149E357E020E0E22F22
:10FCBC00F0E0E40FF51F6080662089F0E0EFFAE0D9
:10FCCC0030E1639E3FE0030E30E0131E041815086C
:10FCDC00E00DF11D34913D932395223340F3F8014F
:10FCEC0020812E30E1F4DC0149E357E020E0E22FE3
:10FCFC00F0E0E40FF51F2080222089F0E0EFFAE01D
:10FD0C0030E1239E37E0030E30E0131E0418150873
:10FD1C00E00DF11D34913D932395223340F3F8010E
:10FD2C0020812231E1F4DC014CE657E020E0E22FA7
:10FD3C00F0E0E40FF51F6080662089F0E0EFFAE058
:10FD4C0030E1639E3FE0030E30E0131E04181508EB
:10FD5C00E00DF11D34913D932395223340F3F801CE
:10FD6C0020812131E9F4DC014CE657E020E0E22F60
:10FD7C00F0E0E40FF51F3081332391F080EF9AE02F
:10FD8C00E0E13E9F37E0030E30E0131E0418150827
:10FD9C00800D911DFC0134913D932395223338F352
:10FDAC00F80120812C3001F5A0913510B0E0A60FA0
:10FDBC00B71F42E056E020E0E22FF0E0E40FF51F21
:10FDCC002080222089F0E0EFFAE030E1239E3FE032
:10FDDC00030E30E0131E04181508E00DF11D3491CC
:10FDEC003D9323952B3040F3F80120812B3009F5FE
:10FDFC00A0913510B0E0A60FB71F42E056E020E00E
:10FE0C00E22FF0E0E40FF51F3081332391F080EF07
:10FE1C009AE0E0E13E9F37E0030E30E0131E041839
:10FE2C001508800D911DFC0134913D9323952B30C9
:10FE3C0038F387E694E08396F80120812F30E1F4C3
:10FE4C00DC014EE056E020E0E22FF0E0E40FF51F7D
:10FE5C006080662089F0E0EFFAE030E1639E3FE0DD
:10FE6C00030E30E0131E04181508E00DF11D34913B
:10FE7C003D9323952B3040F3F80120812E30E1F493
:10FE8C00DC014EE056E020E0E22FF0E0E40FF51F3D
:10FE9C002080222089F0E0EFFAE030E1239E37E069
:10FEAC00030E30E0131E04181508E00DF11D3491FB
:10FEBC003D9323952B3040F3F80120812231E1F45E
:10FECC00DC014AE156E020E0E22FF0E0E40FF51F00
:10FEDC006080662089F0E0EFFAE030E1639E3FE05D
:10FEEC00030E30E0131E04181508E00DF11D3491BB
:10FEFC003D9323952B3040F3F80120812131E1F41F
:10FF0C00DC014AE156E020E0E22FF0E0E40FF51FBF
:10FF1C003081332389F0E0EFFAE060E1369F37E07F
:10FF2C00030E30E0131E04181508E00DF11D34917A
:10FF3C003D9323952B3040F3F801A181B2818CE9DC
:10FF4C0094E006E3402EFC0120818D010E9444B90F
:10FF5C00119601974A94B9F789919991A991B99100
:10FF6C00499059906990799089909990A990B990FD
:10FF7C000895FA92EA92DA92CA92BA92AA929A9254
:10FF8C008A927A926A925A924A92BA93AA939A93C2
:10FF9C008A932D97B80107E6802E04E0902EFB0182
:10FFAC0003810E83E7E6F4E006E310E011930A9573
:10FFBC00E1F7CE80DD2407E00C1910400B871C877D
:10FFCC00000F111F088319830FE010E00C1910406B
:10FFDC00000F111F0A831B8307E110E00C1910405E
:10FFEC00000F111F0C831D83EDE9F4E00281002347
:10FFFC0009F48CC2FB011081011709F063C010E0F9
:020000021000EC
:10000C00EDE9F4E041805524480C591C4BEA55E0CD
:10001C0000E0E02FF0E0E40FF51F2081222309F42B
:10002C0051C0E22FF0E020E330E03E9F302D2F9FB7
:10003C00300D2E9F310D88819981800D931F020107
:10004C001123E0E0F9E191F4E80FF91F2491F2019A
:10005C00208321E0420E20E0521EE0E0F9E10196FF
:10006C00E80FF91F2491F201208326C0E80FF91F35
:10007C00249122952F70F0013081320F308321E0D2
:10008C00420E20E0521EE0E0F9E1E80FF91F249146
:10009C002295207FF2012083E0E0F9E10196E80F40
:1000AC00F91F249122952F70F2013081320F308389
:1000BC0021E0420E20E0521E21E0122703950C3164
:1000CC0008F4A7CFEDE9F4E0828190E00196FB0102
:1000DC00008110E08017904009F062C0EDE9F4E077
:1000EC0041805524480C591C4BEA55E000E0E02FA8
:1000FC00F0E0E40FF51F2081222309F451C0E22F18
:10010C00F0E020E330E03E9F302D2F9F300D2E9FEE
:10011C00310D8A819B81800D931F02011123E0E038
:10012C00F9E191F4E80FF91F2491F201208321E009
:10013C00420E20E0521EE0E0F9E10196E80FF91FB3
:10014C002491F201208326C0E80FF91F24912295F7
:10015C002F70F0013081320F308321E0420E20E00D
:10016C00521EE0E0F9E1E80FF91F24912295207F5F
:10017C00F2012083E0E0F9E10196E80FF91F2491E8
:10018C0022952F70F2013081320F308321E0420E24
:10019C0020E0521E21E0122703950C3108F4A7CF62
:1001AC00EDE9F4E0828190E00296FB01008110E021
:1001BC008017904009F061C0EDE9F4E041805524CE
:1001CC00480C591C4BEA55E000E0E02FF0E0E40F3E
:1001DC00F51F2081222309F450C0222E332420E362
:1001EC0030E0329D302D239D300D229D310D8C81C0
:1001FC009D81800D931F02011123E0E0F9E189F448
:10020C00E80FF91F2491F201208321E0420E531CC8
:10021C00E0E0F9E10196E80FF91F2491F201208347
:10022C0026C0E80FF91F249122952F70F001308120
:10023C00320F308321E0420E20E0521EE0E0F9E163
:10024C00E80FF91F24912295207FF2012083E0E032
:10025C00F9E10196E80FF91F249122952F70F20114
:10026C003081320F308321E0420E20E0521E21E01B
:10027C00122703950C3108F4A8CFEDE9F4E0828144
:10028C0090E00396FB01008110E08017904009F08C
:10029C0062C0EDE9F4E041805524480C591C48EC4F
:1002AC0055E000E0E02FF0E0E40FF51F2081222361
:1002BC0009F451C0E22FF0E020E330E03E9F302DF6
:1002CC002F9F300D2E9F310D88819981800D931FAA
:1002DC0002011123E0E0F9E191F4E80FF91F2491F8
:1002EC00F201208321E0420E20E0521EE0E0F9E111
:1002FC000196E80FF91F2491F201208326C0E80F24
:10030C00F91F249122952F70F0013081320F308328
:10031C0021E0420E20E0521EE0E0F9E1E80FF91F67
:10032C0024912295207FF2012083E0E0F9E10196EF
:10033C00E80FF91F249122952F70F2013081320FB2
:10034C00308321E0420E20E0521E21E0122703955B
:10035C000C3108F4A7CFEDE9F4E0828190E004962B
:10036C00FB01008110E08017904009F062C0EDE9BC
:10037C00F4E041805524480C591C48EC55E000E051
:10038C00E02FF0E0E40FF51F2081222309F451C087
:10039C00E22FF0E020E330E03E9F302D2F9F300D18
:1003AC002E9F310D8A819B81800D931F0201112399
:1003BC00E0E0F9E191F4E80FF91F2491F2012083B8
:1003CC0021E0420E20E0521EE0E0F9E10196E80F38
:1003DC00F91F2491F201208326C0E80FF91F249104
:1003EC0022952F70F0013081320F308321E0420EC4
:1003FC0020E0521EE0E0F9E1E80FF91F249122956C
:10040C00207FF2012083E0E0F9E10196E80FF91F6B
:10041C00249122952F70F2013081320F308321E02C
:10042C00420E20E0521E21E0122703950C3108F4F5
:10043C00A7CFEDE9F4E0828190E00596FB01008105
:10044C0010E08017904009F061C0EDE9F4E04180C4
:10045C005524480C591C48EC55E000E0E02FF0E026
:10046C00E40FF51F2081222309F450C0222E3324DF
:10047C0020E330E0329D302D239D300D229D310D37
:10048C008C819D81800D931F02011123E0E0F9E125
:10049C0089F4E80FF91F2491F201208321E0420E28
:1004AC00531CE0E0F9E10196E80FF91F2491F201E9
:1004BC00208326C0E80FF91F249122952F70F0019C
:1004CC003081320F308321E0420E20E0521EE0E0FA
:1004DC00F9E1E80FF91F24912295207FF201208386
:1004EC00E0E0F9E10196E80FF91F249122952F70B5
:1004FC00F2013081320F308321E0420E20E0521E97
:10050C0021E0122703950C3108F4A8CFEDE9F4E0B3
:10051C000481002309F48CC2FB011081011709F03E
:10052C0063C010E0EDE9F4E043805524480C591CFD
:10053C0045EE55E000E0E02FF0E0E40FF51F2081E0
:10054C00222309F451C0E22FF0E020E330E03E9F7B
:10055C00302D2F9F300D2E9F310D88819981800D6C
:10056C00931F02011123E0E0F9E191F4E80FF91F68
:10057C002491F201208321E0420E20E0521EE0E0A3
:10058C00F9E10196E80FF91F2491F201208326C0AE
:10059C00E80FF91F249122952F70F0013081320F52
:1005AC00308321E0420E20E0521EE0E0F9E1E80F3A
:1005BC00F91F24912295207FF2012083E0E0F9E1DC
:1005CC000196E80FF91F249122952F70F2013081CA
:1005DC00320F308321E0420E20E0521E21E0122720
:1005EC0003950C3108F4A7CFEDE9F4E0848190E099
:1005FC000196FB01008110E08017904009F062C069
:10060C00EDE9F4E043805524480C591C45EE55E0C7
:10061C0000E0E02FF0E0E40FF51F2081222309F425
:10062C0051C0E22FF0E020E330E03E9F302D2F9FB1
:10063C00300D2E9F310D8A819B81800D931F0201FD
:10064C001123E0E0F9E191F4E80FF91F2491F20194
:10065C00208321E0420E20E0521EE0E0F9E10196F9
:10066C00E80FF91F2491F201208326C0E80FF91F2F
:10067C00249122952F70F0013081320F308321E0CC
:10068C00420E20E0521EE0E0F9E1E80FF91F249140
:10069C002295207FF2012083E0E0F9E10196E80F3A
:1006AC00F91F249122952F70F2013081320F308383
:1006BC0021E0420E20E0521E21E0122703950C315E
:1006CC0008F4A7CFEDE9F4E0848190E00296FB01F9
:1006DC00008110E08017904009F061C0EDE9F4E072
:1006EC0043805524480C591C45EE55E000E0E02FA2
:1006FC00F0E0E40FF51F2081222309F450C0222ED4
:10070C00332420E330E0329D302D239D300D229D8B
:10071C00310D8C819D81800D931F02011123E0E02E
:10072C00F9E189F4E80FF91F2491F201208321E00B
:10073C00420E531CE0E0F9E10196E80FF91F2491F9
:10074C00F201208326C0E80FF91F249122952F7007
:10075C00F0013081320F308321E0420E20E0521E36
:10076C00E0E0F9E1E80FF91F24912295207FF201D6
:10077C002083E0E0F9E10196E80FF91F249122951E
:10078C002F70F2013081320F308321E0420E20E0D5
:10079C00521E21E0122703950C3108F4A8CFEDE985
:1007AC00F4E0848190E00396FB01008110E0801757
:1007BC00904009F062C0EDE9F4E043805524480C08
:1007CC00591C46E256E000E0E02FF0E0E40FF51F84
:1007DC002081222309F451C0E22FF0E020E330E025
:1007EC003E9F302D2F9F300D2E9F310D888199818A
:1007FC00800D931F02011123E0E0F9E191F4E80F61
:10080C00F91F2491F201208321E0420E20E0521EB8
:10081C00E0E0F9E10196E80FF91F2491F201208341
:10082C0026C0E80FF91F249122952F70F00130811A
:10083C00320F308321E0420E20E0521EE0E0F9E15D
:10084C00E80FF91F24912295207FF2012083E0E02C
:10085C00F9E10196E80FF91F249122952F70F2010E
:10086C003081320F308321E0420E20E0521E21E015
:10087C00122703950C3108F4A7CFEDE9F4E084813D
:10088C0090E00496FB01008110E08017904009F085
:10089C0062C0EDE9F4E043805524480C591C46E253
:1008AC0056E000E0E02FF0E0E40FF51F208122235A
:1008BC0009F451C0E22FF0E020E330E03E9F302DF0
:1008CC002F9F300D2E9F310D8A819B81800D931FA0
:1008DC0002011123E0E0F9E191F4E80FF91F2491F2
:1008EC00F201208321E0420E20E0521EE0E0F9E10B
:1008FC000196E80FF91F2491F201208326C0E80F1E
:10090C00F91F249122952F70F0013081320F308322
:10091C0021E0420E20E0521EE0E0F9E1E80FF91F61
:10092C0024912295207FF2012083E0E0F9E10196E9
:10093C00E80FF91F249122952F70F2013081320FAC
:10094C00308321E0420E20E0521E21E01227039555
:10095C000C3108F4A7CFEDE9F4E0848190E0059622
:10096C00FB01008110E08017904009F061C0EDE9B7
:10097C00F4E043805524480C591C46E256E000E054
:10098C00E02FF0E0E40FF51F2081222309F450C082
:10099C00222E332420E330E0329D302D239D300D68
:1009AC00229D310D8C819D81800D931F020111239D
:1009BC00E0E0F9E189F4E80FF91F2491F2012083BA
:1009CC0021E0420E531CE0E0F9E10196E80FF91F1B
:1009DC002491F201208326C0E80FF91F249122955F
:1009EC002F70F0013081320F308321E0420E20E075
:1009FC00521EE0E0F9E1E80FF91F24912295207FC7
:100A0C00F2012083E0E0F9E10196E80FF91F24914F
:100A1C0022952F70F2013081320F308321E0420E8B
:100A2C0020E0521E21E0122703950C3108F4A8CFC8
:100A3C00EDE9F4E00681002309F45EC0802F90E01C
:100A4C000196FB0100818017904049F5EDE9F4E037
:100A5C0045805524480C591C43E456E000E0E02F37
:100A6C00F0E0E40FF51F20802220C9F010EF612E7A
:100A7C001AE0712E10E1219EEFE00E0EE0E01E1E3A
:100A8C000C181D08600C711CF3011491F2011083F9
:100A9C0011E0410E10E0511E0395083000F3EDE912
:100AAC00F4E00681FB011081011731F5EDE9F4E06A
:100ABC0045805524480C591C43E456E000E0E02FD7
:100ACC00F0E0E40FF51F20812223B1F0E0EFFAE013
:100ADC0010E1219F17E0010E10E0111E0C181D08EB
:100AEC00E00DF11D1491F201108311E0410E10E0A4
:100AFC00511E0395083018F3EDE9F4E0008500234E
:100B0C0009F45BC0802F90E00196FB0100818017F7
:100B1C00904031F5EDE9F4E047805524480C591C20
:100B2C004CE456E000E0E02FF0E0E40FF51F2080ED
:100B3C002220B1F0E0EFFAE010E1219E1FE0010E5F
:100B4C0010E0111E0C181D08E00DF11D1491F2019E
:100B5C00108311E0410E10E0511E03950A3018F37A
:100B6C00EDE9F4E00085FB011081011731F5EDE9A9
:100B7C00F4E047805524480C591C4CE456E000E046
:100B8C00E02FF0E0E40FF51F20812223B1F0E0EF1D
:100B9C00FAE010E1219F17E0010E10E0111E0C1875
:100BAC001D08E00DF11D1491F201108311E0410EAE
:100BBC0010E0511E03950A3018F3EDE9F4E00285BC
:100BCC00002309F45BC0802F90E00196FB010081AB
:100BDC008017904031F5EDE9F4E041845524480C40
:100BEC00591C47E556E000E0E02FF0E0E40FF51F5C
:100BFC0020802220B1F0E0EFFAE010E1219E1FE00E
:100C0C00010E10E0111E0C181D08E00DF11D1491C1
:100C1C00F201108311E0410E10E0511E03950830D3
:100C2C0018F3EDE9F4E00285FB011081011731F5B1
:100C3C00EDE9F4E041845524480C591C47E556E095
:100C4C0000E0E02FF0E0E40FF51F20812223B1F04B
:100C5C00E0EFFAE010E1219F17E0010E10E0111E09
:100C6C000C181D08E00DF11D1491F201108311E018
:100C7C00410E10E0511E0395083018F30C2D06950B
:100C8C0010E00F8318870FE02F81021B104009879B
:100C9C001A8707E0E02EFF240F811885E01AF10A6D
:100CAC00EDE9F4E00485002309F4BEC02F813885FA
:100CBC0031952195304010E00E5F1F4FFB014081B4
:100CCC000417104039F5EDE9F4E043845524480C41
:100CDC00591C40E756E000E0E02FF0E0E40FF51F70
:100CEC0060806620B9F010EF212E1AE0312E10E151
:100CFC00619EF9013B96E00DF11D2E0E3F1EF10198
:100D0C001491F201108311E0410E10E0511E039575
:100D1C00093010F3EDE9F4E0048510E00D5F1F4F8E
:100D2C00FB0140810417104021F5EDE9F4E0438408
:100D3C005524480C591C40E756E000E0E02FF0E049
:100D4C00E40FF51F20802220A1F0E0EFFAE010E183
:100D5C00219E69847A84600C711CE60DF71D149138
:100D6C00F201108311E0410E10E0511E0395093081
:100D7C0028F3EDE9F4E00485FB011081011739F546
:100D8C00EDE9F4E043845524480C591C40E756E047
:100D9C0000E0E02FF0E0E40FF51F60806620B9F072
:100DAC0010EF212E1AE0312E10E1619EF9013396DD
:100DBC00E00DF11D2E0E3F1EF1011491F201108376
:100DCC0011E0410E10E0511E0395093010F3EDE9CE
:100DDC00F4E0048510E00F5F1F4FFB012081021728
:100DEC00104011F5EDE9F4E043845524480C591CEE
:100DFC0040E756E000E0E02FF0E0E40FF51F208123
:100E0C00222391F0E0EFFAE010E1219F0E0C1F1C61
:100E1C00E00DF11D1491F201108311E0410E10E070
:100E2C00511E0395093038F3EDE9F4E006850023F3
:100E3C0009F45BC0802F90E00196FB0100818017C4
:100E4C00904031F5EDE9F4E045845524480C591CEB
:100E5C004AE756E000E0E02FF0E0E40FF51F2080B9
:100E6C002220B1F0E0EFFAE010E1219E1FE0010E2C
:100E7C0010E0111E0C181D08E00DF11D1491F2016B
:100E8C00108311E0410E10E0511E0395093018F348
:100E9C00EDE9F4E00685FB011081011731F5EDE970
:100EAC00F4E045845524480C591C4AE756E000E010
:100EBC00E02FF0E0E40FF51F20812223B1F0E0EFEA
:100ECC00FAE010E1219F17E0010E10E0111E0C1842
:100EDC001D08E00DF11D1491F201108311E0410E7B
:100EEC0010E0511E0395093018F3EDE9F4E0008988
:100EFC00002309F443C1FB011081011709F063C001
:100F0C0010E0EDE9F4E047845524480C591C44EDFD
:100F1C0054E000E0E02FF0E0E40FF51F20812223E5
:100F2C0009F451C0E22FF0E020E330E03E9F302D79
:100F3C002F9F300D2E9F310D88819981800D931F2D
:100F4C0002011123E0E0F9E191F4E80FF91F24917B
:100F5C00F201208321E0420E20E0521EE0E0F9E194
:100F6C000196E80FF91F2491F201208326C0E80FA7
:100F7C00F91F249122952F70F0013081320F3083AC
:100F8C0021E0420E20E0521EE0E0F9E1E80FF91FEB
:100F9C0024912295207FF2012083E0E0F9E1019673
:100FAC00E80FF91F249122952F70F2013081320F36
:100FBC00308321E0420E20E0521E21E012270395DF
:100FCC00073008F4A7CFEDE9F4E0808990E00196B2
:100FDC00FB01008110E08017904009F062C0EDE940
:100FEC00F4E047845524480C591C44ED54E000E0CF
:100FFC00E02FF0E0E40FF51F2081222309F451C00B
:10100C00E22FF0E020E330E03E9F302D2F9F300D9B
:10101C002E9F310D8A819B81800D931F020111231C
:10102C00E0E0F9E191F4E80FF91F2491F20120833B
:10103C0021E0420E20E0521EE0E0F9E10196E80FBB
:10104C00F91F2491F201208326C0E80FF91F249187
:10105C0022952F70F0013081320F308321E0420E47
:10106C0020E0521EE0E0F9E1E80FF91F24912295EF
:10107C00207FF2012083E0E0F9E10196E80FF91FEF
:10108C00249122952F70F2013081320F308321E0B0
:10109C00420E20E0521E21E012270395073008F47F
:1010AC00A7CFEDE9F4E0808990E00296FB01008186
:1010BC0010E08017904009F061C0EDE9F4E047843E
:1010CC005524480C591C44ED54E000E0E02FF0E0AE
:1010DC00E40FF51F2081222309F450C0222E332463
:1010EC0020E330E0329D302D239D300D229D310DBB
:1010FC008C819D81800D931F02011123E0E0F9E1A9
:10110C0089F4E80FF91F2491F201208321E0420EAB
:10111C00531CE0E0F9E10196E80FF91F2491F2016C
:10112C00208326C0E80FF91F249122952F70F0011F
:10113C003081320F308321E0420E20E0521EE0E07D
:10114C00F9E1E80FF91F24912295207FF201208309
:10115C00E0E0F9E10196E80FF91F249122952F7038
:10116C00F2013081320F308321E0420E20E0521E1A
:10117C0021E012270395073008F4A8CFEDE9F4E03D
:10118C000289002309F45BC0802F90E00196FB01DB
:10119C0000818017904031F5EDE9F4E04188552449
:1011AC00480C591C4CED54E000E0E02FF0E0E40F4B
:1011BC00F51F20802220B1F0E0EFFAE010E1219E33
:1011CC001FE0010E10E0111E0C181D08E00DF11DA2
:1011DC001491F201108311E0410E10E0511E0395A1
:1011EC00063018F3EDE9F4E00289FB0110810117D8
:1011FC0031F5EDE9F4E041885524480C591C4CEDCF
:10120C0054E000E0E02FF0E0E40FF51F20812223F2
:10121C00B1F0E0EFFAE010E1219F17E0010E10E0D1
:10122C00111E0C181D08E00DF11D1491F201108314
:10123C0011E0410E10E0511E0395063018F3EDE954
:10124C00F4E00489002309F45BC0802F90E0019640
:10125C00FB0100818017904031F5EDE9F4E0438803
:10126C005524480C591C44E856E000E0E02FF0E00F
:10127C00E40FF51F20802220B1F0E0EFFAE010E13E
:10128C00219E1FE0010E10E0111E0C181D08E00D30
:10129C00F11D1491F201108311E0410E10E0511E6A
:1012AC000395043018F3EDE9F4E00489FB01108197
:1012BC00011731F5EDE9F4E043885524480C591C2D
:1012CC0044E856E000E0E02FF0E0E40FF51F208149
:1012DC002223B1F0E0EFFAE010E1219F17E0010EBC
:1012EC0010E0111E0C181D08E00DF11D1491F201F7
:1012FC00108311E0410E10E0511E0395043018F3D9
:10130C00EDE9F4E00689002309F45BC0802F90E03E
:10131C000196FB0100818017904031F5EDE9F4E076
:10132C0045885524480C591C49E856E000E0E02F4C
:10133C00F0E0E40FF51F20802220B1F0E0EFFAE09E
:10134C0010E1219E1FE0010E10E0111E0C181D086B
:10135C00E00DF11D1491F201108311E0410E10E02B
:10136C00511E0395063018F3EDE9F4E00689FB01F4
:10137C001081011731F5EDE9F4E045885524480C4E
:10138C00591C49E856E000E0E02FF0E0E40FF51FAF
:10139C0020812223B1F0E0EFFAE010E1219F17E069
:1013AC00010E10E0111E0C181D08E00DF11D14911A
:1013BC00F201108311E0410E10E0511E039506302E
:1013CC0018F3EDE9F4E0008D002309F4FCC2802F42
:1013DC0090E00196FB0100818017904031F5EDE91A
:1013EC00F4E047885524480C591C43ED56E000E0C6
:1013FC00E02FF0E0E40FF51F20802220B1F0E0EFA9
:10140C00FAE010E1219E1FE0010E10E0111E0C18F5
:10141C001D08E00DF11D1491F201108311E0410E35
:10142C0010E0511E0395023318F3EDE9F4E0008D42
:10143C00FB011081011731F5EDE9F4E047885524E3
:10144C00480C591C43ED56E000E0E02FF0E0E40FAF
:10145C00F51F20812223B1F0E0EFFAE010E1219F8B
:10146C0017E0010E10E0111E0C181D08E00DF11D07
:10147C001491F201108311E0410E10E0511E0395FE
:10148C00023318F3EDE9F4E0808D90E00396FB0154
:10149C00008110E08017904031F5EDE9F4E04788C9
:1014AC005524480C591C46E057E000E0E02FF0E0D2
:1014BC00E40FF51F20802220B1F0E0EFFAE010E1FC
:1014CC00219E1FE0010E10E0111E0C181D08E00DEE
:1014DC00F11D1491F201108311E0410E10E0511E28
:1014EC000395023318F3EDE9F4E0808D90E0029659
:1014FC00FB0100818017910731F5EDE9F4E0478895
:10150C005524480C591C46E057E000E0E02FF0E071
:10151C00E40FF51F20812223B1F0E0EFFAE010E197
:10152C00219F17E0010E10E0111E0C181D08E00D94
:10153C00F11D1491F201108311E0410E10E0511EC7
:10154C000395023318F3EDE9F4E0808D90E00596F5
:10155C00FB0100818017910731F5EDE9F4E0478834
:10156C005524480C591C49E357E000E0E02FF0E00B
:10157C00E40FF51F20802220B1F0E0EFFAE010E13B
:10158C00219E1FE0010E10E0111E0C181D08E00D2D
:10159C00F11D1491F201108311E0410E10E0511E67
:1015AC000395023318F3EDE9F4E0808D90E0049696
:1015BC00FB0100818017910731F5EDE9F4E04788D4
:1015CC005524480C591C49E357E000E0E02FF0E0AB
:1015DC00E40FF51F20812223B1F0E0EFFAE010E1D7
:1015EC00219F17E0010E10E0111E0C181D08E00DD4
:1015FC00F11D1491F201108311E0410E10E0511E07
:10160C000395023318F3EDE9F4E0808D90E0079632
:10161C00FB0100818017910731F5EDE9F4E0478873
:10162C005524480C591C4CE657E000E0E02FF0E044
:10163C00E40FF51F20802220B1F0E0EFFAE010E17A
:10164C00219E1FE0010E10E0111E0C181D08E00D6C
:10165C00F11D1491F201108311E0410E10E0511EA6
:10166C000395023318F3EDE9F4E0808D90E00696D3
:10167C00FB0100818017910731F5EDE9F4E0478813
:10168C005524480C591C4CE657E000E0E02FF0E0E4
:10169C00E40FF51F20812223B1F0E0EFFAE010E116
:1016AC00219F17E0010E10E0111E0C181D08E00D13
:1016BC00F11D1491F201108311E0410E10E0511E46
:1016CC000395023318F3EDE9F4E0808D90E0099670
:1016DC00FB0100818017910731F5EDE9F4E04788B3
:1016EC005524480C591C4FE957E000E0E02FF0E07E
:1016FC00E40FF51F20802220B1F0E0EFFAE010E1BA
:10170C00219E1FE0010E10E0111E0C181D08E00DAB
:10171C00F11D1491F201108311E0410E10E0511EE5
:10172C000395023318F3EDE9F4E0808D90E0089610
:10173C00FB0100818017910731F5EDE9F4E0478852
:10174C005524480C591C4FE957E000E0E02FF0E01D
:10175C00E40FF51F20812223B1F0E0EFFAE010E155
:10176C00219F17E0010E10E0111E0C181D08E00D52
:10177C00F11D1491F201108311E0410E10E0511E85
:10178C000395023318F3EDE9F4E0808D90E00B96AD
:10179C00FB0100818017910731F5EDE9F4E04788F2
:1017AC005524480C591C42ED57E000E0E02FF0E0C6
:1017BC00E40FF51F20802220B1F0E0EFFAE010E1F9
:1017CC00219E1FE0010E10E0111E0C181D08E00DEB
:1017DC00F11D1491F201108311E0410E10E0511E25
:1017EC000395023318F3EDE9F4E0808D90E00A964E
:1017FC00FB0100818017910731F5EDE9F4E0478892
:10180C005524480C591C42ED57E000E0E02FF0E065
:10181C00E40FF51F20812223B1F0E0EFFAE010E194
:10182C00219F17E0010E10E0111E0C181D08E00D91
:10183C00F11D1491F201108311E0410E10E0511EC4
:10184C000395023318F3EDE9F4E0808D90E00D96EA
:10185C00FB0100818017910731F5EDE9F4E0478831
:10186C005524480C591C45E058E000E0E02FF0E00E
:10187C00E40FF51F20802220B1F0E0EFFAE010E138
:10188C00219E1FE0010E10E0111E0C181D08E00D2A
:10189C00F11D1491F201108311E0410E10E0511E64
:1018AC000395023318F3EDE9F4E0808D90E00C968B
:1018BC00FB0100818017910731F5EDE9F4E04788D1
:1018CC005524480C591C45E058E000E0E02FF0E0AE
:1018DC00E40FF51F20812223B1F0E0EFFAE010E1D4
:1018EC00219F17E0010E10E0111E0C181D08E00DD1
:1018FC00F11D1491F201108311E0410E10E0511E04
:10190C000395023318F3EDE9F4E0808D90E00F9627
:10191C00FB0100818017910731F5EDE9F4E0478870
:10192C005524480C591C48E358E000E0E02FF0E047
:10193C00E40FF51F20802220B1F0E0EFFAE010E177
:10194C00219E1FE0010E10E0111E0C181D08E00D69
:10195C00F11D1491F201108311E0410E10E0511EA3
:10196C000395023318F3EDE9F4E0808D90E00E96C8
:10197C00FB0100818017910731F5EDE9F4E0478810
:10198C005524480C591C48E358E000E0E02FF0E0E7
:10199C00E40FF51F20812223B1F0E0EFFAE010E113
:1019AC00219F17E0010E10E0111E0C181D08E00D10
:1019BC00F11D1491F201108311E0410E10E0511E43
:1019CC000395023318F3EDE9F4E0028D002309F4DA
:1019DC00F3C6802F90E00396FB01008110E0801786
:1019EC00904091F5EDE9F4E0818D90E00C96863312
:1019FC00904054F5418C5524480C591C0AE0400E7B
:101A0C00511E88819981FC01E559F74F008102959F
:101A1C000F70F2011081100F108301E0400E00E0F6
:101A2C00501EFC01E559F74F00810295007FF20131
:101A3C0000830196FC01E559F74F008102950F7068
:101A4C00F2011081100F1083EDE9F4E0828D90E02B
:101A5C000496FB01008110E08017904091F5EDE9B0
:101A6C00F4E0818D90E00C968633904054F5418CD7
:101A7C005524480C591C0AE0400E511E8A819B814A
:101A8C00FC01E559F74F008102950F70F2011081AE
:101A9C00100F108301E0400E00E0501EFC01E559D0
:101AAC00F74F00810295007FF20100830196FC0143
:101ABC00E559F74F008102950F70F2011081100F5C
:101ACC001083EDE9F4E0828D90E00596FB01008136
:101ADC0010E08017904091F5EDE9F4E0818D90E0F5
:101AEC000C968633904054F5418C5524480C591C67
:101AFC000AE0400E511E8C819D81FC01E559F74F87
:101B0C00008102950F70F2011081100F108301E01B
:101B1C00400E00E0501EFC01E559F74F0081029584
:101B2C00007FF20100830196FC01E559F74F00811B
:101B3C0002950F70F2011081100F108300918E0F1F
:101B4C000023EDE9F4E0028DFB01108109F4F9C0EA
:101B5C00011799F5EDE9F4E0818D90E00C96863350
:101B6C0090405CF5418C5524480C591C0AE0400E01
:101B7C0000E0501E88819981FC01E556F74F0081E9
:101B8C0002950F70F2011081100F108301E0400ECE
:101B9C0000E0501EFC01E556F74F00810295007FD6
:101BAC00F20100830196FC01E556F74F0081029586
:101BBC000F70F2011081100F1083EDE9F4E0828DAB
:101BCC0090E00196FB01008110E08017904091F5A8
:101BDC00EDE9F4E0818D90E00C968633904054F55D
:101BEC00418C5524480C591C0AE0400E511E8A8128
:101BFC009B81FC01E556F74F008102950F70F201B5
:101C0C001081100F108301E0400E00E0501EFC010B
:101C1C00E556F74F00810295007FF2010083019693
:101C2C00FC01E556F74F008102950F70F20110810F
:101C3C00100F1083EDE9F4E0828D90E00296FB0129
:101C4C00008110E08017904091F5EDE9F4E0818D72
:101C5C0090E00C968633904054F5418C5524480CFA
:101C6C00591C0AE0400E511E8C819D81FC01E556E9
:101C7C00F74F008102950F70F2011081100F108345
:101C8C0001E0400E00E0501EFC01E556F74F0081CC
:101C9C000295007FF20100830196FC01E556F74F97
:101CAC00008102950F70F2011081100F1083EDE985
:101CBC00F4E0028DFB011081011709F030C310E034
:101CCC00EDE9F4E0418C5524480C591C018D03308E
:101CDC0020F00DEF400E0FEF501E48E155E000E0F4
:101CEC00E02FF0E0E40FF51F2081222309F417C345
:101CFC00222E332420E330E0329D302D239D300DF5
:101D0C00229D310D88819981800D931F0201112331
:101D1C00E0E0F9E109F0D5C2E80FF91F2491F201D6
:101D2C003081320F308321E0420E531CE0E0F9E1A8
:101D3C000196E80FF91F2491F2013081320F3083A4
:101D4C00E8C2011709F06AC010E0EDE9F4E0418C3B
:101D5C005524480C591C43EE54E000E0E02FF0E011
:101D6C00E40FF51F2081222309F458C0222E3324BE
:101D7C0020E330E0329D302D239D300D229D310D1E
:101D8C00C7010497880F991F800D931F020111231F
:101D9C00E0E0F9E1A9F4E80FF91F2491F201308198
:101DAC00320F308321E0420E531CE0E0F9E1019642
:101DBC00E80FF91F2491F2013081320F308328C0D3
:101DCC00E80FF91F249122952F70F0013081320F0A
:101DDC00308321E0420E20E0521EE0E0F9E1E80FF2
:101DEC00F91F24912295207FF2013081320F30832C
:101DFC00E0E0F9E10196E80FF91F249122952F708C
:101E0C00F2013081320F308321E0420E20E0521E6D
:101E1C0021E012270395073008F4A0CFEDE9F4E098
:101E2C00828D90E00196FB01008110E080179040BC
:101E3C0009F068C0EDE9F4E0418C5524480C591CBC
:101E4C0043EE54E000E0E02FF0E0E40FF51F2081BA
:101E5C00222309F457C0222E332420E330E0329D94
:101E6C00302D239D300D229D310DC701880F991FF8
:101E7C00800D931F02011123E0E0F9E1A9F4E80FB2
:101E8C00F91F2491F2013081320F308321E0420E90
:101E9C00531CE0E0F9E10196E80FF91F2491F201DF
:101EAC003081320F308328C0E80FF91F249122951E
:101EBC002F70F0013081320F308321E0420E20E090
:101ECC00521EE0E0F9E1E80FF91F24912295207FE2
:101EDC00F2013081320F3083E0E0F9E10196E80F36
:101EEC00F91F249122952F70F2013081320F30832B
:101EFC0021E0420E20E0521E21E01227039507300C
:101F0C0008F4A1CFEDE9F4E0828D90E00296FB019C
:101F1C00008110E08017904009F06AC0EDE9F4E010
:101F2C00418C5524480C591C43EE54E000E0E02F42
:101F3C00F0E0E40FF51F2081222309F459C0222E72
:101F4C003324E0E3F0E0F29DF02DE39DF00DE29DF3
:101F5C00F10D89859A850497880F991F800D9F1F15
:101F6C0002011123E0E0F9E1A9F4E80FF91F249133
:101F7C00F2013081320F308321E0420E531CE0E03D
:101F8C00F9E10196E80FF91F2491F2013081320F2B
:101F9C00308328C0E80FF91F249122952F70F0018F
:101FAC003081320F308321E0420E20E0521EE0E0FF
:101FBC00F9E1E80FF91F24912295207FF20130817D
:101FCC00320F3083E0E0F9E10196E80FF91F24911C
:101FDC0022952F70F2013081320F308321E0420EB6
:101FEC0020E0521E21E012270395073008F49FCF02
:101FFC00EDE9F4E0828D90E00396FB01008110E0A6
:10200C008017904009F069C0EDE9F4E0418C55244B
:10201C00480C591C43EE54E000E0E02FF0E0E40FD4
:10202C00F51F2081222309F458C0222E332420E3EB
:10203C0030E0329D302D239D300D229D310D898550
:10204C009A85880F991F800D931F02011123E0E0E0
:10205C00F9E1A9F4E80FF91F2491F2013081320F54
:10206C00308321E0420E531CE0E0F9E10196E80FC9
:10207C00F91F2491F2013081320F308328C0E80F10
:10208C00F91F249122952F70F0013081320F30838B
:10209C0021E0420E20E0521EE0E0F9E1E80FF91FCA
:1020AC0024912295207FF2013081320F3083E0E0C1
:1020BC00F9E10196E80FF91F249122952F70F20196
:1020CC003081320F308321E0420E20E0521E21E09D
:1020DC0012270395073008F4A0CF07E1202E3324F4
:1020EC000F811885201A310AEDE9F4E0828D90E019
:1020FC000496FB01008110E08017904009F06AC043
:10210C00EDE9F4E0418C5524480C591C43EE54E0A5
:10211C0000E0E02FF0E0E40FF51F2081222309F40A
:10212C0059C0E22FF0E020E330E03E9F302D2F9F8E
